:020000040000FA
:10000000C05C00201121000013510000E520000019
:10001000E5200000E5200000E520000000000000D1
:10002000000000000000000000000000491C00006B
:10003000E520000000000000E5200000E5200000B1
:10004000C51C0000C51C0000C51C0000C51C00002C
:10005000C51C0000C51C0000C51C0000C51C00001C
:10006000C51C0000C51C0000C51C0000C51C00000C
:10007000C51C0000C51C0000C51C0000C51C0000FC
:10008000C51C0000C51C0000C51C0000C51C0000EC
:10009000C51C0000C51C0000C51C0000C51C0000DC
:1000A000C51C0000C51C0000C51C0000C51C0000CC
:1000B000C51C0000C51C0000C51C0000C51C0000BC
:1000C000C51C0000C51C0000C51C0000C51C0000AC
:1000D000C51C0000C51C0000C51C0000C51C00009C
:1000E000C51C0000C51C0000C51C0000C51C00008C
:1000F000C51C0000C51C0000C51C0000C51C00007C
:1001000053B94AB9002908BF00281CBF4FF0FF317E
:100110004FF0FF3000F00CB8ADF1080C6DE904CEE3
:1001200000F008F8DDF804E0DDE9022304B07047D0
:10013000704700BF2DE9F04786468C460846089E6A
:10014000154674461946002B40F0C2808542B2FA2B
:1001500082F245D94AB1C2F1200300FA02FC2EFA1C
:1001600003F3954043EA0C0C94404FEA154EA8B2B5
:10017000BCFBFEF8230C0EFB18CC08FB00F943EA8D
:100180000C43994528D9EB1808F1FF3704D299455B
:1001900002D9A8F102072B44A3EB0903A4B2B3FBD5
:1001A000FEFC0EFB1C330CFB00F044EA0344A042AF
:1001B00014D92C190CF1FF3304D2A04202D9ACF1AE
:1001C00002032C44241A43EA07401EB1D440002302
:1001D00034607360BDE8F0874746DDE76346F1E7CA
:1001E00092BB431B01214FEA154EAFB2B3FBFEFC9D
:1001F000200C0EFB1C330CFB07F840EA0343984528
:1002000062D9EB180CF1FF3004D2984502D9ACF159
:1002100002002B44A3EB0803A4B2B3FBFEFC0EFBCD
:100220001C330CFB07F744EA0344A7424ED92C19B0
:100230000CF1FF3304D2A74202D9ACF102032C44E3
:10024000E41B43EA0040C0E7C2F1200320FA03F1B7
:10025000954090402EFA03F303434FEA154EAFB298
:10026000B1FBFEFC0EFB1C10190C0CFB07F841EA5D
:100270000041884504FA02F422D969180CF1FF30D4
:1002800004D2884502D9ACF102002944A1EB08014F
:100290009BB2B1FBFEFC0EFB1C110CFB07F743EA03
:1002A00001439F420ED9EB180CF1FF3104D29F425B
:1002B00002D9ACF102012B44DB1B41EA004192E779
:1002C0006046E3E76146F7E76046A3E76346B7E7C2
:1002D000834206D916B9002108467BE7C6E900E04B
:1002E000F9E7B3FA83F78FB9834201D3724508D88F
:1002F000BEEB020460EB030301209C461EB9002103
:1003000068E73846FAE7C6E9004CF8E7C7F1200C81
:10031000BB4022FA0CF41C432EFA0CF120FA0CF329
:10032000B84001434FEA14490EFA07F5B3FBF9F858
:100330001FFA84FE09FB18300B0C08FB0EFA43EA87
:1003400000439A4502FA07F240D9E31808F1FF305A
:1003500004D29A4502D9A8F102002344A3EB0A0370
:1003600089B2B3FBF9F809FB183308FB0EFE41EA2A
:1003700003418E452CD9611808F1FF3304D28E4514
:1003800002D9A8F10203214443EA0040A0FB0298ED
:10039000A1EB0E014145CE46434602D306D14D4561
:1003A00004D2B9EB020E68EB04030138002EA6D08C
:1003B000B5EB0E0261EB030101FA0CFC22FA07F324
:1003C0004CEA0303F940C6E9003198E74046C5E727
:1003D0004346D9E7F0B52D4B2D4AC3F800262D48EA
:1003E000C3F8042685B0C3F808264921C3F80C26B3
:1003F000C3F81026C3F81426C3F81826C3F81C2621
:1004000004F003FE00F074F801A800F0D5FC224BC4
:100410001B68834204D02148452104F0F6FDFEE725
:10042000039A1F48492104F0F0FD1E48492104F0B9
:10043000ECFD4FF44041002005F0E8F8044620B1FF
:100440001948452104F0E1FDFEE769469DF80800E2
:1004500000F02EF8009B039D1D44019B1E8900F0B7
:1004600089FFAF1900F05CFF01F07CFEAB5983F30C
:10047000088884F31488BFF36F8FBFF36F8F7B6896
:1004800098470A48452104F0C0FDFEE700000140FE
:100490003546526E54770000900100206D770000C1
:1004A00090770000BF770000E47700001778000025
:1004B00008B5024638B105480023452104F0A5FDE2
:1004C0006FF0150008BD0860FCE700BF3A78000037
:1004D0001FB50C46014601AA044804F07FFF18B975
:1004E000019B2360029B636004B010BD1872000082
:1004F00002484FF4C05103F071B900BF580F0020FB
:100500002DE9F04FF9B0DDE98448DFF8E0A138A823
:10051000DAF8006017461D4606F024FC002138A8D2
:1005200003F07AFA3CB1B8F1000F04DD42462146EF
:1005300038A806F01BFC7B89B7F808809844FB6854
:100540004FF000099844C84521D80DA938A806F0F5
:1005500046FC869B23B120220DA9184604F001FE1B
:10056000002300932A464FF6FF73394607A804F08C
:10057000FDF9044638B928460C9F00F0DDF98742A2
:100580001BD94FF0FF34204679B0BDE8F08F839B34
:10059000829AA8EB090B9B4528BF9B465B464946C0
:1005A000284604F040FD04460028ECD182995A46C2
:1005B00038A806F0DBFBD944C5E7DFF834914FF0EB
:1005C000FF370DF1160305AA06A907A804F01CFAC7
:1005D000B0F10008C0F288807BD1BDF816B0BBF145
:1005E000100F18D1BDF81440202CCAD1069923460B
:1005F00038AA284604F017FD8046002874D1224608
:1006000038A90DA804F04CFA04463A4B1B68834203
:10061000B9D10124D5E7BBF1010F37D1BDF81430B2
:10062000202BAED8069938AA284604F0FCFC804658
:10063000002859D19DF814B0BBF1200F03D94FF019
:10064000FF384746BDE7D9F800302B4F0393039B93
:100650009845F4DA1DA806F085FB00211DA803F0DB
:10066000DBF97A6857F8081B12681DA806F07EFBB4
:1006700015A91DA806F0B3FB5A4638A915A804F021
:1006800060FD0028DDD008F10108E0E7BBF1200F94
:1006900097D17B1C95D0D9F80030BB4216DDBDF850
:1006A0001430B3F5807F7FF46CAF069938AA2846E2
:1006B00004F0B9FC8046B8B9FFB2BDF81430009719
:1006C00038AA59460DA800F019F806464FF0FF3732
:1006D00077E73CB1074B1B68B34218BFDAF80060FC
:1006E000344650E74FF0010844464CE70000002034
:1006F00048740000900100204C7400002DE9F04F78
:100700001F46ADF54B7D6A4B9DF850631D688046D2
:1007100027A88A46914606F0E2FA664B53F836401F
:10072000029403EBC6038AAA5B681B681C4421463B
:10073000302302A805F066F868BB029B8A9A13442E
:100740009C4228D129AA214602A805F06FF810BBC7
:100750000DF1B00B5A46214602A805F067F806468F
:10076000C8B929A805F083FB029B28909C4212D1AE
:10077000CDE9006B3346324629A927A806F06CFA6A
:1007800048B927A803F0DAF828B929A805F06FFBC3
:10079000874228900AD027A806F0ABFA27A806F0CF
:1007A000A8FA28460DF54B7DBDE8F08FB7F5807FA0
:1007B00002D04FF0FF35F1E7BAF1200FF9D18AAA44
:1007C000494627A803F0E0F804460028F1D19DF837
:1007D0002733BC2BEDD152AF0390DF263D460CA84A
:1007E00006F0C0FA00210CA803F016F920220DF241
:1007F00007310CA806F0BAFA042203A90CA806F0E7
:10080000B5FA04A90CA806F0EAFA202E9DF80F30DC
:10081000B146A8BF4FF02009013338464A4604A923
:10082000A6EB09068DF80F3004F09BFC002E4F4418
:10083000D5DC2F468AAB29460022087813F8016BD5
:1008400001327040DF2A01F8010BF6D12B7803F05A
:100850007F032B7017F8016B002EAAD10134BE2C38
:10086000F8D195F8BE30012BA3D10CA806F07AFA86
:1008700031460CA803F0D0F80F4908220CA806F066
:1008800075FA414620220CA806F070FA20220DF2DB
:1008900007210CA806F06AFA04A90CA806F09FFA32
:1008A00020220DF2073104A804F0FAF8054682E789
:1008B000000000204C740000607800002DE9F04139
:1008C00086B00223DFF86C80ADF800300D466F462D
:1008D000002617F8010B01A901F0CAF80446A0B9D7
:1008E00001988168102302AA103904F09CFB044689
:1008F000019804F097FB44B91022414602A804F085
:1009000020FC40B12EB14FF0FF34204606B0BDE8C8
:10091000F0810126DDE7019804F07BFE0423A0F1BD
:1009200008012A46019804F07EFB0446019804F071
:1009300079FBEAE74477000007B504F0C5F869469B
:10094000FFF7C6FD38B10548452104F05EFB0020E5
:1009500003B05DF804FB0098FAE700BF6878000078
:100960002DE9F041354B88B0064600200C461D6845
:1009700003F0F1FF06A9C0B201F07AF8002857D1C0
:10098000214603F0E8FF2C2507A9C0B205FB04654A
:1009900001F06EF8002833D02C27674306EB0708D8
:1009A000069BD8F8101011F0100138D14FF4807266
:1009B0000192234A0092CDE903112A46029108468A
:1009C000FFF79EFD05461F4BF25906989A420CD13F
:1009D000D8F80C20B8F808309B1806D282689342E9
:1009E00003D2194B1B68AB421FD02CB38268002185
:1009F00004F043FB154A1648452104F006FB13E0BA
:100A0000079804F055FB0746079804F00BFB6B1E94
:100A1000EA1C13F8011FB942BED19342F9D11CB1AF
:100A20000699304604F034F90125069804F0FAFAE4
:100A3000284608B0BDE8F081064ADCE70000002047
:100A4000582700203DB8F39690010020AB780000B5
:100A5000B5780000A378000073B50D460446002168
:100A60002846CDE9001104F0D2F830B3164E2368C1
:100A7000B34203D101AA204604F05EF8E36AB34210
:100A800004D16A460121204604F056F8DDE900321F
:100A9000934288BF0193019BAB60019A294620468F
:100AA00000F034FB094B1A68002A03DD084857217F
:100AB00004F0ABFA002002B070BD05F10801FFF7A9
:100AC000FDFEAB680193E8E73DB8F396F40D002016
:100AD000DD7800002DE9F84FDFF870B01C4C1D4D9B
:100AE000884691469A4600260B9B9E4201D30020E1
:100AF0000FE00B9B154A9F1BB7F5806F28BF4FF483
:100B000080673B4606EB0A01404604F08CFA10B1C0
:100B10000120BDE8F88F0A993B465A4671184846AD
:100B200004F096FA0028F3D1C4F800563E44C4F805
:100B30000456C4F80856C4F80C56C4F81056C4F845
:100B40001456C4F81856C4F81C56CDE79409002072
:100B5000000001403546526E2DE9FF418F4B436244
:100B60000E468F4B036500210446084603F0F3FE52
:100B700004F12001C0B200F07BFF0121002003F04E
:100B8000EAFE04F14C01C0B200F072FF05462046B7
:100B900004F013F8074668B900221146204603F016
:100BA000B5FF074600B37F480022572104F02DFA15
:100BB00001238FE07C488022572104F026FA01238C
:100BC0009F4284F85830E7D194F858308DF80730B8
:100BD000042B00F28280012B00F2858000F09C80C3
:100BE000FF2384F8583097E0204600F0A7F900284A
:100BF000DED0684604F002F86946204604F09DF80D
:100C000018B16A483A465721D0E7684603F0FFFF1B
:100C100080F001016A46C9B2204603F077FF024620
:100C20000028C0D1684603F0F2FF074660BB694662
:100C30002046FFF711FF9DF8073084F85830033B3A
:100C4000012B06D8384604F0C6F810B1FF2384F80B
:100C500058309DF80730023B022B0BD8002004F0DF
:100C6000A8F838B1FF2384F858305148452104F0E2
:100C7000CCF9FEE794F85830FF2BF6D06A460021F5
:100C8000204603F043FF93E79DF80780B8F1010F7A
:100C900015D1104602F0D2FB831E022B07460BD85B
:100CA00041462046FFF75CFE424B1B68984203D04A
:100CB000012814BF0527012784F8587084E7012113
:100CC0002046FFF74DFE3B4B1B6898420CBF9DF83A
:100CD0000730052384F8583076E7052B80D10020B3
:100CE00004F079F813E069462046FFF7B5FE94F862
:100CF0005830DA1E012A05460CD8002004F06BF8A3
:100D0000054600287FF46CAF002004F052F8054639
:100D100010B165E7022BF7D094F85830FF2B04D1BF
:100D20002348452104F071F9FEE7012B10D06A46F3
:100D30000021204603F0EAFE054648B1E06C04F0CD
:100D400071F9206A04F06EF9284604B0BDE8F0811C
:100D500000212046FFF704FE0746DFF85880D8F848
:100D6000003098420FD110220021684604F004FAA6
:100D7000206A03F0F9FD3071236A5B683460D8F8AB
:100D80000050B360DAE7E06C04F04CF9206A04F03C
:100D900049F9002D08BF3D46D6E700BF9405002065
:100DA000940100204E7900000C7900007A7900004F
:100DB000A47900009001002038B5064D0446602259
:100DC0000021284604F0D8F921462846FFF7C4FE42
:100DD00038BD00BF940D002073B516461D4643B1C3
:100DE0005B79012B07D121B9204B2A681B689A42F5
:100DF00017D8002418E0022BFBD12B68012B07D950
:100E00001A4A12689342F4D8B1FA81F14909F0E71D
:100E1000EFD131B10129ECD12979023918BF012173
:100E2000E7E7436A5C680021002003F094FD01A914
:100E3000C0B200F01DFE30B10124019804F0F2F8B8
:100E4000204602B070BD214601982023324604F0AE
:100E5000EAF804460028EFD1002DEED03468044BA8
:100E6000E41A18BF4FF0FF34E7E700BF040000208A
:100E70003DB8F3962DE9F04F074685B00C46014684
:100E80000020164603F013FE051E50DB3846E46DC5
:100E900003F01AFE5FFA84F96B1E09FB03084FF09A
:100EA000000A4FF0010B4FF0FF349DB9BAF1010F6A
:100EB00003DD2148452104F0A8F8631C06D07F2CEF
:100EC0002ADC013440F201133460B380284605B0B7
:100ED000BDE8F08F6B1E00930DF10F020123414618
:100EE000384604F0A0F8031E019322DB01220DF125
:100EF0000F01384604F0A1FB019B40B15B4501D0D6
:100F00000AF1010A009DA8EB09089B46CDE7B4F160
:100F1000FF3F08BF2C46F5E70223803C7371631046
:100F200004F001040133013433603471CEE7072546
:100F3000CCE70125CAE700BFB079000038B5816A67
:100F4000426D914208D0531C8B4205D01348572163
:100F500004F05BF8002038BD80291CD910485721C7
:100F6000F6E7446A056D04EBC30405EBC30564684A
:100F70006D68AC4202D00B485721E9E701339A4231
:100F8000EFD1914205D9436A03EBC2035B68A342E8
:100F9000F1D10120DFE700231C46F0E7D379000000
:100FA0000B7A00003A7A000000B589B004A902204B
:100FB00004F0B5FB9DF81020012A41D0254B2649AD
:100FC000032A08BF0B469DF8132002929DF81220B9
:100FD00001929DF81120214800924921204A04F0F5
:100FE00014F806A9052004F09AFB9DF81820012AA0
:100FF00028D0184B1849032A08BF0B469DF81B2020
:1010000002929DF81A2001929DF81920009213482F
:10101000144A492103F0F9FF9DF81030012B13D138
:101020009DF81230032B0FD19DF81830012B0BD0F7
:101030000D48492103F0E9FF022009B05DF804FBE7
:101040000A4BC0E7094BD9E70948492103F0DDFF06
:101050000020F2E7667A00006F7A0000837A0000D1
:10106000757A0000C47A0000D47A00006A7A000021
:10107000F37A000070B54B6814461E4A03F0FF2354
:10108000934286B006460D462FD10B68012B2CD11A
:1010900004A9204602F07CF99DF81020012A26D0F0
:1010A000154B1649032A08BF0B469DF813200292E0
:1010B0009DF8122001929DF8112000921048114ACB
:1010C000492103F0A2FF9DF81030032B0DD12146DA
:1010D000304603F0DDFD204604F014FBA9682046ED
:1010E00003F005FD204602F033F906B070BD064B53
:1010F000DBE700BF00010004667A00006F7A0000A1
:10110000837A0000C47A00006A7A00002DE9F04F6B
:10111000054689B07D480C464921174603F075FF06
:101120006B6A01225E6800233344BB42114602F120
:101130000102F9D3764F2046396003F068FD08B309
:10114000E86D03F0AFFCAB6A03F1FF3800233344D2
:10115000834202D208F1FF38F9E73B68434511D3D7
:101160006C48572103F051FF3A686B4808FB06F3BF
:1011700002FB0662572103F048FF0123E37109B027
:10118000BDE8F08F06A9022000F072FC07A9052037
:1011900000F06EFC079A21462846FFF76BFF637943
:1011A000012B0BD1D7F80080DFF870B13B68DDF878
:1011B0001890B8F1000F11D101232360022363714D
:1011C0004FF001083B68DDF818A0984549D9504612
:1011D00003F028FF079803F025FFD0E722680133CA
:1011E0009B1A98453AD86B6A196853F8380003EB94
:1011F000C803012A53F8083CA3EB0103A0EB010A42
:10120000049311D1079B0393E368022B08D049464E
:10121000284603F03DFD22464946284603F06EFD70
:101220000399284603F034FD32465146484603F000
:101230002DFD049B4A464946CDE900A62846FFF706
:1012400049FC2146284603F0EFFC23680133236064
:1012500020B1DBF800300133CBF8003008F1FF3863
:10126000A4E7236898454ED36A6ADDF81CB052F8AB
:10127000381004914FEAC803083B11680391D15814
:101280002A6DD0581368A0EB03092379012B38D1BC
:10129000039B3246C91A5046059103F0F7FC0599A5
:1012A00000914B465246594601962846FFF712FCDC
:1012B0002146284603F0B8FC0223237118B1174ACF
:1012C00013680133136032464946584603F0DEFC8A
:1012D000DDE9032351469B1ACDE900965A4628467C
:1012E000FFF7F8FB2146284603F09EFC23680133F4
:1012F00023600123237130B1084A1368013313605E
:1013000001E0022BDFD008F101085BE70A7B000057
:1013100004000020337B0000627B0000F40D0020FD
:10132000BFF36F8F72B6124B4FF0FF32C3F88020BD
:10133000C3F88420C3F88820C3F88C20C3F8902019
:10134000C3F89420C3F89820C3F89C20C3F88021E8
:10135000C3F88421C3F88821C3F88C21C3F89021F5
:10136000C3F89421C3F89821C3F89C21704700BFAB
:1013700000E100E0164A4FF0FF3301215160C2F84E
:101380004833C2F8083302F5C0425160C2F848330E
:10139000C2F8083302F598325160C2F84833C2F8F7
:1013A0000833A2F508320021C2F80015C2F808334C
:1013B00002F51832C2F80015C2F80833A2F510423F
:1013C000C2F808354FF08042C2F80833704700BFBA
:1013D00000B00040014B1B68184700BF0800002008
:1013E000014B1860704700BF0800002007B50B468E
:1013F000002102460091034800F014F903B05DF8A3
:1014000004FB00BFD51300002DE9F047058B04460F
:101410002807904611D4022905F0070540F0CD8039
:10142000204603F018FD78B10138218B042811D82B
:10143000DFE800F0C3106D85950001290CBF45F071
:10144000100545F02005258388F31188BFF36F8FC1
:10145000BDE8F08701F0070AAA4500F0A680002742
:10146000B9463E46A368002B00F0BD8041F008015C
:10147000218388F31188BFF36F8FA168002900F0E2
:10148000BB800D68002900F0B780D1F80480334696
:1014900052462046C047002D76D02B6829461D466F
:1014A000F0E701F007035A1F012A1BD8002221F0A0
:1014B0000701062B276889B2C4E9002209D13B46FF
:1014C00003E0628B013262831B68002BF9D141F08B
:1014D00002012183204603F0BEFC00287BD041F0AE
:1014E000200177E0042B0AD121F0070189B2218382
:1014F000204603F0B0FC10B141F020012183218B84
:1015000001F0070AAA4550D00027B946AAE7236987
:1015100021F0070141F00601062DD3F80090218348
:101520002DD1B9F1000F40D041F00801218388F39B
:101530001188BFF36F8F3A492046C84729E021F050
:101540000701236941F0040189B2042DD3F8049006
:101550002183E6D000273E464FF0040A82E721F0BF
:101560000701236941F0050189B2052DD3F80890E0
:101570002183D6D000273E464FF0050A72E70027A8
:101580003E464FF0060A6DE72B4687E7B9F1000F9C
:10159000D1D14FF02003EFF3118883F31288BFF30A
:1015A0006F8F238B23F008032383258BEA062ED528
:1015B00025F01003238305F007056669218B002EB3
:1015C000BFF66FAF00232768C4E9003321F007019D
:1015D00041F001012183218B01F0070AAA454FF058
:1015E00000097FF43FAF002F9BD041F00801218319
:1015F00088F31188BFF36F8F002FC7D03D6839463D
:1016000033465246204603F052FC2F46F4E7AB0621
:101610007FF51AAF25F02003238305F00705FFE6C9
:10162000DB4E00002DE9F04F8DB01D46531E824663
:10163000019103934FF00009039B5878252803F18B
:10164000010419D11E4600204FF0FF380236034630
:101650000290444631780396392954D81F2914D86A
:10166000002900F0F08101992520D04701993078B8
:10167000D04709F10209DFE7002800F0E481019971
:10168000D04709F101090394D6E7A1F12002192AF4
:10169000E9D801A757F822F00117000067160000EB
:1016A0006716000001170000671600008117000090
:1016B0006716000067160000671600006716000036
:1016C000CD1700000117000067160000E1170000A9
:1016D0008D170000671600009B170000BB17000065
:1016E000BB170000BB170000BB170000BB170000B2
:1016F000BB170000BB170000BB170000BB170000A2
:1017000008460136A6E7582900F0EE80A1F16302F1
:10171000D7B2172FA7D8172AA5D801A757F822F0B4
:101720008F190000071800006716000067160000F8
:1017300067160000E7170000071800006716000092
:1017400067160000E7170000671600006716000024
:1017500067160000C3180000671600006716000037
:1017600063190000671600000718000067160000E4
:1017700067160000C318000067160000E717000096
:1017800001992520D04709F1010955E7029A02F095
:10179000FE0202924FF00008B3E7002C0DDAB8F118
:1017A000000F0DDA029A002A00F0458124EAE47461
:1017B0000A2202FB0414303CA3E7B8F1000FF5DB6A
:1017C0000A2202FB0812A2F130089AE7B8F1000FD2
:1017D00055F8042B80F23181002A80F23081544286
:1017E000022202928DE7682903D1682B06D1482393
:1017F00087E76C2902D16C2B00F02381002B7FF44A
:1018000032AF0B467DE77A2B06D1752955F8046B6C
:1018100014D14FF0000B0CE06C2BF6D04C2BF4D114
:10182000073525F007037529D3E9006B03F1080597
:1018300006D120283ED1864F013C09E04FEAE67BE5
:10184000BBF1000FF5DA7642824F6BEB4B0B013C9C
:101850000DF12D03059300230493304659460A22C7
:101860000023FEF74DFC049B03F1FF3CCDF810C0B4
:10187000DDF814C030320CF8012DCDF814C0B44698
:101880005A46BCF10A0F72F1000206468B46E4D2BA
:10189000C3F1010B30330DEB0306B8F1000FA6F1D5
:1018A00004066DDA029BD9077CD4A8EB0B03A4EBEA
:1018B0000B0413E02B280ABF674F684F04F1FF3475
:1018C000C6E770290FD155F8042B0023FAB9644EEE
:1018D000053C6FF004034FF0050B604F029A92072E
:1018E0006FD4A04665E078216C2B03D155F8042B0A
:1018F000002308E04C2BF9D1073525F007031D46DE
:101900005B6855F8082B232825D1880621D5554F2B
:10191000023C01F06001A1F1390B0DF12D0E002602
:1019200002F00F01092988BF594430310EF8011D1A
:10193000102A4FEA121141EA03714FEA131073F1B2
:10194000000306F1FF3C08D2C6F1010B06F130039B
:10195000A1E7454FDCE7414FDBE766460A46034611
:10196000DEE755F8046B304603F0E4FBB8F1000FF6
:10197000834602DB4045A8BFC346384F4FF00008FE
:10198000A8EB0B03002B92DDA4EB0804A6E755F8A7
:10199000043B8DF81830013C4FF0FF334FF0010B42
:1019A00006AE9AE7A046EBE7029301992020D047C4
:1019B000029BB8F10108F7D524EAE472013C914496
:1019C000A41AB84606E0049302920199D047029AFD
:1019D000049B9046424612F8010B0028F3D11A46A8
:1019E000013A15D5002BACBFC7EB03077F425B461E
:1019F000013B15D5BBF1000FA8BF5F444F442646FD
:101A0000013E14D5002CA8BF3F1907EB080913E6C7
:101A10000493029201993020D047049B029ADFE799
:101A20000293019916F8010BD047029BE0E7019958
:101A30002020D047E4E70122D3E6904661E6144631
:101A40005FE64C235DE648460DB0BDE8F08F00BF71
:101A50002E800000B27C0000B47C00002E840000C8
:101A6000BC7C0000B67C0000B97C000002F0E2B84B
:101A700070B5114B1C680D46DCB1104B1968002382
:101A80008B4202DB6FF0010070BD224612F8106B32
:101A9000864202D001331446F2E7E06810B96FF0D5
:101AA0001200F1E705F033FB0028F8D02C6000208D
:101AB000EAE76FF00C00E7E70C0000205874000024
:101AC00070B588B005460C46C0B269461646FFF7A9
:101AD000CFFF00281BDB0098C8B1436802938368DE
:101AE00022680195CDE903360023CDE9062305934D
:101AF000C56803F097FA6DB12846084901AA03F0BA
:101B000071FC079808B9059B236008B070BD6FF0A1
:101B10001500FAE76FF01200F7E700BFBF500000B2
:101B2000014910220A60704710ED00E072B649408A
:101B300081F31188BFF34F8F20BF80F3118862B605
:101B4000704700BF37B505460C46C9B18B68009396
:101B5000D1E900230E48452103F057FA6369009349
:101B6000D4E903230B48452103F04FFAE2690A4800
:101B7000452103F04AFAA2690848452103F045FAD5
:101B80002146284603B0BDE8304002F061BD00BFE9
:101B9000C27C0000F67C00002A7D00003E7D000033
:101BA00040B2002807DB044A4109012300F01F006E
:101BB000834042F82130704700E100E0054B4209C4
:101BC00000F01F0053F82220012303FA00F0104018
:101BD000704700BF00E100E040B20028A8BF00F15C
:101BE000604001F10101B8BF064B4FEA4111ACBFA3
:101BF00000F5614000F00F00C9B2B4BF195480F87D
:101C00000013704714ED00E030BFFFF7FDBF00BFC9
:101C10000B4A08B50B4B22F07F029A60BFF34F8F3F
:101C2000BFF36F8FD3F8882022F47002C3F88820A6
:101C300002F086FD02F0CCFD00F05EFA02F08CFDB1
:101C40000000000000ED00E01EF0040F0CBFEFF3F9
:101C50000880EFF30980816911F8021C0229FFD086
:101C600001B503F04EFA01BD10F1160F074B08D075
:101C7000984208D34033834205D98B4203D90448A4
:101C800070474033F9E70020704700BFC0340020A0
:101C90000035002004462025084611461A46084B08
:101CA00083F3098863B64FF0000383F31188BFF311
:101CB0006F8FA04785F31188BFF36F8FFEE700BFDA
:101CC000005D002001B5EFF30580A0F110004FEAA0
:101CD000C0000449014409C99847BDE801400249D0
:101CE0000847000030720000ED1C0000704700BF84
:101CF0002DE9F041324C07468846324845211546C9
:101D000003F083F9A36ADE0603D52F48452103F0CB
:101D10007CF9A36A180703D52C48452103F075F90F
:101D2000274CA36A990728D46FF01506244CA36AA0
:101D3000DB0703D52648452103F067F9A36A9C0613
:101D400003D52448452103F060F91D4CA36AD80649
:101D500028D4A36A990725D40020A36A184A9B06B1
:101D600042BF636A23F400536362936A43F0FF0344
:101D7000936200232B70BDE8F0811748452103F0E2
:101D800044F9666BA36A1A06CED51448324645213B
:101D900003F03BF9B8F1000FC8D0A36A23F0800329
:101DA000A362C3E763681A05D6D539463046FFF704
:101DB0005BFF0028D0D080F309880220CDE700BF68
:101DC00000ED00E0717D00008C7D0000C47D00000E
:101DD000147E0000387E0000DC7D0000F97D0000EC
:101DE00010B51D4C1D48452103F00FF9A36A9B0156
:101DF00003D51B48452103F008F9A36ADC0103D58C
:101E00001848452103F001F9134CA36A180303D5C0
:101E10001548452103F0F9F8A36A590303D513487F
:101E2000452103F0F2F80C4CA36A9A0303D510483D
:101E3000452103F0EAF8A36ADB0303D50D484521E9
:101E400003F0E3F8044A936A6FEA03436FEA13432B
:101E50009362002010BD00BF00ED00E06C7E00002A
:101E6000897E0000A17E0000C07E0000E37E0000AD
:101E70000D7F00002C7F000070B5234C06460D46F8
:101E80002248452103F0C1F8A36AD90403D52048AC
:101E9000452103F0BAF8A36A1A0503D51D48452168
:101EA00003F0B3F8184CA36A9B0510D51A484521D6
:101EB00003F0ABF8A26BA36A180408D517484521B4
:101EC00003F0A3F81EB1A36A23F40043A3620E4CEF
:101ED000A36A590503D51248452103F096F8A36A71
:101EE000DA050BD50F48452103F08FF8064A936AAF
:101EF000002043F47F439362287070BDA36A9B0463
:101F0000F4D509484521EFE700ED00E05C7F0000D3
:101F1000777F0000C47D00008D7F0000AB7F000054
:101F2000C57F0000E57F0000387E00002DE9F0410C
:101F30005D4B5F688AB00546C7F30804002686F348
:101F40001188BFF36F8F02F07F43B3F17F4F07D14A
:101F500002F00C03082B14D15448452103F055F826
:101F6000002635464FF00008E31E8DF80780092B48
:101F700000F28780DFE803F00A7A7E768585858522
:101F8000858210074CBF0D460126EBE74848464CBA
:101F9000452103F03AF88DF80780E36A9A0705D5E2
:101FA0004448452103F031F8002433E0E36A002B74
:101FB00002DA41484521F5E7E36A5B00F4D53F4882
:101FC000452103F022F86369AA6943F480736361D1
:101FD000BFF34F8FBFF36F8F636932F8022C23F486
:101FE00080736361BFF34F8FBFF36F8F4DF6027342
:101FF0009A4209D0A36ADBB233B30DF10702012183
:102000002846FFF775FE2FE02A682D48452102F08B
:10201000FCFF2C689DF807309BB92022294602A8B6
:1020200003F09FF8099B002E38D0C3F3080222B9B1
:102030006FEA53236FEA4323099302A92046FFF76F
:1020400081FD0AB0BDE8F081A36A13F47F4F05D08B
:102050000DF107010120FFF70FFF05E0A36AB3F5BB
:10206000803FA1D3FFF7BCFE0446D3E70DF1070282
:102070000021C5E70DF107010020ECE711484521DB
:1020800090E71149114A124817F4F87F08BF0A4631
:10209000A4F11003452102F0B8FF85E723F4FF7394
:1020A00023F00103C8E700BF00ED00E0308000002E
:1020B000608000007C800000A2800000B5800000ED
:1020C000D9800000FA800000028000001780000024
:1020D00023810000024A536943F0100353617047A3
:1020E00000ED00E0EFF30880EFF3098101B57246DF
:1020F000FFF71CFF01BD00BF044800232021C218C8
:102100000133302B82F80013F9D1704700E100E071
:10211000002080F31488BFF36F8FFFF7A7FC002027
:102120000D490860BFF34F8F0C4880F3088800F01A
:102130002BF8202080F3118809484FF404614018DF
:1021400080F30988EFF314800221084380F3148898
:10215000BFF36F8FFFF75CFD94ED00E0C05C0020E3
:10216000802C00200749D1F890200023C2F30722D9
:102170001846934200DB7047C1F89830C1F8A000C0
:102180000133F6E700ED00E008B572B6002383F3F3
:102190001388FFF7E7FF144B4FF0FF32C3F880209E
:1021A000C3F88420C3F88820C3F88C20C3F890209B
:1021B000C3F89420C3F89820C3F89C20C3F880216A
:1021C000C3F88421C3F88821C3F88C21C3F8902177
:1021D000C3F89421C3F89821C3F89C2162B6BFF3D9
:1021E0004F8FBFF36F8F08BD00E100E0024B034A41
:1021F0000348022100F06CB800000220000000201B
:10220000CC740000F8B5244E00258D420FDA4468E6
:10221000002C3ED09BB104F1FF3C14EA0C0F08D017
:102220001E482A46452102F0F0FE6FF015021046C6
:10223000F8BD1F2CF4D907681CEA070FF0D1202C39
:102240000768D0F808C05FFA82FE10D9B4F1004FD9
:102250000FD8013CB4FA84F4C4F11F046400BEF149
:10226000070F4CEA040C06D90D484521DBE708248A
:10227000F5E73E24F3E727F01F04144344F010046D
:10228000C6F89820C6F89C404CF00104C6F8A0405F
:10229000013201350C30B8E700ED00E03F8100006D
:1022A00067810000044B0522C3F89420BFF34F8FD1
:1022B000BFF36F8F704700BF00ED00E0BFF35F8F8B
:1022C000024B0022C3F89420704700BF00ED00E0ED
:1022D00010B5034C01232278FFF794FF207010BD46
:1022E0005828002014490868082810B521D8FFF79D
:1022F000E5FF124C49680022904201F10C0105D122
:102300000F4B1870FFF7CEFF002010BDC4F89820C7
:1023100051F80C3C23F01F03134343F01003C4F89F
:102320009C3051F8043C43F00103C4F8A030013262
:10233000E2E74FF0FF30E8E7E474000000ED00E072
:1023400058280020014B1860704700BF1000002083
:102350004FF02003EFF3118283F31288BFF36F8FE6
:1023600006490123C1F840354FF08041C1F8783566
:1023700082F31188BFF36F8F0020704700E00140A7
:102380004FF08043C0B2C3F81C05BFF34F8F05491F
:10239000054BCA6802F4E0621343CB60BFF34F8F72
:1023A00000BFFDE700ED00E00400FA0520B1034B9B
:1023B000800143F001031847704700BF40740000DC
:1023C000084B70B5C31A0D4607499B100446594384
:1023D0000648402202F0F8FE2B4601462046BDE8A2
:1023E000704018470C0E0020B76DDBB6A0710000DE
:1023F00073B50C4C0C4A4023041B00930D460B464E
:102400000A49A41061430646094802F009FF011E6B
:1024100005DA30462B4602B0BDE87040184702B0DE
:1024200070BD00BF0C0E002091520000B76DDBB6EE
:10243000A071000010B54FF02003EFF3118483F377
:102440001288BFF36F8F074A136823F00201DB077E
:10245000116002D4012004F0EAFD84F31188BFF377
:102460006F8F10BD5C0E0020002270B50121044664
:102470001046FFF7B1FB0F4801F0CAFC0E4B984223
:1024800015D104F08BFD26690C49304602F033FD6E
:1024900000280BDB012535642469084904F11C0080
:1024A00002F029FD002801DBE564002070BD6FF01B
:1024B0000400FBE7F52400000000AD0B04750000EC
:1024C00070B501460C2309484B43C418D4E90E5695
:1024D00000224033A263184402F063FE2DB132465D
:1024E0002B460348BDE87040184770BD0C0E002015
:1024F000A071000010B1012804D07047034B1B6C81
:102500005B0701D1FFF7DCBF704700BF0C0E002056
:1025100008B54FF02003EFF3118183F31288BFF366
:102520006F8F124A136843F002001060DA0708D474
:1025300081F31188BFF36F8F0120BDE8084004F0DC
:102540003ABD4FF08043D3F80C24D3F80C34D307B2
:10255000EED5074802F025FE81F31188BFF36F8F97
:102560000020BDE80840FFF7ABBF00BF5C0E0020B5
:102570004C0E00202DE9F8433649BFF35B8F074628
:10258000012251E8003F41E800200028F9D1BFF3C3
:102590005B8F33B9304931484B60CB608A6002F0C1
:1025A000BDFC7B1E012B2DD8012F07D14FF080439E
:1025B000D3F81C3403F00303012B23D004F0B6FD41
:1025C000054608BB264B1B78F3B14FF0804302222F
:1025D000C3F808230646DFF88C904FF080444FF094
:1025E0000108D4F81834D4F81824D20316D503F00F
:1025F0000303012B01D0012F10D12DB386F31188D5
:10260000BFF36F8FBDE8F8834FF02003EFF311861F
:1026100083F31288BFF36F8F0125DCE73046FFF7A5
:1026200085FAD4F81835002BDBD1D4F80421002A20
:10263000D7D0C4F80431D4F80431C4F81885C9F8E7
:102640008081C4F80880CCE74FF080430222C3F8B1
:102650000423D7E7080E0020F80D0020280E0020E4
:102660006D2C002000E100E008B5074804F04FFDA4
:1026700038B10648FFF766FE0448FEF7B1FE0020B9
:1026800008BD6FF01200FBE7007200009126000009
:102690000A2838B5074D044604D1AB680D215B68A4
:1026A00028469847AB6803485B68E1B298472046E4
:1026B00038BD00BF0072000030B54068057B01F0F6
:1026C0001F04B2F5001F85B044EA451405D1204629
:1026D00001F01EFE002005B030BD0025B2F5800FD0
:1026E000CDE9025514D1B3F1007F0CBF04230523BB
:1026F0008DF808300023194602AA204601F046FC56
:102700001F4B984239D10121204601F0B9FDE1E784
:10271000B3F1C06F26D0B3F1007F14BF01230223B1
:102720008DF808308368CB40D907E3D4B2F1A07F9D
:10273000E0D16209012A04F01F03124A03F5E07395
:1027400018BF4FF0A04252F82330DB07D2D40DF16E
:1027500007052946204601F03FFD0B4B984203D068
:102760000395C7E70323DBE7284601F083FD044B0D
:102770009842F5D06FF00B00ADE76FF01500AAE7B7
:102780000000AD0B000300500400AD0B10B501F0CC
:1027900061FD044668B901F035FD084B98420AD145
:1027A0000748214601F012FD224605210620FFF7C9
:1027B00013FA002010BD6FF00400FBE70000AD0B22
:1027C000C5270000420970B5034602D0012A17D080
:1027D00070BD0D4E326951680029F9D003F01F0316
:1027E00001250C689D400029F2D08A682A4002D059
:1027F0004B68304698472CB1236821461C46F2E7C7
:10280000024EE7E72346F8E7D0710000B8710000F8
:102810002DE9FF4147683B7B01F01F0545EA431561
:102820000E4628460DF10301144601F0D5FC14F4C0
:10283000403F80460BD1284601F092FD3D4B984524
:1028400003D19DF8030001F00FFD00200CE00023F0
:10285000194602AA2846CDE9023301F097FB354B11
:10286000984204D06FF0150004B0BDE8F0818045B7
:1028700003D19DF8030001F0F7FCA3034BD540F210
:1028800006332340B3F5837F19D00CD8062B17D01D
:1028900004D8ABB1022BE5D1042311E0B3F5807F5E
:1028A000E0D101230CE040F20222934227D0B3F59D
:1028B000407F26D0B3F5007FD4D1022300E0072368
:1028C0008DF8043084F48033C3F30043E0068DF8C0
:1028D000053054BFC4F34013032321038DF80630A1
:1028E00011D57A680123B340C2F80835002201A946
:1028F000284601F0F9FB0F4B9842A6D0B2E705231A
:10290000DEE70323DCE7620341BF01237A68B340BB
:10291000C2F80C35EAE7E3064FF0000354BFC4F3F6
:10292000401403241A4601A928468DF8044001F0FA
:102930002DFBE0E70000AD0B024B0B6001231360A1
:10294000704700BF780E0020004870479C7500005B
:1029500010B504F0D0FB034C206004F0C8FB6060AD
:10296000002010BD780E0020F8B50E46144604F085
:10297000BEFB21460546304602F0EEFC374600B36A
:10298000B6FBF5F305FB136323B9B4FBF5F305FBC5
:10299000134343B10D4823463246452102F035FB2F
:1029A0006FF0150002E0A54201D90020F8BD04F047
:1029B0009EFB0546384601F0E1FD641B2F44F9D12A
:1029C000F3E70348234632464521E7E7EA81000062
:1029D0000E820000F8B50E463046194617461D46D1
:1029E00002F0BAFC40B913482B463246452102F0AA
:1029F0000CFB6FF01500F8BD46EA050414F0030463
:102A000004D00D482B4632464521F0E74DB12B1935
:102A1000032BA6EB040006D8084AD2F80034DB07E3
:102A2000FBD50020E7E73B1B043C196801F0C6FD1D
:102A3000EDE700BF0E8200003082000000E00140A0
:102A400070B50D462846194616461C4602F084FC11
:102A500040B9084823462A46452102F0D6FA6FF0CD
:102A6000150070BD24B122462946304602F079FB9C
:102A70000020F6E70E820000F8B5044607690D460F
:102A800004F054FB90B92C4B1B787BB16426606832
:102A900002F0F7FCE0B9012004F024FA013EF6D17F
:102AA000F4E786F31188BFF36F8FEFE74FF0200351
:102AB000EFF3118683F31288BFF36F8F606831469E
:102AC00002F0DFFC90B986F31188BFF36F8FEDE75A
:102AD0004FF02003EFF3118683F31288BFF36F8F5B
:102AE0006068314602F0CDFC0028DAD03B691D70E9
:102AF000626838691368C3F844050120C3F84805C3
:102B00000020C3F82001D3F82051C3F858015268BF
:102B1000D3F85801D20608D5626812680820C2F8B6
:102B200000054FF48002C3F8042301229A6081F368
:102B30001188BFF36F8FF8BD6D2C0020F0B54B7975
:102B4000012B29D0032B24D110278B79032B20D1E3
:102B5000CE790EB1012E1CD10A79012A1ED0022A8B
:102B600020D0B2B914460B684568B3F5164FD5F8B6
:102B700000C06ED033D8B3F5165F6DD01CD8B3F556
:102B8000966F6BD010D8B3F5967F6AD0B3F5167FE9
:102B90006AD06FF085005BE00027D6E74FF48074C1
:102BA0000E22E0E70024FBE7B3F5166F5FD0B3F524
:102BB000965FEED1384B3CE0B3F5E14F5AD007D8E1
:102BC000B3F5615F58D0B3F5964FE2D1334B30E0A7
:102BD00047F61225AB42DCD14FF4000329E0B3F5F0
:102BE000613F4BD013D8B3F5963F4AD009D84DF684
:102BF000C025AB4247D0B3F5614FCAD14FF46B0348
:102C000017E0B3F5E13FC4D14FF0EB7311E0B3F53A
:102C1000612F3BD008D8224DAB423AD0B3F5E12F1B
:102C2000B7D14FF0E86304E01E4DAB42B1D14FF095
:102C300080530569CCF8243543683A431B68344314
:102C40002243C3F86C2503C92B1D83E80300002031
:102C5000F0BD4FF41D03ECE7134BEAE74FF49E235E
:102C6000E7E74FF4A033E4E74FF41C33E1E74FF418
:102C70001D23DEE70D4BDCE70D4BDAE74FF06C73FD
:102C8000D7E70C4BD5E74FF46503D2E74FF07063FD
:102C9000CFE74FF08063CCE700B0130000A04E00F8
:102CA00090D0030040420F000050270000C0750084
:102CB00000F03A0000903A012DE9F74347680669B1
:102CC0003C680021C4F800153060D7F80C908046AD
:102CD00001AA484602F048FC051E1EDB019BD9F8FC
:102CE00000201979186800F06BFA051E15DB311DFC
:102CF0004046FFF723FF054678B97B68990724D53E
:102D000006F1180001F068FC244B984209D02448D1
:102D1000452102F07AF96FF00405284603B0BDE8BA
:102D2000F083337EDB0003F1804303F5F83304F1D5
:102D30000C0204F59071C3F81015C3F81425327E07
:102D400001239340174AC2F804350823C4F800351C
:102D50003B7A53B9C4F81031D4F810317369C4F810
:102D600034350123C4F8383523607B689A075CBF8B
:102D70004FF48073C4F804337B68DB0644BF4FF420
:102D80008003C4F804333369C4F844350023C4F81D
:102D900048350123A360E360BFE700BF0000AD0B2F
:102DA0007782000000F0014070B5012383400E4A95
:102DB000BFF35B8FDC4352E8001F01EA040542E8E1
:102DC0000056002EF7D1BFF35B8F4FF48032824064
:102DD0000648C0F80823BFF35F8FBFF36F8F0B4225
:102DE00014BF0120002070BD840E0020001001409F
:102DF00070B40E49D1E90034D01AC31844F100046C
:102E000022F07F46C1E90034A6F50013B3F5400F68
:102E100009D2074B1B681A0A1B069C19054B42F185
:102E20000005C3E9004570BC01F032BDF800002088
:102E3000880E00200001002011B3BFF35B8F012337
:102E4000104A834052E800CF4CEA030C42E800C12C
:102E50000029F7D1BFF35B8F0B4A4FF480338340D7
:102E6000C2F80433094BBFF35B8F1B68BFF35B8F62
:102E7000C340DB0742BF064B4FF40032C3F80021CA
:102E8000704700BF840E002000100140800E00201B
:102E900000E100E00D4B1868010A0006BFF35F8FE8
:102EA0000B4BD3F80435181841F10001B3F5801F1E
:102EB0000AD2084BD3E90023904271EB030303D2FB
:102EC00010F1807041F10001704700BF880E0020B2
:102ED00000100140000100202DE9F74F16461F4663
:102EE0000446FFF761FF0090FFF7D4FFB04271EB9B
:102EF000070351D23A4B301A67EB0101984271F146
:102F000000016AD2374B03EB0413D3E902239F423B
:102F100008BF96424ED034494FF4803904F1500531
:102F200009FA04F9AD00C1F848932046ADB202F0A9
:102F30000FFB26F07F4B05F1804504F5A8732B4A63
:102F4000019305F58835DC464FF0030A019B2CF010
:102F50007F4041F82300C1F84493D1F804856FF015
:102F60000200A0EB0800604420F07F40904221D98D
:102F7000286860B1D1F80485A8EB0B0020F07F40F1
:102F8000B0F5000F16D9204602F0E2FA174A0AEB14
:102F9000080C0AF1010AD9E70123154ABFF35B8F38
:102FA000A34052E8000F184342E800010029F8D17D
:102FB000BFF35B8F0B490C98230101EB0412C2E9AC
:102FC0000267C8500D9B5360002520460099FFF70B
:102FD00033FF284603B0BDE8F08F6FF01505F4E726
:102FE00001008000E800002000100140FDFF7F008C
:102FF000800E002073B5194B194D00244FF0FF309F
:103000004FF0FF31C5F80845C3E902014FF48033A2
:10301000C5F80433134B02264FF400320121C5F8E2
:1030200004631120C3F880212246FEF7D5FD11204C
:10303000FEF7B6FD0C4A0123AB602B6013600B4B0F
:103040000B4A0093019400232046FFF745FF3046CA
:10305000FFF790FA204602B070BD00BFE8000020E4
:103060000010014000E100E0840E0020F12D00007E
:10307000FFFF7F002DE9F7432F4CD4F80433990765
:103080000BD5D4F8043143B12C4A0023C4F80431E1
:10309000D4F80431136801331360D4F80433DA032D
:1030A0002AD5BFF35B8F264B53E8002F22F0010196
:1030B00043E800100028F7D1BFF35B8FD30702D499
:1030C000D4F84031C3B10025C4F84051D4F84031A0
:1030D000FFF7E0FE4FF02003EFF3118283F3128835
:1030E000BFF36F8F174BD3E90267B042B94106D2E5
:1030F00082F31188BFF36F8F03B0BDE8F0834FF008
:10310000FF384FF0FF39C3E90289D3E900101D6091
:103110004FF48033C4F84833C4F84051D4F84031F8
:1031200082F31188BFF36F8F0029E5D000903246FB
:103130003B4628468847DFE700100140880E002004
:10314000800E0020E8000020431C13B522D0012887
:1031500022DD124A124B9042D4BF04461C46FFF7B0
:1031600099FE104B0E49D3E90023801AB0F5000FE9
:1031700028BF002404448C4228BF0C46A2180A49E8
:1031800000914FF00000019043F10003FFF7A4FE0F
:1031900002B010BD024CE2E70124E0E7FEFF7F0031
:1031A000FFFF7F00F8000020F12D000008B5FFF7B9
:1031B00071FE024B1B68C01A08BD00BFF80000205A
:1031C0002DE9F0414D4E00EB81010127814202D1F2
:1031D0000020BDE8F081056805F07F03C5F34324B6
:1031E0007F2B4FEA154508BF4FF0FF33192D00F232
:1031F0008180DFE805F00D1F24272A3E277F7F7F8F
:103200007F426B7F7F7F7F7F7F7F7F7F6E76797C42
:10321000C2F80C354FEA531CBCF1010F03F01F0537
:1032200014BF4FF0A04CB44607FA05F5CCF808558A
:10323000012502E0C2F814350025AE4624E0C2F8AC
:103240000835E7E7C2F81035F6E7C2F8083500257B
:103250004FEA531EBEF1010F14BF4FF0A04EB64609
:1032600003F01F0C07FA0CFCCEF80CC54FF0010E52
:103270000AE0C2F80C350125EAE7C2F80835002C4F
:10328000DAD10025AE46062450F804CB0CF40058E1
:10329000B8F1000F4FEA0424CCF3C11803F01F0C5F
:1032A0004FEA53131CBF01254FF0000E44EA880477
:1032B000012B0CBF33464FF0A04344EA0E040CF53B
:1032C000E07C44EA450443F82C407FE7C2F80C3523
:1032D000D5E7C2F860350568C5F38035002DCAD042
:1032E00098E7C2F86435F6E7C2F86835F3E7C2F844
:1032F0006C35F0E76FF085006BE700BF000300500E
:1033000030B50C490C4D0B680246002405EB031048
:10331000D0F80808C0B218B904B10B60002007E06B
:103320000133072B4FF00104F0D90B606FF01B0045
:10333000136030BD8C0E002000E00140034808B54A
:10334000452101F062FE0020FFF71AF8C782000055
:1033500030B5816885B0103921F00704054601F0C9
:10336000A7FE10220146684601F006FF0749102219
:10337000684601F0F6FE10236A462146284601F011
:1033800067FE003818BF012005B030BD447700004B
:1033900030B50D46816887B0102302AA1039044663
:1033A00001F041FE002802DA012007B030BD1022F2
:1033B00002A9204602F041F900283AD11E49102204
:1033C00002A801F0BEFE00280CBF012302232B70CF
:1033D000204602F01EF9012301460DF107022046A6
:1033E00001F021FE0028DFDB9DF8073003F00F021B
:1033F0001B096A702B7101220DF10701204602F0B2
:103400001CF910B96B78042B03D901236B700023CE
:103410002B71A268183A22F00702083AA91C20462C
:1034200002F01EF90028BFD1E91C204602F071F914
:10343000BBE70323CBE700BF447700007FB5054619
:103440006946022002F06BF9044610B1FF2004B077
:1034500070BD02A9052002F062F9012836D1294881
:103460002A46492101F0D1FD274B02938DF80C40EB
:103470009DF800509DF80860244C002220782946D1
:1034800002F0CDF848B36078314602F0C8F820B3B6
:10349000A378042B03D09DF8031099421DD1E37843
:1034A000042B03D09DF80B10994216D12379042BDD
:1034B0000FD16379022B1BD1154A1648492101F01F
:1034C000A4FD6079831E022BC1D9BFE70028CFD0AD
:1034D000BCE79DF802109942EBD00132032A04F1B7
:1034E0000604CBD10C48492101F08FFD0120AEE745
:1034F000032B05D0094A0A49042B08BF0A46DCE71A
:10350000084ADAE70C830000030103037F8300000D
:10351000EE820000578300006A830000F3820000FF
:1035200005830000E982000001680E4A91420346CB
:1035300015D1C169A2F11022A2F1EF1291420ED170
:103540008268012A0BD8C26812B101698A4206D08A
:10355000586928B19B691B1A58425841704701208D
:10356000704700BF55AA00FF70B50D4B9E68A6B10D
:103570003046FFF7D9FF044678B9F3686BB935696F
:103580000DB9204670BD2846FFF7CEFF28B9EB687D
:10359000B34202D12E462D69F2E70124F1E700BFC4
:1035A000900E00202DE9F8433F4F3C68D4B1BC6831
:1035B000C4B100284AD0002948D001FB00F5B5FB72
:1035C000F0F0884242D1281D40D8A9070DD025F03F
:1035D00003060436FC6803E06368B34238D2A4698A
:1035E000002CF9D12046BDE8F8832E46F2E7FB60B7
:1035F00041E006F120016318203A5A600022C3E935
:1036000002242A4822691A6160502949D96102B10D
:10361000D36062695A61A1699961AAB193619A699B
:1036200002B153614FF00109C4E90169236100232C
:10363000C4E905333B69DB072ED5FFF795FF58B387
:103640001C4B48461B6826E0FB60E8E70024C9E7FE
:10365000A3681BB1174B01201B6898476268921B37
:10366000232A04F12008C4D80123A360D4E9052348
:10367000002ABCD09361A3690BB162695A6100232F
:10368000C4E905333B69DA0706D5FFF76DFF18B1CA
:10369000084B1B68012098472A46002140464446B3
:1036A00001F06AFD9EE700BF900E002055AA00FFC2
:1036B000669911EE4C00002070B50546002800F018
:1036C0008880444E3368002B00F08380B268002A63
:1036D0007FD0834203D872681344984203D33E4B91
:1036E00001201B689847A5F120042046FFF71CFF26
:1036F00018B1394B01201B68984755F8183C012B2D
:1037000003D0354B01201B689847002345F8183C2F
:1037100055F8143C3BB39A682ABB55F81C2C02F1AF
:1037200020015A680A445A6055E905321A6155F871
:10373000145C2B6903B1DD6020220021204601F0DA
:103740001BFD286910B18368002B2ED033699B07BD
:103750003FD5FFF709FF00283BD01F4BBDE8704065
:103760001B680120184755F8100C00282AD08368E0
:1037700043BB426863681344203363600369236179
:10378000D4E905239AB9CBB9436963618269A2611F
:10379000B3B19C61A36903B15C61236903B1DC60CF
:1037A0002022002101F0E8FCD0E72C46E1E79361FC
:1037B000A369002BE8D062695A61E5E7F360F7E797
:1037C000F460E7E7F36845F8083C03B15C61F46036
:1037D000BCE770BD900E00204C00002038B51422CC
:1037E0000C4605460021134801F0C6FC1249134857
:1037F00000F034F8232C1CD915F003031FBF043C40
:10380000E418C3F10403ED1822460021284601F014
:10381000B3FC084B0A499D60C3E90054203C6C602E
:103820009A6811609A68DA60A1F11021A1F1EF1194
:10383000D16138BD900E0020B9360000A5350000DA
:1038400055AA00FF014B1B68184700BF5400002019
:10385000014B1B68184700BF50000020024B186046
:10386000024B0020196070475400002050000020D7
:103870000A4619B1024B00211B681847704700BF68
:1038800058000020F8B500F10806476804463046A5
:103890000D4602F0ECFA87424BD16368B3F5807FA6
:1038A00047D80021304602F04DFC002841DD0021C0
:1038B000304602F0ADFAE0B345B9294604F11400F0
:1038C00002F040FC002834DD0020F8BD04F12C0596
:1038D0000021284602F036FC00282ADD0021284677
:1038E00002F096FA28B304F138050021284602F0C8
:1038F00029FC00281DDD0021284602F089FAC0B10C
:10390000002104F1140002F01DFC002811DD00214B
:1039100004F1440002F016FC00280ADD002104F145
:10392000500002F00FFC002803DD002104F15C00D0
:10393000C6E70148C9E700BF80BFFFFF70B500219F
:103940000446FFF79FFF054610B10E4D284670BD97
:1039500004F10806304602F06BFA7F28F5D91434DA
:103960002946204602F054FA0028EED0204602F004
:103970005FFA0128E9D93146204602F0A2FB00286F
:10398000E4DBE2E700BEFFFFF0B50C4687B00021A4
:1039900005461646FFF776FF002839D103A802F046
:1039A0008DF921466A6803A802F067FA044618B147
:1039B00003A802F089F90CE005F10804214603A8E8
:1039C00002F07FFB002807DB03A802F07DF96FF00F
:1039D0000304A4F5854418E005F1680303A96F68A2
:1039E000009305F114022346084602F0C5FE044682
:1039F0000028DDD13A46314603A802F05FFA0446BA
:103A000003A802F061F9002CE3D1204607B0F0BD15
:103A1000004CFAE780BFFFFF234A2DE9F041B1F1E6
:103A2000000818BF9646214A2149224F224E234DB5
:103A3000234C18BF944602F1794208BF8E4602F526
:103A40007402204902F5016208BF8C461E4918BF66
:103A500011461E4A18BF17461D4A18BF164602F1E6
:103A6000D14202F5C01202F51E6218BF1546194A6E
:103A7000034618BF14461848C3F86880A2F11162C3
:103A8000A2F50C22A2F28E2218BF02460020C3E942
:103A90000000C3E902ECC3E90417C3E90665C3E902
:103AA0000842BDE8F08100BFD89E05C107D57C362D
:103AB00067E6096A3AF54FA57F520E518C68059B5F
:103AC000ABD9831F85AE67BB72F36E3C39590EF7D5
:103AD000310BC0FFA78FF964A44FFABE2DE9F04F58
:103AE000D1B0031D019300F124030DF58E7B0393E8
:103AF000019B5A4653F8040F42F8040F039898426A
:103B0000F8D14F9B02934CADDDE94AE395E82011D3
:103B1000DDE948070493424B059306AA4FF00009DC
:103B2000B9F10F0F63D84C780B78240444EA03648E
:103B3000CB7823438C7843EA04234FEAF52A8CEAB6
:103B40000804059E93608AEAB51A2C408AEA756AD1
:103B500084EA0C04544456F804AB059654442344B8
:103B6000029CCDF808C023444FEA703A40EA0704AB
:103B70008AEAB00A04EA0E0400EA07068AEAB05AA2
:103B80003443544409F10109DDF810A0CDF810E0E8
:103B9000B9F1400F9A4402F10402234401F10401F7
:103BA0001ED1CDE90634CDE94E8CCDE94CA5CDE949
:103BB0004A7ECDE94830019A52F8043F01925BF801
:103BC000042F1344019A1360039B9342F3D106A878
:103BD0004FF49471FFF74CFE002051B0BDE8F08F18
:103BE000BE46C4460746A8461846554698E7136899
:103BF00052F8384C52F8346C4FEAF34A8AEA734A66
:103C00008AEA932A52F8143C234452F8344C4FEA7F
:103C1000B44484EAF614534484EAD60423448CE77B
:103C200018760000024AD2F80034002BFBD070470F
:103C300000E0014010B54FF08053D3F830210D2A39
:103C400055D14FF080410022C1F80C21C1F810215C
:103C5000C1F83825484AD3F80404C2F82005D3F83F
:103C60000804C2F82405D3F80C04C2F82805D3F8D8
:103C70001004C2F82C05D3F81404C2F83005D3F8A8
:103C80001804C2F83405D3F81C04C2F84005D3F870
:103C90002004C2F84405D3F82404C2F84805D3F838
:103CA0002804C2F84C05D3F82C04C2F85005D3F808
:103CB0003004C2F85405D3F83404C2F86005D3F8D0
:103CC0003804C2F86405D3F83C04C2F86805D3F898
:103CD0004004C2F86C05D3F84434C2F87035D1F80A
:103CE0000034DB0709D56FF00103C1F800344FF051
:103CF0008053D3F830310D2B0CD14FF08053D3F8D3
:103D000034313BB14FF01023D3F808224FF08043F9
:103D1000C3F858254FF01023D3F80022002A03DB04
:103D2000D3F80432002B22DA144901234FF010207B
:103D3000C1F804351224FFF775FFC0F80042FFF701
:103D400071FFC0F80442FFF76DFF0023C1F804358E
:103D5000FFF768FFBFF34F8F09490A4BCA6802F4A7
:103D6000E0621343CB60BFF34F8F00BFFDE7064B0C
:103D7000064A1A6010BD00BF00C0004000E00140CC
:103D800000ED00E00400FA055C0000200090D00384
:103D900070B501250268BFF35B8FB2FA82F3C3F1FD
:103DA0001F03DBB205FA03F422EA040450E8006FB3
:103DB000964204D140E8004CBCF1000FF6D1BFF3AD
:103DC0005B8FE7D101480B7070BD00BF0000AD0BE9
:103DD00010B50368CB40DB0714D401238B40026885
:103DE000BFF35B8F43EA020150E8004F944204D1D5
:103DF00040E8001CBCF1000FF6D1BFF35B8FEED1A1
:103E0000014810BD0148FCE70000AD0B0400AD0BFC
:103E1000044B1A7922B9012218601A7102487047BE
:103E200002487047A40E00200000AD0B0C00AD0B43
:103E300010B54FF08043D3F8002152B10020C3F8F1
:103E40000001D3F800210122C3F80823104B1B689E
:103E500098474FF08043D3F8042172B10022C3F891
:103E60000421D3F80421D3F81824D3F818149207A6
:103E700004D10122C3F818259A6010BD0222C3F8AC
:103E80000823034BBDE810401B680120184700BF02
:103E9000A40E0020036803F01F025B09012B0260DF
:103EA000024818BF4FF0A040704700BF0003005009
:103EB000034B083033F81000C0F34010704700BFC8
:103EC0006000002070B500F108030C4C34F813308A
:103ED000DA0505460E4607D5C3F3432304EBC302B8
:103EE00054F8333052689847A3682BB1E2683146E2
:103EF0002846BDE87040184770BD00BF6000002034
:103F000010B4124A083032F81030D9051BD5C3F36B
:103F1000432123F4F85322F8103002F10E0400205C
:103F200034F8023F13F4807F03D0C3F34323994254
:103F300009D001302A28F3D1002342F83130044857
:103F400010BCFFF745BF10BC704700BF60000020E9
:103F5000C800002038B50246FFF7AAFF094C02F15D
:103F6000080540B134F8153007495B0B03F5A2731F
:103F7000002041F823001046FFF7C2FF002324F879
:103F8000153038BD60000020006000402DE9FF4181
:103F9000044616461D4601B34E4F00F1080837F897
:103FA00018309B0702D5FFF783FF10BB0023CDE934
:103FB00000338DF80E308DF80F300DF10F020B46E7
:103FC00020460DF10E0103F034F837F8183023F0D5
:103FD000020343F0010327F8183046B33D4B96F82F
:103FE00000C0726804F1080733F81710880702D57B
:103FF000AAB139481DE021F02001C904C90C23F8F9
:10400000171062B1BCF1030FF3D872681678BCF1D7
:10401000000F11D1314A06F5A27642F826C033F8D6
:10402000172022F01C0242EA8C0223F8172045BB1D
:104030002B4804B0BDE8F081B20002F1804202F5E5
:10404000C04241EA4631D2F8100520F00300C2F820
:104050001005D2F8100520F44F3020F44070C2F85B
:1040600010052002D2F810E500F47C5040EA0C4024
:1040700040EA0E0041F0200123F81710C2F81005A5
:10408000CDE7D5E900672046FFF73AFF002ECFD0F5
:10409000104DD5E90023964201D19F4218D0114816
:1040A0000DF10F01FFF774FE0D4B9842C1D19DF841
:1040B0000F2045F8326005EBC20308345F6035F825
:1040C000143043EA422343F4807325F81430AFE7F9
:1040D0000022EEE7600000200400AD0B006000400D
:1040E0000000AD0BC8000020F0B5044685B01546B1
:1040F00019B3334E00F1080736F81720930703D49D
:10410000FFF7D6FE002858D112F01C0F02D04B78D2
:10411000012B52D001238DF80F300023CDE900137D
:104120004A1C8B1C20460DF10F0102F082FF36F86D
:10413000173043F0030326F8173015B9214805B0AE
:10414000F0BD1F4E04F1080736F81700830734D579
:1041500095F800C06146890020F0200001F18041FF
:10416000C00401F5C041C00C26F817000023C1F8B7
:1041700010356A78002AE1D0D1F81035AD7823F4F3
:10418000991323F4F853C1F81035D1F810E5230240
:1041900003F47C53120402F4403243EA0E03134347
:1041A0002A0502F4801240EA4C30134340F020000C
:1041B00026F81700C1F81035C0E70348BFE700BF75
:1041C000600000200000AD0B0400AD0B014BC3E903
:1041D000020170476000002008B50246FFF768FE44
:1041E00038B1054B0548083233F812305B0B0B70C1
:1041F00008BD0348FCE700BF600000200000AD0BD5
:104200000400AD0B38B50F4C94F86C50BDB9542276
:10421000294604F1100000F0AFFF0620FDF7C0FCB6
:10422000094B0A48C3F87C51D3F87C214FF0004277
:10423000C3F80423012384F86C30A36638BD044816
:10424000FCE700BF60000020006000400000AD0BF4
:104250000500AD0B034B93F86C00003818BF01202C
:10426000704700BF6000002001460148FFF7B0BD65
:10427000C400002001460148FFF78ABDC4000020A9
:1042800037B50446FFF714FE04F108021E4B33F85D
:104290001230E8B113F002051AD15B0B9A0002F15B
:1042A000804000F5C24002F1804202F5C042056044
:1042B0000068D2F8100540F00100C2F8100529B1DD
:1042C000012202FA03F3114AC2F8043303B030BDED
:1042D000C3F38203042B12D0052B12D001A8019442
:1042E000FFF7D8FD019BD0F81015D94001F001016E
:1042F0000231204603B0BDE8304002F0E3BE0321A6
:10430000F7E70221F5E700BF6000002000600040F1
:1043100008B50246FFF7CCFDC0B102F108010E4B13
:1043200033F81130990711D45B0B01229A409B009E
:104330000A4903F1804303F5C043C1F80823D3F8C9
:10434000102522F00302C3F8102508BDBDE808407F
:104350000021104602F0B6BE600000200060004060
:1043600013B50E4B00F10802044633F81230DB0798
:1043700011D5FFF7CDFF2046FFF7ECFD01A8019412
:10438000FFF788FD019B03F5E073022240F823202C
:10439000034802B010BD0348FBE700BF60000020E7
:1043A0000000AD0B0400AD0B2DE9F04F684B6948E0
:1043B0006949002687B0012234461D6835B1D0F81E
:1043C000045315421EBF1C601D68164304338B4204
:1043D0004FEA4202F1D1DFF87C91D9F87C31002B11
:1043E00000F099804FF0A043D3F820250492C3F841
:1043F0002025D3F820280592C3F820284FF0000884
:104400000DF1100A4FEA481300934FF0010B49E0F9
:10441000009B524A94FAA4F4B4FA84F41C44E008D1
:1044200004F10803039432F813701AF8003004F012
:1044300007020BFA02F223EA02030AF8003003A88B
:10444000FFF728FD039B03F5E073B90850F823300C
:10445000C7F382054A072F46C3F301432CD52046F4
:104460003946DDB2FFF72EFD03A80394FFF712FDD6
:10447000039B03F5E07350F82330C3F301439D42DF
:1044800007D10021204602F01DFE2946204602F0F9
:1044900019FE03A80394FFF7FDFC039B0BFA03F33B
:1044A000C0F820355AF82840002CB1D1B8F1000FDF
:1044B0001DD14FF00108A5E7022B0CD103212046A6
:1044C00002F000FE05F00503012BE2D1394620463B
:1044D000FFF7F8FCDDE702212046019302F0F2FD30
:1044E000032DF3D0019B032BD3D1022DEDE74FF029
:1044F000A042C9F87C41D9F87C311949D2F820355D
:104500000493C2F82035D1F8202505921343C1F851
:1045100020257FF473AF012416B907B0BDE8F08FF2
:1045200096FAA6F3B3FA83F304FA03F29B0003F1BD
:10453000804303F5C04326EA0206D3F81005D3F8FA
:104540001015C0F30520C1F30141FFF7BBFCE3E701
:1045500000610040006000402061004060000020D9
:1045600000030050044AD2F80034DB07FBD5016099
:10457000BFF35F8F704700BF00E001404FF08053F2
:104580001A69B0FBF2F302FB130373B9084B022262
:10459000C3F80425C3F80805D3F80024D207FBD5D7
:1045A00000220448C3F8042570470348704700BF41
:1045B00000E001400000AD0B0A00AD0B10B5054C4A
:1045C0000123C4F80435FFF7CDFF0023C4F80435F8
:1045D00010BD00BF00E0014001460148FFF7D8BB15
:1045E000D000002010B5144C144A15490323236150
:1045F0006361144BA261E3614FF480632362002383
:10460000A3626362E36222660F4A62661022A266B8
:10461000E01D2367E366636700F082FDBFF35F8FF1
:104620000A49204600F07CFDBFF35F8F2023A37171
:10463000BFF35F8F10BD00BFAC0E0020BA83000037
:10464000C38300006D2800205D280020C783000080
:1046500073B504460D464FF02003EFF3118683F344
:104660001288BFF36F8F042896BF124B124B53F87A
:1046700020300022009245210246104800F0C5FC7F
:104680003DB1EB69C3F308031BB10D48452100F0B0
:10469000BCFC0C4B0C480022452100F0B6FC29461E
:1046A0002046FEF74BFE86F31188BFF36F8F02B0F2
:1046B00070BD00BF18770000CE830000DC830000CF
:1046C000098400002F840000378400000F4B70B570
:1046D00053F82040013053F82060A64200D870BD46
:1046E000D4E90035284698476DB138B10028B8BFE5
:1046F0004042EB68FF28A8BFFF201870EA68537893
:1047000043F0010353700834E7E700BF2C77000043
:1047100008B5094B012203201A70FFF7D7FF00F0FC
:1047200013F90420FFF7D2FFFBF754FE034A137B73
:1047300023F00103137308BD6D2C00200801002035
:1047400008B50348034A0021121A02F0EBFC08BD29
:10475000E8000020702C002008B50020FFF7B6FF0D
:10476000184B83F30888184C636943F40073636142
:104770000025E02384F82230E57725766576A57656
:1047800084F82050636A43F4E023636284F8235082
:10479000FDF7A0FCFDF7C4F94FF0FF33A362E3621D
:1047A000FDF7A0FDFDF722FD02F0B0FC0120FFF7B0
:1047B0008DFF0220FFF78AFF04482B462A46294630
:1047C000FDF768FAC034002000ED00E0114700005A
:1047D00008B50648064A0749121A02F0A5FCBDE8CA
:1047E0000840054A0549064802F09EBC000000202A
:1047F000E8000020D084000000000000D084000009
:1048000000000020034B1B680BB9FEF7CFBC002053
:10481000704700BF540F002010B50E4B1C689C421F
:1048200004D1FFF7EFFF6FF0004010BDFFF7EAFF84
:10483000002CF8D0D4E904321B1A62EBE072B3F119
:10484000004F72F10001EEDA002AACBF18460020DA
:10485000EBE700BFD400002030B570B10B4B5B68B4
:1048600098420AD0036843B1D3E90421D0E9044552
:10487000121941EB0501C3E90421D0E900321360AC
:104880005A600023C0E9003330BD00BFD4000020CF
:104890002DE9F84303464FF02002EFF3118482F331
:1048A0001288BFF36F8F254FDFF89490D9F800007E
:1048B000DFF890C03B604845DCE9001E4FEAE37535
:1048C0000CD058B1D0E90486434575EB060217DADF
:1048D000B8EB030266EB0506C0E9042659184EEB57
:1048E0000505CCE9001500253D60FFF795FF294639
:1048F000FEF72AFC84F31188BFF36F8FBDE8F883BD
:1049000018EB01014EEBE873CCE900130022002301
:10491000C0E90423FFF7A0FF84F31188BFF36F8F72
:10492000836898474FF02003EFF3118483F31288D4
:10493000BFF36F8F3B68A3EB0803B7E7540F00206A
:10494000D400002088010020014800F077BA00BFA1
:10495000A1840000704729B101290CBF05206FF028
:104960001500704702207047002070472DE9F7437B
:104970000E4617469946044628B94FF0FF38404680
:1049800003B0BDE8F0830029F7D0002AF5D0CB684A
:104990000D891D4404230DEB03022946384600F01F
:1049A00042FB80460028E8D1BDF80410738946F622
:1049B0000812914225D1BDF806109942DDD1042399
:1049C0000DEB03022944384600F02DFB0028D4D11A
:1049D000BDF8042046F607139A42CED1C4E9006719
:1049E0009DF82830A4F80890A3727389BDF80620BA
:1049F0002B44E360738913442B44043563612561C0
:104A0000BDE7002BE4D0B8E72DE9F3410E46174689
:104A10001D46044620B94FF0FF3002B0BDE8F081DA
:104A20000368002BF7D04368002BF4D04FF6FF78D3
:104A3000D4E904239A4216D223685B8923B1E36840
:104A4000934204BF043323610423216960680DEBA2
:104A5000030200F0E8FA0028DDD1A37A2BB1D4E9F3
:104A600003329A4201D30120D7E72389BDF806100B
:104A7000434501F1040203D0BDF804C09C450BD1AD
:104A800015B1BDF804302B802369043333603980BD
:104A9000236913442361C0E7236913442361C7E7F3
:104AA00000F04FBB4FF4C0735843303070470B7861
:104AB000022B06D0052B14BF4FF0FF304FF4C0700F
:104AC00070474FF4C070704710B5044600F0E9FA23
:104AD000A3684FF4C072303B02FB103010BD8168F8
:104AE000183921F007010122083900F001BE13B581
:104AF0000446019100F08DFD0423A0F108010DEBA7
:104B00000302204600F0C8FD02B010BD70B5134688
:104B10000E461546002102460446FCF75DF950B9E1
:104B20002B4604F12C0201212046FCF755F910B167
:104B3000002E08BF002070BD73B5044600200D464E
:104B40001646FFF708FF6946C0B2FCF791FF30BB7D
:104B50002C2303FB05440098E36825891D440423A6
:104B60000DEB0302294600F05EFAC0B9BDF804203F
:104B70006489009846F608139A4215D1BDF80630AC
:104B80009C420CD104230DEB0302611900F04BFA97
:104B900028B9BDF8042046F607139A4207D00098BA
:104BA00000F040FA02B070BD002CF2D0F7E7BDF87B
:104BB0000610214429443160F1E737B50446426AC2
:104BC000802501A902200195FCF77AFF58B9019BC5
:104BD000226DA36201A905200195FCF771FF05462E
:104BE00028B1092500E00125284603B030BD019B0E
:104BF000206A636500F055FAE065F5E7012303607C
:104C000003F1012343600023C0E902337047437975
:104C1000012B07D10368012B04D10079431E5842B0
:104C200058417047002070477FB506460D46022068
:104C300001A9FCF71DFF38BB0198FFF745FFF16D97
:104C40000446284600F0E5F80444019800F029FAEB
:104C50000646019800F02CFA082201460DEB0200EE
:104C600000F08AFA2B798DF80830214601983346F6
:104C700002AA00F0EDF9041E019818BF012400F00B
:104C8000D1F9204604B070BD0124FAE700F0F5B96F
:104C90002DE9F8430E46002107460846FFF75BFE64
:104CA000012104460020FFF756FE33789C4221D0B4
:104CB000984221D101252C2303FB0575F86DAC6AC0
:104CC000FFF7F0FE013C07464FF000086B6A03EB6C
:104CD000C40253F83410D2F804901B684A46C91A2B
:104CE0003046C844FFF7D2FFB84504F1FF34EDD396
:104CF000BDE8F8830025DEE70120F9E737B5154662
:104D00000C460520694600F00AFDE979012903D027
:104D10000022204600F017FD9DF80330012B02D140
:104D2000204600F0EFFCA9682046FFF7E0FE204691
:104D3000FEF70EFB002003B030BD73B50D460646EE
:104D4000FCF732F90446E86050B302282DD101A9DE
:104D5000FCF78EFE58BB01982A463146FCF78AF8CC
:104D60000446D0B9019800F054FC012301460DF12E
:104D70000302019800F057F90446A0B901980122F6
:104D80000DF1030100F059FC10B101238DF803303F
:104D90009DF8033003F00F03EB71019800F042F926
:104DA000204602B070BD0124F7E70724F8E701248C
:104DB000F6E713B5022001A9FCF75AFE48B901989D
:104DC000FFF78DFE0446019800F02CF9204602B052
:104DD00010BD0124FAE71FB5022001A9FCF748FE27
:104DE000A8B9019802A9FEF7D3FA044668B99DF85C
:104DF0000B30032B03D1019800F084FC044601988A
:104E000000F010F9204604B010BD0124F7E701249A
:104E1000F8E710B543790279012B14BFCB010023C9
:104E200002F1FF3201FB0233026814BF4C000C4652
:104E3000013A04FB023010BD002070470FB407B5E3
:104E400004A951F8040B0191FCF7D0FA03B05DF806
:104E500004EB04B07047038B13F0070305D103681C
:104E6000002B0CBF002003207047022B05D1408B84
:104E7000B0FA80F0400980007047012B05D103682B
:104E8000002B0CBF0020052070470020704710B594
:104E90000C4600B111B96FF0150010BD081D00F0EF
:104EA00095F80028F9D1A368032BF6D9F3E72DE98B
:104EB000F0410D4607461946281D90461E4600F053
:104EC00096F8044638B13346424629463846A44649
:104ED000BDE8F0416047BDE8F08110B44FF0200418
:104EE000EFF3118284F31288BFF36F8F416110BC1E
:104EF0000121FCF789BA38B50C46054658B151B1C5
:104F00000B6843B14B6833B11C22002100F034F927
:104F10002C61002038BD6FF01500FBE770B5054629
:104F20000E46FFF7B4FF041E15DB4FF02003EFF32E
:104F3000118283F31288BFF36F8F6B8B2C8B4FF62C
:104F4000FF718B4204F0070407D182F31188BFF38D
:104F50006F8F6FF00A04204670BD022C0CD1013314
:104F60006B8382F31188BFF36F8F00232246314693
:104F70002846FFF79CFFEEE7062C14D8DFE804F084
:104F800004131313041A0400002333606B683BB945
:104F9000C5E90066ACB902212846FCF735FADAE724
:104FA0001E606E60F6E782F31188BFF36F8F6FF0BB
:104FB0000404D0E782F31188BFF36F8F6FF085048C
:104FC000C9E782F31188BFF36F8FC4E7034658B176
:104FD000426802F00302012A03D0032A04D10268C6
:104FE00012B10020986070476FF01500704742685A
:104FF000816002F00302032A4FF0000203460CBF57
:10500000006810465A60704770470FB407B504A98E
:1050100051F8040B0191FCF7E9F903B05DF804EBDA
:1050200004B070477047002930B4044618460BDBC3
:10503000A5680844A84207D8E068646821448468E9
:105040002468A44630BC60476FF0150030BC704740
:10505000002930B4044618460BDBA5680844A84272
:1050600007D8E0686468214484686468A44630BC5A
:1050700060476FF0150030BC70470029034610B43C
:1050800010460ADB9C680844A04206D8D8685B68D2
:105090001944836810BC9B6818476FF0150010BC5A
:1050A000704708B5C0688368DB689847006808BD2A
:1050B00008B5C0688368DB689847007908BD70B59B
:1050C0004C680368A34201D2012070BD8A68224463
:1050D000934201D30020F8E7D1E903254E69B54298
:1050E00003D36FF00B038B61F4E71B1B42F83530E1
:1050F0004368086902EBC00253600B6901330B611E
:10510000E2E701460068FCF71DBD00210120FCF725
:1051100019BD08B5FCF778FDBDE80840FCF7E6BD11
:105120000139034611F8012F0AB91A70704703F8C4
:10513000012BF7E7034600201A5C02B970470130E3
:10514000FAE710B55AB10139841810F8012B11F89B
:10515000013FA04201D09A42F7D0D01A10BD1046AC
:10516000FCE710B5431E0A44914200D110BD11F86E
:10517000014B03F8014FF7E7C9B2024403469342DB
:1051800000D1704703F8011BF9E74FF0FF3070477B
:105190000369C9B20C2201FB0233186C00F007004E
:1051A00070474FF02003EFF3118283F31288BFF3AF
:1051B0006F8F036803F0C00343F00203036082F3C0
:1051C0001188BFF36F8F704770B5C9B203694FF094
:1051D0002004EFF3118584F31288BFF36F8F0C2640
:1051E00006FB0134246C14F0C00408D0A24206D09F
:1051F00085F31188BFF36F8F4FF0FF3070BD71439F
:105200000B4401221A6485F31188BFF36F8F436842
:105210000B445B6898470020F0E78022FFF7D4BF7B
:10522000F8B5069F0469C9B24FF02005EFF3118667
:1052300085F31288BFF36F8F0C2569430C44256CEE
:1052400005F0070CBCF1010F0BD1276486F3118820
:10525000BFF36F8FC4E90E2343685B589847002063
:10526000F8BD05F0C005AF4286F31188BFF36F8F1C
:105270000CBF6FF077004FF0FF30F1E713B58024DB
:105280000094FFF7CDFF02B010BD6FF085007047AE
:1052900010B40069CBB21C2403FB0400002110BC35
:1052A0001047002001F087BE002001F0C0BE436817
:1052B0005B68D3F810350B600020704743685B686B
:1052C00002EA010021EA0201C3F80805C3F80C153F
:1052D0000020704743685B680020C3F808157047DA
:1052E00043685B680020C3F80C15704743685A6830
:1052F000D2F8043521EA03000B40C2F80805C2F8D1
:105300000C350020704710B503695868F8B1884221
:1053100019D19C6808685860A14200D198600020AB
:1053200008602AB15A680A609A68596002B999609F
:10533000002010E0814206D1086820609868814210
:10534000EDD19C60EBE7044600680028F2D1002A0A
:10535000E8D16FF0150010BD38B505460C4601F0D8
:10536000C0FE002D07DBA84205D9401B84428CBF3C
:105370000020012038BD0020FCE7F7B51C4616468A
:10538000002382682360A36013690D4601AA694661
:105390009847019B5A1E01921BB96FF0150003B08C
:1053A000F0BD0098A26847682168676085B9B31AA4
:1053B000D0F800C0634528BF63461A4403FB0711B9
:1053C0002160A26002689A4206D808300090E0E7A7
:1053D0006B1AB3FBF7F3EBE70020E0E7134600227C
:1053E000FFF7CBBF2DE9F047836886B01B6988467D
:1053F000914601A902AA98470024A2462546029B8D
:10540000AB4202D806B0BDE8F087019F07EBC507A5
:1054100000267B6804933A68B2420AEB060302D87E
:1054200001359A46EBE703940593494603A8C04724
:105430000028E7D0049B01361C44ECE702690B46C8
:10544000D2E9010183E803000020704743681B682C
:10545000D3F88004C3F880047047436802691B686E
:10546000D3F8100150B15269002012780A70C3F8C5
:105470001001D3F8102101221A6070474FF0FF305D
:10548000704702680346D2F8580140B95B689B0731
:1054900006D4D2F82001003818BF0120704701203F
:1054A000704742681368D3F80413C90518D5D3F8B8
:1054B0002011A9B14FF02000EFF3118180F3128881
:1054C000BFF36F8FD3F8200130B10020C3F8200163
:1054D000D3F820010120D86081F31188BFF36F8FCA
:1054E0005268D20615D54FF02001EFF3118281F3F7
:1054F0001288BFF36F8FD3F8581111B10021C3F890
:1055000000154FF48001C3F8081382F31188BFF32C
:105510006F8F704710B50022044601212820FCF748
:105520005BFB2820FCF73CFB2046BDE81040FDF764
:10553000C3BB10B50022044601210220FCF74CFB3E
:105540000220FCF72DFB2046BDE81040FDF7B4BB60
:1055500000F150039B009BB203F1804303F58833B5
:1055600000221A601B68704730B543681360057AE3
:10557000446804EBC504A34202D36FF0010030BDC0
:105580005C798C4201D00833F0E70020F7E773B56F
:10559000054601A80C461646FDF7B2FE70BB4FF05B
:1055A00080531969B5FBF1F201FB125242BB196934
:1055B000B4FBF1F201FB124212BB1A695B6953435F
:1055C000A3421DD3E4B1019B1B0103F1804101F50E
:1055D000F031C1F80058C1F80448C1F80868D1F8A2
:1055E000002895420FD1D1F8042894420BD1D1F86C
:1055F0000838DBB2B34218BF6FF00D0002B070BDC7
:105600006FF01500FAE76FF00D00F7E70222FFF7E1
:10561000BEBF8068183820F0070010387047042893
:1056200009D0052803D1481E18BF01207047431A2E
:105630005842584170470120704738B515460C460E
:1056400061B15AB1FFF734FD2544214611F8013B01
:10565000834203D1A942F9D1012038BD0020FCE7E3
:1056600038B50C460123114622460546FFF7DBFC00
:1056700000280FDB012221462846FFF7DEFF38B95C
:105680002378012B14BF022301232370002038BD8F
:105690000323FAE70120FAE72DE9F7431D46064602
:1056A0000F469046FFF7FDFC6C1E04444042044048
:1056B000082C1AD83046FFF7FBFC2A4681464146A3
:1056C0006846FFF74EFD621B49460DEB0500FFF7EC
:1056D00053FD23466A4639463046FFF7B9FC003889
:1056E00018BF012003B0BDE8F0834FF0FF30F9E7A9
:1056F00007B501238DF8042001AAFFF7CDFF03B001
:105700005DF804FB81681839012221F00701FFF7D9
:10571000EFBF8268183A22F00702FFF7A1BF13B566
:105720000C46C0B201A9FCF7A3F950B92146019873
:10573000FDF72EFE04460198FFF774FC204602B0E8
:1057400010BD0124FAE713B541EA021104468DF8B1
:105750000710FFF75EFF012301460DF10702204607
:10576000FFF79AFF02B010BD0020704770B50368C4
:10577000CD1A002D02DC6FF05F0070BD93F9006060
:105780001C78002E0ADB5C1C04601B781360036825
:10579000C91A13688B42EED80020EEE704F07F04AC
:1057A000013C032C2BD8DFE804F0020A1421012D60
:1057B000E1D05B781360036802330360E7E7022DF2
:1057C000D9DDB3F801305BBA9BB2136003680333D1
:1057D000F3E7032DCFDD9C785D78DB78240244EA83
:1057E00005442343136003680433E6E7042DC2DD58
:1057F000D3F801301BBA136003680533DDE76FF09F
:105800006300BAE770B404680E1B002E07DD26782B
:105810009E4208D10134046070BCFFF7A7BF6FF04F
:105820005F0070BC70476FF06100FAE773B5022348
:10583000154601AA0446FFF7E5FF40B9019E21681D
:105840003246284600F019FB23683344236002B037
:1058500070BDF0B5844617460E4614460025BCF1CF
:105860000F0F06F1400604F1400477D804096FF0E9
:105870000F0202FB040007284FEA841C01EB841688
:1058800007EB84145DD951F80C10A3FB01126918C1
:1058900057F80C5042F10002491947F80C10716892
:1058A00042F10002A3FB01515219656841F1000168
:1058B00052196260B26841F10001A3FB025249191A
:1058C000A56842F100024919A160F16842F10002A5
:1058D000A3FB01515219E56841F100015219E26040
:1058E000326941F10001A3FB02524919256942F1D5
:1058F000000249192161716942F10002A3FB0151C3
:105900005219656941F1000152196261B26941F1B0
:105910000001A3FB02524919A56942F1000249198D
:10592000A161F16942F10002A3FB01155218E1697E
:1059300045F100055218E26145F1000508382034B0
:1059400020364FEA800C274606EB8000B04240F03C
:1059500006816444002D40F01081F0BD56F8402CC3
:10596000A3FB02E215EB0E0E54F8405C42F100027C
:1059700015EB0E0544F8405C56F83C5C42F1000221
:10598000A3FB05E512EB0E0E54F83C2C45F1000587
:1059900012EB0E0244F83C2C56F8382C45F1000569
:1059A000A3FB02E215EB0E0E54F8385C42F1000244
:1059B00015EB0E0544F8385C56F8345C42F10002F1
:1059C000A3FB05E512EB0E0E54F8342C45F100054F
:1059D00012EB0E0244F8342C56F8302C45F1000539
:1059E000A3FB02E215EB0E0E54F8305C42F100020C
:1059F00015EB0E0544F8305C56F82C5C42F10002C1
:105A0000A3FB05E512EB0E0E54F82C2C45F1000516
:105A100012EB0E0244F82C2C56F8282C45F1000508
:105A2000A3FB02E215EB0E0E54F8285C42F10002D3
:105A300015EB0E0544F8285C56F8245C42F1000290
:105A4000A3FB05E512EB0E0E54F8242C45F10005DE
:105A500012EB0E0244F8242C56F8202C45F10005D8
:105A6000A3FB02E215EB0E0E54F8205C42F100029B
:105A700015EB0E0544F8205C56F81C5C42F1000260
:105A8000A3FB05E512EB0E0E54F81C2C45F10005A6
:105A900012EB0E0244F81C2C56F8182C45F10005A8
:105AA000A3FB02E215EB0E0E54F8185C42F1000263
:105AB00015EB0E0544F8185C56F8145C42F1000230
:105AC000A3FB05E512EB0E0E54F8142C45F100056E
:105AD00012EB0E0244F8142C56F8102C45F1000578
:105AE000A3FB02E215EB0E0E54F8105C42F100022B
:105AF00015EB0E0544F8105C56F80C5C42F1000200
:105B0000A3FB05E512EB0E0E54F80C2C45F1000535
:105B100012EB0E0244F80C2C56F8082C45F1000547
:105B2000A3FB02E215EB0E0E54F8085C42F10002F2
:105B300015EB0E0544F8085C56F8045C42F10002CF
:105B4000A3FB055E521954F8045C4EF1000EAA182E
:105B50004EF1000544F8042CACF1100C7FE656F829
:105B6000042BA3FB0221AA1841F10005396889180A
:105B700047F8041B45F10005E8E623685B1944F883
:105B8000043B2CBF01250025E4E62DE9F04F85B04C
:105B900017460E9C00906268A06803938A469200A4
:105BA0000021FFF7E9FA7E68DAF80430A568B3420D
:105BB00028BF3346741C0193A400A9464FF0000887
:105BC000009BB04598681CD1043C254422462946D8
:105BD000FFF7C7FA2B5901332B510022D7F808E001
:105BE000281F13469E422BD12B5900999B1A2B51EB
:105BF0008968DBB22A46304605B0BDE8F04F00F0B8
:105C0000E6BFDAF8081050F828B0D9F80030086874
:105C1000039A00FB0B335343019802934A465B46B9
:105C2000FFF717FE029BB9684A463046FFF711FEA0
:105C300049F804BB002349F8043008F10108BFE724
:105C400050F804CF5EF82370ACEB0201B9422CBFD0
:105C50004FF000084FF00108C91B94452CBF424685
:105C600008F1010201600133BCE773B501F1804224
:105C7000013A00EB8202824201D202B070BD036899
:105C8000019304230DEB03050024294615F8016B4D
:105C9000013B13F0FF0346EA0424F7D11568019590
:105CA0001D46013311F8016BDBB2042B46EA0525D2
:105CB000F7D140F8045B42F80449DCE700230122F5
:105CC000C0E900238360704710B5044668B180685E
:105CD00030B161688900FDF7CBFDA068FDF7B8FD24
:105CE00000230122C4E90023A36010BD42F2107317
:105CF000994270B504460D4602D96FF00F0070BD91
:105D000043688B4201D30020F9E704212846FDF7C0
:105D100099FD06460028F0D0A16859B1626892004A
:105D2000FFF71FFA6168A0688900FDF7A1FDA06870
:105D3000FDF78EFDC4E90156E5E738B504460D468A
:105D400019B9FFF7C1FF002038BD42688A4207D168
:105D5000806892000021FFF70FFA01232360F2E729
:105D6000FFF7B2FF29462046BDE83840FFF7BEBF27
:105D7000884270B505460E4609D04968426841B967
:105D80002AB10123036092008068FFF7F5F9002033
:105D900070BD4C1E84B9013433682B60944212D913
:105DA00021462846FFF7A2FF0028F1D1B168A86874
:105DB000A200FFF7D6F9EAE7B36853F82430002BC6
:105DC000E9D1013CE6E7A868121B9200002100EB34
:105DD0008400FFF7D1F9E9E770B50E4601210446CA
:105DE000FFF784FF054688B9626801469200A06803
:105DF000FFF7C2F9A36886EAE672002EA2EBE6720C
:105E00001A60ACBF01234FF0FF332360284670BDFA
:105E10004368B1EB431F3FBF83684A0901F01F018C
:105E200053F822003ABFC84000F00100002070473C
:105E300002464068A0B19268431E93B952F82310FD
:105E400000294FF0000008DB4FF00042013020280D
:105E50004FEA520201D01142F8D00133C0EB431097
:105E6000704752F823100029E8D1013BE5E708B557
:105E7000FFF7DEFF0730C00808BD2DE9F04112F042
:105E8000030418BF012404EB920488462146074608
:105E90001546FFF752FF064668B965B1BB68C5EB0A
:105EA00084002A4641461844FFF75BF9B86814B1EC
:105EB0002146FFF7DAFE3046BDE8F081F8B504462A
:105EC00008466368B2EB830F4FEA83051AD9521B69
:105ED0008E180021FFF750F930462A46831800211A
:105EE0008A4211D10020F8BDA16823F0030703F016
:105EF0000306C959F600F140C9B289B90133AB4272
:105F0000F2D1EBE71346FAE7A66821F0030001F0AF
:105F100003053058ED00E84003F8010D0131DFE7DB
:105F20006FF00700DFE7F8B505460E464C0901F0B3
:105F30001F07FFF77DFF6B683044B0EB431F05D8A8
:105F40001F2E0FD8002F41D100200AE010F01F01B2
:105F500018BF012101EB50112846FFF7C7FE0028AA
:105F6000EED0F8BD6B686FF003009A0060431946ED
:105F7000A142A2F104020CD8E21A9C4288BF00227E
:105F800013449B000022043B191DDBD0A968CA50B2
:105F9000F9E7AE6806EB020C01395CF800C046F880
:105FA00002C0E5E7AB6853F8241001FA07F043F8A4
:105FB0002400A86850F82430134340F8243021FA14
:105FC00006F201346B68A342ECD8BDE70022C7F1AA
:105FD0002006F7E7F0B443684C09A34201F01F0222
:105FE00001D309D11AB1F0BC0021FFF7F5BE1F297A
:105FF00004D80020F0BC70471F2909D9A500002350
:106000004168091B99421BD80024416899421ED857
:10601000002AEED043680024C2F12007013BE8D3F8
:10602000816851F8235025FA02F641F8236086680A
:1060300056F82310214346F8231005FA07F4EDE73C
:1060400081684E5941F8236004350133D8E78168EF
:1060500041F823400133D8E710B542683AB94B689C
:1060600073B9B2B9181E18BF0120404210BD836831
:1060700003EB820353F8043C002BF0D1013AEDE727
:106080008C6804EB830454F8044C002CE9D1013BE8
:10609000E6E79A4210D811D3013A836853F82240B8
:1060A0008B6853F822309C4206D802F1FF3205D3A8
:1060B000531CF2D10020D9E70120D7E74FF0FF3081
:1060C000D4E730B54368024623B9486858B9002B75
:1060D00036D12FE0906800EB830050F8040C0028C4
:1060E000F3D1013BF0E78C6804EB800555F8045CC4
:1060F00015BB0138EAE70D6802D20868404220E08B
:106100001068002803DD002D07DA012019E0002DBA
:1061100003DD10B14FF0FF3013E0013B916851F8FF
:10612000235054F823108D420BD803F1FF33E5D3ED
:10613000591CF3D1002004E0002BDED08342DAD9D1
:10614000106830BD1FB581EAE173A3EBE17300294C
:106150000093ACBF01234FF0FF33019301A901234A
:106160000293CDF80CD0FFF7ACFF05B05DF804FB4F
:1061700090422DE9F04106460F46154602D088426E
:1061800029D12F46012333607D6865BB29463046FF
:10619000FFF7ACFD044618BBB368B9689C460746D8
:1061A000854229D103EB8503D7B17268AA4205F174
:1061B000010807D841463046FFF798FD68BBB36831
:1061C00003EB85031A68D21943F8042B2CBF01276F
:1061D00000274546E8E7FFF7CBFD04460028D0D06E
:1061E0002046BDE8F081BB6803EB850353F8043C0F
:1061F000002BCBD1013DC8E7DCF80020D21951F8C3
:1062000020702CBF4FF0010E4FF0000ED2194CF849
:10621000042B4EF100070130C2E70446E0E72DE908
:10622000F843546805460E4690463CB97168A14251
:106230000ED26FF009073846BDE8F883D8F8083069
:1062400003EB840353F8043C002BEFD1013CECE753
:106250002846FFF74BFD07460028ECD17268A242A2
:1062600009D9B168A868121B920001EB840100EB08
:106270008400FEF776FF6A687068824207D9AB68CF
:10628000121A9200002103EB8000FEF775FF002236
:10629000D5F808C0D6F808E0D8F8088013469C4224
:1062A00012D172B14FF0FF316B68A34225D9AB68B0
:1062B00053F82420EAB1AA6852F82430013B42F88E
:1062C000243001232B60B6E75EF8236058F82300E2
:1062D000B11A81422CBF4FF000094FF00109091A91
:1062E0004CF8231096422CBF4A4609F101020133B3
:1062F000D5E743F824100134D6E7DCD199E7F8B5A7
:106300000F6813687B4305460C46164616D51146A2
:106310002046FFF7A1FE002806DB3246214628462C
:10632000FFF77DFF38B1F8BD22462846FFF777FF1B
:106330000028F8D17F422F600020F4E7FFF718FF14
:10634000F0E7F8B50F6813687B43002B05460C4651
:10635000164616DD11462046FFF77EFE002806DBB6
:10636000324621462846FFF75AFF38B1F8BD22468B
:106370002846FFF754FF0028F8D17F422F60002005
:10638000F4E7FFF7F5FEF0E72DE9F0414E6805462A
:106390000F46904646B1BB6803EB860353F8043CB6
:1063A00043B1B8F1000F07D128460021BDE8F04104
:1063B000FFF712BD013EEDE7711C2846FFF796FC82
:1063C000044660B939462846FFF7D2FC044630B986
:1063D000AA68B96808F1FF333046FFF73AFA204659
:1063E000BDE8F0812DE9F04F9DB083460F46184679
:1063F000002116460393FFF7A5FE002800F08781D1
:1064000003230024012517930399169519AB3046F1
:10641000CDE90A54CDE90C45CDE90E44CDE910543F
:10642000CDE91245CDE914441893FFF715FEA042BB
:1064300028DABBF1000F05D1E7B9002420461DB0D2
:10644000BDE8F08F21465846FFF7C6FC04460028F9
:10645000F2D00AA8FFF738FC0DA8FFF735FC10A80A
:10646000FFF732FC13A8FFF72FFC0C2119A8FDF74A
:10647000FFF9E3E731463846FFF77AFC0446002887
:10648000E7D1DAE731460AA8FFF772FC0446002894
:10649000DFD103990DA8FFF76BFC04460028D8D183
:1064A00071680D95023110A80A95FFF71FFC04468C
:1064B0000028CED1014610A8FFF78EFC0446002824
:1064C000C7D1716813A80231FFF710FC04460028F9
:1064D000BFD10DA8FFF7ACFC00F01F001F2870D043
:1064E000C0F11F0319460AA80193FFF71CFD0446DB
:1064F0000028AED101990DA8FFF715FD044600282C
:10650000A7D10B9DDDF83880A5EB080A4FEA4A19A0
:1065100049460DA8FFF707FD0446002899D14FEA28
:106520008A0A0DA90AA8FFF7CCFD00284BDA4946D4
:106530000DA8FFF74FFD044600288AD108F1FF336C
:1065400005939B0005F1FF3A069305F1804508F19C
:106550008043023B013D9B00A5EB08050893AB007F
:106560000293059B9A453DD8BBF1000F0CD010A9B2
:106570005846FFF7FDFB002840F0C580039A3368BA
:1065800012685343CBF80030002F3FF462AF0199FB
:106590000AA8FFF71FFD002840F0B58033680A9372
:1065A0000AA93846FFF7E4FB0146002840F0AD8019
:1065B0003846FFF7C7FD00287FF44BAF01233B604F
:1065C00047E701949DE7129A52F80A300AA901336D
:1065D00042F80A3008460DAAFFF7B3FE0446002829
:1065E0009FD036E70F9B069A04931344DDF8309052
:1065F0000793049B59F82A109A58129D4FEA8A086B
:10660000A8F104030993029B91421D4476D2A8F19C
:106610000400002359F80000F9F772FD002914BFA7
:106620004FF0FF330346BAF1010F2B6016BF09EBA1
:106630000803002353F8083C1993A8F1040359F800
:1066400003301A9359F808301B932B68DDF810803B
:1066500001332B60089B98442B68013B2B60002181
:1066600013A8FFF7B9FB00284DD1059B002B48D09C
:10667000D8F80020159B1A60079A12685A6013A96F
:106680002A680846FFF780FE00283CD116A913A807
:10669000FFF717FD0028DFDC2A680DA913A8FFF714
:1066A00073FE80BB029B4FEAC308414613A8FFF765
:1066B0003AFC40BB0AA9084613AAFFF742FE01466E
:1066C00018BB0AA8FFF73EFD002812DA0DA913A88F
:1066D000FFF74EFBB8B9414613A8FFF724FC90B969
:1066E0000AA913AA0846FFF70AFE60B92B68013B06
:1066F0002B60029B0AF1FF3A043B31E74FF0FF3376
:1067000091E7059AB6E70446A3E60C46A1E66FF0CA
:106710000B0493E670B504460D461046002116465C
:10672000FFF710FD002824DB2A46334621460020CF
:10673000FFF758FE054638B1284670BD324621465F
:106740002046FFF7DCFD90B900212046FFF7FAFC58
:106750000028F3DB31462046FFF7B3FC0028EBDBD3
:10676000324621462046FFF7ECFD0028F2D00546D0
:10677000E2E76FF00905DFE72DE9F04FADF55B7D4E
:10678000064689461846002105921D46FFF7DAFCA9
:10679000002840F31382AB681C6814F001030893CF
:1067A00000F00C8205980021FFF7CCFC0028C0F215
:1067B00005820598FFF73CFBB0F5006F00F2FE8103
:1067C0002846FFF735FBB0F5006F00F2F78104F1C2
:1067D00002084FEA480808F00808A044032108FB13
:1067E00004F3C3F10203013903FB08F8F7D10123D5
:1067F0004FF440721AA8CDE90B31CDE90D13CDE964
:106800000F11CDE91431CDE9113116911391FEF735
:10681000B3FC0598FFF70CFBB0F5287F80F0F580FE
:10682000EF2800F2F4804F2800F2F380089B18282C
:1068300034BF1F4603276B6803F1010A51463046F7
:10684000FFF754FA0446002840F0BD8051461DA8C9
:10685000FFF74CFA0446002840F0B5804FEA4A01A1
:106860000EA8FFF743FA0446002840F0AC80D9F8A0
:106870000030069301330BD1494614A8FFF778FA8C
:106880000446002840F09F80012314930DF1500925
:10689000E49B1BB19B68002B40F0BD8001210BA83D
:1068A000FFF79AFA0446002840F08D8069680BA82B
:1068B0008901FFF738FB0446002840F084800BA9CB
:1068C0002A460846FFF726FF044600287BD1E49BB2
:1068D00023B10C220BA91846FEF743FC2946484673
:1068E000FFF7EFFB0028C0F29A802A4649461DA810
:1068F000FFF710FF0446002865D169681DA8013123
:10690000FFF7F4F9044600285DD10DF1380BC8F10A
:1069100000032A460BA91DA8CDF800B00393FFF78A
:1069200034F90BA93046FFF723FA044600284AD170
:1069300001230AAACDE917330A931992039BCDF8D4
:1069400000B02A4617A93046FFF71FF9012F6BD177
:10695000059B4FF0000A5B680493D046D346D146AE
:10696000BBF1000F40F0AF80049B002B40F0A680ED
:106970004FF0010B0BFA07FB0DF1380A049B43455E
:1069800040F0FA8001230AAACDE917330A9319923D
:10699000039BCDF800A02A4617A93046FFF7F5F86B
:1069A000069B01330FD1059B5B6863B1059B9B6818
:1069B0001B68DB0707D5069B336032462946304605
:1069C000FFF79DFC04467D1E012303FA07F603FA38
:1069D00005F50C27AE4200F2EA801DA8FFF774F916
:1069E0000EA8FFF771F914A8FFF76EF911A8FFF7C9
:1069F0006BF9E49B0BB19B6813B90BA8FFF764F923
:106A000020460DF55B7DBDE8F08F062713E70527CF
:106A100011E704270FE7E4990C220BA85CE749462D
:106A20001DA8FFF7A5F96DE707F1FF390C23696889
:106A300003FA09F31AAA02EB030801314046FFF7F3
:106A400055F90028BED11DA94046FFF791F900284D
:106A5000B8D1A246039BCDF800B02A464146404635
:106A60000AF1010AFFF791F8CA45F3D34FF0010A82
:106A70000AFA09F9D1440AFA07FACA457FF668AF5B
:106A8000696808F10C0B01315846FFF72FF900280F
:106A900098D141465846FFF76BF9002892D10EABCA
:106AA00000932A46039B1DA95846FFF76EF809F18B
:106AB0000109D846E1E74FF0020A51E7049B013B88
:106AC00004934FF0200B059B049A9B6853F82230E7
:106AD0000BF1FF3B23FA0BF313F001030FD1BAF1D3
:106AE000000F3FF43DAFBAF1010F08D10EAB009398
:106AF0002A46039B31463046FFF747F830E708F156
:106B00000108A7EB08029340474549EA0309D2D19F
:106B10004FF0000A0EAB00932A46039B31463046E5
:106B20000AF1010AFFF731F8D045F3D8012303FA3F
:106B300008F34FF0000A0DF16808494650460993E2
:106B400000F03FF84146C2B211A800F052F8079099
:106B500058BB099B0AF1010A534508F10C08ECD116
:106B60000EAB00932A46039B11A93046FFF70DF8A0
:106B7000DDE9079AC846F3E6039BCDF800A02A4654
:106B8000314630464FEA4909FEF7FFFF1BEA090F7D
:106B900007D0039BCDF800A02A461DA93046FEF77A
:106BA000F4FF049B01330493E8E6079C0BE71AAB60
:106BB00007FB0530FFF788F801350BE76FF003049A
:106BC0001EE7414048420843C043C00F7047F0B53C
:106BD00004395F420025013B854200D1F0BD52F8E7
:106BE000256051F8044F3E401C4034430C60013591
:106BF000F2E72DE9F8430F46496805469146FFF74D
:106C000075F88046C8B92B683C68A968013301341F
:106C10005C4004EA49045C40013C2C60C9F1000678
:106C20004B46BA68786846EA0906FFF7D0FFF617C0
:106C30007B68F6436A689A4202D84046BDE8F8830A
:106C4000A96851F82320324041F823200133F1E7AD
:106C500000207047704770472DE9F8430446DDE98E
:106C60000876914698460D4651B9B9F1000F10D1FA
:106C7000B8F1000F15D1E7B91EBB55BB002006E0E7
:106C80000830FFF775F80028EFD0A0F58140BDE887
:106C9000F883494604F12C00FFF76AF80028E7D092
:106CA000F3E7414604F13800FFF762F80028E2D02C
:106CB000EBE7394604F12000FFF75AF80028DBD053
:106CC000E3E7314604F11400FFF752F80028D4D06E
:106CD000DBE704F10800FFF7CAF86060CEE710B503
:106CE000AC2200210446FEF747FA0023C4E9293309
:106CF00010BD10B50446A0B38C30FEF7E5FF04F1DB
:106D00009800FEF7E1FF04F16800FEF7DDFF04F1F3
:106D10002000FEF7D9FF04F13800FEF7D5FF04F19B
:106D20002C00FEF7D1FF04F11400FEF7CDFF04F1B3
:106D30000800FEF7C9FF04F18000FEF7C5FF04F16B
:106D40007400FEF7C1FF04F15C00FEF7BDFF04F123
:106D50005000FEF7B9FF04F14400BDE81040FEF713
:106D6000B3BF10BD6C220021FEF706BA2DE9F8432F
:106D700005460E4614467AB3036803F03F079B1896
:106D8000036022BF4368013343609FB1C7F14009EC
:106D90004A450FD300F128084A4608EB0700FEF7E2
:106DA000E0F941462846FCF799FEB0B93C444E4410
:106DB000403C0746264404E02846FCF78FFE60B9B5
:106DC000403C3F2CA6EB0401F6D82CB105F128007D
:106DD00022463844FEF7C5F90020BDE8F88370B5B7
:106DE000036803F03F035A1C03440D4600F12806D4
:106DF0008021382A044683F8281006EB020061D867
:106E0000C2F138020021FEF7B7F9D4E900315A0F78
:106E100042EAC102DB0012BA1BBA2266636631463F
:106E20002046FCF75BFE00284BD1E37A2B70638988
:106E30006B70A3681B0AAB70A368EB70E37B2B71CC
:106E4000E3896B71E3681B0AAB71E368EB71E37C68
:106E50002B72638A6B7223691B0AAB722369EB7214
:106E6000E37D2B73E38A6B7363691B0AAB736369FE
:106E7000EB73E37E2B74638B6B74A3691B0AAB7497
:106E8000A369EB74E37F2B75E38B6B75E3691B0AD6
:106E9000AB75E369EB7594F823302B76638C6B76D6
:106EA000236A1B0AAB76236AEB76A36E4BB994F880
:106EB00027302B77E38C6B77636A1B0AAB77636AA7
:106EC000EB7770BD0021C2F14002FEF755F9314663
:106ED0002046FCF703FE0028F3D101463822304655
:106EE00091E7004700F028B9F7B5044618B101282A
:106EF00020D003B0F0BD4FF080430222C3F8082336
:106F0000C3F80401D3F804210122DA600746012303
:106F10008DF8073042F210754FF08046BCB1012C5D
:106F2000E7D18FB3D6F80C3403F001033B70D6F8E9
:106F30000C3414E04FF080430022C3F80803C3F878
:106F40000021D3F8002158600DF10707DFE78FB16A
:106F5000D6F8183403F003033B60D6F81834DA038C
:106F6000C7D59DF807000128C3D1FFF7BBFF013D3E
:106F7000D4D1BEE7D6F81834D903BAD50120FFF72B
:106F8000B1FF013DF6D1B4E7D6F80C34DB03B0D540
:106F90000120FFF7A7FF013DF6D1AAE708B50020C1
:106FA000FAF70CFE08B9FAF7FBFD4FF08043002218
:106FB000C3F8182508BD08B510B101282CD008BDAC
:106FC0004FF08042D2F81834D2F81814C8030BD40A
:106FD000D2F81434D9070FD5D2F81C349B0708D443
:106FE0000223C2F80433EAE703F00303012B04D0C1
:106FF00013B10020FFF778FF00234FF08042C2F862
:1070000018350023C2F80431D2F804310223C2F843
:10701000043301239360D2E74FF080430022C3F88A
:107020000021D3F80021C3F804031860C7E7FFF775
:107030005BBFF7B5019001A8DDE9084716461D467C
:10704000FCF728FF019BB6F1000C18BF4FF0010CB4
:1070500000EB83000B1E18BF0123002D43EA4C03F5
:1070600014BF4FF00C0C4FF0000C002C43EA0C0343
:1070700014BF4FF4E06C4FF0000C002F43EA0C03F8
:10708000D0F8002714BF4FF4403C4FF0000C43EA07
:107090000C0322EA030301B109780EB136787600B9
:1070A00019430DB12D78AD0031430CB12478240281
:1070B00029430FB13F783F040C433C43C0F80047DD
:1070C00003B0F0BD1FB50DF10F03019300238DF840
:1070D0000F1000931A461946FFF7ABFF05B05DF895
:1070E00004FB4FF080531A695869504370474FF0C2
:1070F0008053186970474FF0805358697047FDF707
:1071000071BA08B5FFF7FBFF002008BD704740B11A
:10711000C368587810F001001EBF1878B0FA80F0EC
:1071200040097047FEF728B8FEF71BB8EFF305805B
:10713000003818BF0120704708B1FBF737B9704716
:10714000F48FFF7F010000005123000000000000C9
:1071500069240000A071000003710000000000001D
:107160008D270000B87100008D270000D07100004D
:1071700015550000E8710000335500000072000052
:107180006926000000000000F52F0000000000004C
:10719000695700000000000051290000187200002B
:1071A000A58100001075000028750000DC0000209B
:1071B0000C0E0020CE730000CE810000447500004C
:1071C00064750000DE000020600E0020C87300001F
:1071D000DC8100005475000064750000E0000020B0
:1071E0006C0E0020C27300009B820000A47500009A
:1071F00004760000E400002014000020BC730000AE
:10720000A9820000D075000004760000E60000208E
:1072100030000020B6730000538200000000000020
:1072200088750000E200002000000000B07300003C
:10723000313E0000E36E0000000000000B51000032
:1072400000720000A3540000000000000B51000079
:10725000000000000B510000000000000B51000076
:10726000A9430000E36E0000000000000B51000085
:10727000000000000B510000000000000B51000056
:10728000000000000B510000000000000B51000046
:10729000000000000B510000000000000B51000036
:1072A000000000000B510000000000000B51000026
:1072B000000000000B5100000000000075300000CD
:1072C000000000000B510000000000000B51000006
:1072D000000000000B510000000000000B510000F6
:1072E000000000000B510000000000000B510000E6
:1072F000000000000B510000000000000B510000D6
:10730000000000000B510000000000000B510000C5
:10731000000000000B510000000000000B510000B5
:10732000000000000B510000000000000B510000A5
:10733000000000000B510000000000000B51000095
:10734000000000000B510000000000000B51000085
:10735000000000000B510000000000000B51000075
:10736000000000000B510000000000000B51000065
:10737000E8710000A3540000000000000B51000061
:10738000000000000B510000000000000B51000045
:10739000000000000B510000000000000B51000035
:1073A000000000000B510000000000000B51000025
:1073B00000800080FF7F00800080FF7F00800080D1
:1073C000FF7F00800080FF7F00800080FF7F0080C3
:1073D0000080FF7F91830000000000009C8300007C
:1073E00000000000A883000000000000B18300003E
:1073F00000000000A17C000003000000C08100002C
:1074000003000000DD820000030000006D82000028
:107410000300000032780000030000003B81000000
:10742000030000009E84000003000000A181000012
:1074300003000000B782000003000000FFFFFFFF11
:107440000338FDD87047000001000000937B000066
:10745000547400000E01000007000000000000004E
:107460000000000000C000001872000001000000D1
:1074700000C00000000200001872000002000000BE
:1074800000C000000090030018720000030000001C
:1074900000C20000008E030018720000040000000B
:1074A00000C20000008E03001872000005000000FA
:1074B0000050040000900300187200000600000055
:1074C00000E007000020000018720000000000200B
:1074D0000000000000000B06C03400204000000047
:1074E00000000B1502000000EC740000000000001A
:1074F0009281000024000202000000209A81000016
:1075000020000B11F1230000C12300000000000047
:107510001125000035240000B4810000A3520000B2
:10752000A9520000BA8100008B5200001B520000DB
:107530007D5200000000000091510000000000009A
:1075400000000000FF0300000003005000000000E6
:1075500001000000FFFFFFFF0000005000000000DE
:107560000000000011280000AF520000BD520000D2
:10757000D5520000E1520000ED520000B926000093
:107580000753000000000000412A0000D529000038
:107590006929000049290000392900000400000081
:1075A000FF00000000800240020000000000000018
:1075B000B475000000800240C075000001000000AA
:1075C000C875000002000000A101010022000000B7
:1075D000002000400200000000000000E0750000F4
:1075E00000200040EC75000001000000F475000070
:1075F00004000000060000000500020088010100F0
:10760000870103005B540000792A00004D540000FC
:107610003D2B00003D540000982F8A429144377161
:10762000CFFBC0B5A5DBB5E95BC25639F111F15905
:10763000A4823F92D55E1CAB98AA07D8015B831247
:10764000BE853124C37D0C55745DBE72FEB1DE80F3
:10765000A706DC9B74F19BC1C1699BE48647BEEF22
:10766000C69DC10FCCA10C246F2CE92DAA84744AAD
:10767000DCA9B05CDA88F97652513E986DC631A823
:10768000C82703B0C77F59BFF30BE0C64791A7D502
:107690005163CA0667292914850AB72738211B2E8A
:1076A000FC6D2C4D130D385354730A65BB0A6A7672
:1076B0002EC9C281852C7292A1E8BFA24B661AA87E
:1076C000708B4BC2A3516CC719E892D1240699D68E
:1076D00085350EF470A06A1016C1A419086C371E07
:1076E0004C774827B5BCB034B30C1C394AAAD84EE5
:1076F0004FCA9C5BF36F2E68EE828F746F63A57820
:107700001478C8840802C78CFAFFBE90EB6C50A4B2
:10771000F7A3F9BEF27871C65484000062840000B9
:107720007684000085840000918400004871000088
:10773000487100008871000090710000A071000085
:10774000A071000077C295F360D2EF7F3552500FE1
:107750002CB6798025633A205374617274696E6720
:1077600020626F6F746C6F616465720A0025633A02
:1077700020556E61626C6520746F2066696E6420AE
:10778000626F6F7461626C6520696D6167650A0084
:1077900025633A20426F6F746C6F61646572206379
:1077A0006861696E6C6F6164206164647265737393
:1077B000206F66667365743A20307825780A002554
:1077C000633A204A756D70696E6720746F20746823
:1077D0006520666972737420696D61676520736CDA
:1077E0006F740A0025633A2050726F7465637420C9
:1077F0006D6375626F6F7420666C6173682066617B
:10780000696C65642C2063616E63656C20737461C0
:10781000727475702E0A0025633A204E6576657283
:107820002073686F756C6420676574206865726585
:107830000A006D6375626F6F740025633A20696E8C
:1078400076616C696420666C617368204944202508
:10785000643B2065787065637465642025640A0064
:10786000000000000000000025633A20556E6162B0
:107870006C6520746F2064657465726D696E652037
:10788000666C61736820736563746F72206F662025
:1078900074686520696D61676520747261696C65E3
:1078A000720A007072696D617279007365636F6E40
:1078B000646172790025633A20496D6167652069CA
:1078C0006E2074686520257320736C6F7420697353
:1078D000206E6F742076616C6964210A0025633A1A
:1078E00020256420737461747573207772697465E0
:1078F000206661696C7320706572666F726D696E67
:10790000672074686520737761700A0025633A20E8
:107910004661696C65642072656164696E67207395
:107920006563746F72733B20424F4F545F4D4158F3
:107930005F494D475F534543544F52533D256420A3
:107940002D20746F6F20736D616C6C3F0A0025638E
:107950003A204661696C65642072656164696E678E
:1079600020696D61676520686561646572733B209D
:10797000496D6167653D25750A0025633A204661BA
:10798000696C65642072656164696E6720626F6FFF
:1079900074207374617475733B20496D6167653D34
:1079A00025750A0025633A2070616E6963210A001B
:1079B00025633A20446574656374656420696E6369
:1079C0006F6E73697374656E74207374617475730C
:1079D000210A0025633A2043616E6E6F7420757032
:1079E00067726164653A206E6F74206120636F6D09
:1079F00070617469626C6520616D6F756E74206F63
:107A00006620736563746F72730A0025633A2043BE
:107A1000616E6E6F7420757067726164653A206D77
:107A20006F726520736563746F7273207468616E22
:107A300020616C6C6F7765640A0025633A204361AE
:107A40006E6E6F7420757067726164653A206E6F38
:107A5000742073616D6520736563746F72206C614F
:107A6000796F75740A0062616400676F6F640075F6
:107A70006E736574005072696D61727920696D6111
:107A800067650025633A2025733A206D6167696355
:107A90003D25732C20737761705F747970653D307C
:107AA0007825782C20636F70795F646F6E653D3048
:107AB0007825782C20696D6167655F6F6B3D307844
:107AC00025780A005365636F6E6461727920696D71
:107AD0006167650025633A20426F6F7420736F758C
:107AE0007263653A207072696D61727920736C6F90
:107AF000740A0025633A20426F6F7420736F7572A9
:107B000063653A206E6F6E650A0025633A205374F0
:107B1000617274696E672073776170207573696E26
:107B200067206D6F766520616C676F726974686D30
:107B30002E0A0025633A204E6F7420656E6F7567BC
:107B400068206672656520737061636520746F20BC
:107B500072756E20737761702075706772616465ED
:107B60000A0025633A207265717569726564202583
:107B70006420627974657320627574206F6E6C790D
:107B80002025642061726520617661696C61626C98
:107B9000650A003082010A0282010100D106081A3A
:107BA00018442C18E8FBFDF70DA34F1FBBEE5EF940
:107BB000AAD24B18D35AE96D188019F9F09C341BDE
:107BC000CBF3BC74DB42E78C7F10537E435E0D57D2
:107BD0002C44D167080F0DBB5CEEECB399DFE04D90
:107BE000840BAA774160ED152849A701B43C10E643
:107BF000698C2F5FAC414D9E5C14DFF2F8CF3D1EC7
:107C00006FE75BBAB4A9C8887E473C94C3776754D2
:107C10004BAA8D3835CA62617EB7E115DB7773D424
:107C2000BE7B7221896924FBF8656E643EC80ED75D
:107C300085D55C4AE4530D2FFFB7FDF31339833F1D
:107C4000A3AED20FA76A9DF9FEB8CEFA2ABEAFB88E
:107C5000E0FA823754F43EE12BD0D3085818F65E90
:107C60004CC8888131AD5FB08217F28A692723F34F
:107C7000AB873E931A1DFEE8F81A246659F81CAB30
:107C8000DCCE681B666435ECFA0D119DAF5C3AA73B
:107C9000D167C647EFB14B2C62E1D1C902030100A5
:107CA0000163627072696E74665F7061636B6167B5
:107CB00065002D002B00307800305800286E696C6C
:107CC000290025633A2072302F61313A2020307824
:107CD00025303878202072312F61323A20203078D8
:107CE00025303878202072322F61333A20203078C6
:107CF000253038780A0025633A2072332F61343AF0
:107D00002020307825303878207231322F69703A4F
:107D10002020307825303878207231342F6C723A38
:107D200020203078253038780A0025633A202078E2
:107D30007073723A20203078253038780A00256335
:107D40003A204661756C74696E6720696E7374724F
:107D5000756374696F6E2061646472657373202843
:107D60007231352F7063293A203078253038780AFF
:107D70000025633A202A2A2A2A2A204D50552046D7
:107D800041554C54202A2A2A2A2A0A0025633A20DF
:107D90002020537461636B696E67206572726F7225
:107DA0002028636F6E746578742061726561206D40
:107DB00069676874206265206E6F742076616C69F3
:107DC00064290A0025633A202020556E737461638C
:107DD0006B696E67206572726F720A0025633A20C4
:107DE0002020446174612041636365737320566988
:107DF0006F6C6174696F6E0A0025633A2020204D14
:107E00004D46415220416464726573733A20307864
:107E100025780A0025633A202020496E7374727514
:107E20006374696F6E204163636573732056696F75
:107E30006C6174696F6E0A0025633A202020466CDD
:107E40006F6174696E672D706F696E74206C617AF2
:107E500079207374617465207072657365727661E0
:107E600074696F6E206572726F720A0025633A2022
:107E70002A2A2A2A2A205553414745204641554C53
:107E800054202A2A2A2A2A0A0025633A202020443C
:107E900069766973696F6E206279207A65726F0AFC
:107EA0000025633A202020556E616C69676E656419
:107EB000206D656D6F7279206163636573730A006D
:107EC00025633A2020204E6F20636F70726F6365C8
:107ED00073736F7220696E737472756374696F6EF9
:107EE000730A0025633A202020496C6C6567616C39
:107EF000206C6F6164206F66204558435F52455483
:107F000055524E20696E746F2050430A0025633A23
:107F1000202020496C6C6567616C20757365206F4B
:107F2000662074686520455053520A0025633A2044
:107F30002020417474656D707420746F20657865BD
:107F40006375746520756E646566696E6564206925
:107F50006E737472756374696F6E0A0025633A20DC
:107F60002A2A2A2A2A20425553204641554C542079
:107F70002A2A2A2A2A0A0025633A202020537461DB
:107F8000636B696E67206572726F720A0025633ACF
:107F900020202050726563697365206461746120DC
:107FA000627573206572726F720A0025633A202031
:107FB000204246415220416464726573733A203016
:107FC0007825780A0025633A202020496D70726573
:107FD00063697365206461746120627573206572E2
:107FE000726F720A0025633A202020496E73747202
:107FF000756374696F6E20627573206572726F723B
:108000000A00526573657276656420457863657011
:1080100074696F6E20280053707572696F757320D4
:10802000696E74657272757074202849525120000F
:1080300025633A20535053454C20696E2074687272
:10804000656164206D6F646520646F6573206E6F79
:108050007420696E646963617465205053500A002E
:1080600025633A202A2A2A2A2A20484152442046B7
:1080700041554C54202A2A2A2A2A0A0025633A20EC
:108080002020427573206661756C74206F6E2076B7
:108090006563746F72207461626C652072656164DF
:1080A0000A0025633A2020204465627567206576C2
:1080B000656E740A0025633A2020204661756C7451
:1080C00020657363616C6174696F6E2028736565E8
:1080D0002062656C6F77290A0025633A204152437C
:1080E000485F45584345505420776974682072654D
:1080F00061736F6E2025780A0A0025633A202A2AC8
:108100002A2A2A204465627567206D6F6E69746F34
:108110007220657863657074696F6E202A2A2A2A36
:108120002A0A0025633A202A2A2A2A2A202573208F
:10813000256429202A2A2A2A2A0A006D707500251A
:10814000633A20506172746974696F6E2025753AC4
:108150002073616E69747920636865636B20666162
:10816000696C65642E0A0025633A204661696C6576
:108170006420746F20616C6C6F63617465206E6540
:1081800077204D505520726567696F6E2025750AFE
:108190000A00464C4153485F30005352414D5F3016
:1081A00000736F6300636C6F636B4034303030304A
:1081B000303030006866636C6B006C66636C6B001B
:1081C000636C6F636B5F636F6E74726F6C0067706C
:1081D000696F403530303030333030006770696F50
:1081E0004035303030303030300025633A20756E05
:1081F000616C69676E656420616464726573733A6B
:108200002030782530386C783A257A750A00256355
:108210003A20696E76616C6964206164647265738A
:10822000733A2030782530386C783A257A750A0010
:1082300025633A206E6F7420776F72642D616C69CC
:10824000676E65643A2030782530386C783A257A44
:10825000750A00666C6173682D636F6E74726F6C63
:108260006C657240343030316530303000666C619E
:1082700073685F6E72660025633A204661696C65BB
:108280006420746F20616C6C6F6361746520505062
:1082900049204368616E6E656C0A007561727440B6
:1082A00034303032383030300075617274403430E0
:1082B00030303230303000756172745F6E726678C3
:1082C0005F75617274650025633A20526573657449
:1082D00074696E672073797374656D0A00666174E2
:1082E000616C5F6572726F72007065726D007465AB
:1082F0007374004255473B2063616E2774206861A8
:108300007070656E007265766572740025633A2040
:108310005365636F6E6461727920696D6167652072
:108320006F6620696D61676520706169722028251C
:10833000642E2920697320756E72656163686162BD
:108340006C652E20547265617420697420617320FD
:10835000656D7074790A0025633A20537761702047
:10836000747970653A2025730A0025633A205377A3
:10837000617020747970653A206E6F6E650A000432
:1083800001040304020401040104030103030401C2
:10839000044E5246585F434C4F434B004E52465892
:1083A0005F4750494F5445004E5246585F50504920
:1083B000004E5246585F574454005465726D696EC2
:1083C000616C005254540053454747455200556E66
:1083D0006B6E6F776E206572726F720025633A2044
:1083E0003E3E3E205A455048595220464154414C49
:1083F000204552524F522025643A202573206F6E3B
:10840000204350552025640A0025633A20466175B3
:108410006C7420647572696E6720696E746572721F
:108420007570742068616E646C696E670A0A007505
:108430006E6B6E6F776E0025633A204375727265BE
:108440006E74207468726561643A20257020282556
:1084500073290A0043505520657863657074696F0D
:108460006E00556E68616E646C656420696E74653B
:10847000727275707400537461636B206F766572ED
:10848000666C6F77004B65726E656C206F6F7073F2
:10849000004B65726E656C2070616E6963006F736E
:1084A000002A2A2A20426F6F74696E67205A65700D
:1084B000687972204F53206275696C642076332E80
:1084C000322E39392D6E637332202A2A2A0A00008F
:1084D000FFFFFFFFFFFFFFFF394E00005C7400004D
:1084E0008B5100000000000000C2010000010300E9
:1084F000000000005A280020592800200000000039
:108500000000000000C201000001030000000000A4
:108510005C2800205B28002000000000556C000053
:10852000576C0000516C0000795100000090D0039E
:10853000000000000000000000000000000000003B
:10854000000000000000000000000000000000002B
:10855000000000000000000000000000000000001B
:10856000000000000000000000000000000000000B
:1085700000000000000000000000000000000000FB
:1085800000000000000000000000000000000000EB
:1085900000000000FF0000000000000000000000DC
:1085A000FFFF0F00D4000020D400002000000000D6
:0C85B000000000000000000015E015E0D5
:10C000003DB8F39600000000000200004852030013
:10C010000000000000000000000000000000000020
:10C02000FFFFFFFFFFFFFFFFFFFFFFFFFFFFFFFF20
:10C03000FFFFFFFFFFFFFFFFFFFFFFFFFFFFFFFF10
:10C04000FFFFFFFFFFFFFFFFFFFFFFFFFFFFFFFF00
:10C05000FFFFFFFFFFFFFFFFFFFFFFFFFFFFFFFFF0
:10C06000FFFFFFFFFFFFFFFFFFFFFFFFFFFFFFFFE0
:10C07000FFFFFFFFFFFFFFFFFFFFFFFFFFFFFFFFD0
:10C08000FFFFFFFFFFFFFFFFFFFFFFFFFFFFFFFFC0
:10C09000FFFFFFFFFFFFFFFFFFFFFFFFFFFFFFFFB0
:10C0A000FFFFFFFFFFFFFFFFFFFFFFFFFFFFFFFFA0
:10C0B000FFFFFFFFFFFFFFFFFFFFFFFFFFFFFFFF90
:10C0C000FFFFFFFFFFFFFFFFFFFFFFFFFFFFFFFF80
:10C0D000FFFFFFFFFFFFFFFFFFFFFFFFFFFFFFFF70
:10C0E000FFFFFFFFFFFFFFFFFFFFFFFFFFFFFFFF60
:10C0F000FFFFFFFFFFFFFFFFFFFFFFFFFFFFFFFF50
:10C10000FFFFFFFFFFFFFFFFFFFFFFFFFFFFFFFF3F
:10C11000FFFFFFFFFFFFFFFFFFFFFFFFFFFFFFFF2F
:10C12000FFFFFFFFFFFFFFFFFFFFFFFFFFFFFFFF1F
:10C13000FFFFFFFFFFFFFFFFFFFFFFFFFFFFFFFF0F
:10C14000FFFFFFFFFFFFFFFFFFFFFFFFFFFFFFFFFF
:10C15000FFFFFFFFFFFFFFFFFFFFFFFFFFFFFFFFEF
:10C16000FFFFFFFFFFFFFFFFFFFFFFFFFFFFFFFFDF
:10C17000FFFFFFFFFFFFFFFFFFFFFFFFFFFFFFFFCF
:10C18000FFFFFFFFFFFFFFFFFFFFFFFFFFFFFFFFBF
:10C19000FFFFFFFFFFFFFFFFFFFFFFFFFFFFFFFFAF
:10C1A000FFFFFFFFFFFFFFFFFFFFFFFFFFFFFFFF9F
:10C1B000FFFFFFFFFFFFFFFFFFFFFFFFFFFFFFFF8F
:10C1C000FFFFFFFFFFFFFFFFFFFFFFFFFFFFFFFF7F
:10C1D000FFFFFFFFFFFFFFFFFFFFFFFFFFFFFFFF6F
:10C1E000FFFFFFFFFFFFFFFFFFFFFFFFFFFFFFFF5F
:10C1F000FFFFFFFFFFFFFFFFFFFFFFFFFFFFFFFF4F
:10C20000C0820020C11F0200716A0300951F020056
:10C21000951F0200951F0200951F020000000000FC
:10C2200000000000000000000000000021180200D3
:10C23000951F020000000000CD170200951F0200AC
:10C24000D118020045980300D1180200D11802004D
:10C25000D1180200D1180200D1180200D118020032
:10C260000D980300D1180200D11802002B9803008A
:10C27000D1180200D1180200D1180200D118020012
:10C28000D1180200D1180200D1180200D118020002
:10C29000D1180200D1180200D1180200D1180200F2
:10C2A000D1180200D1180200D1180200D1180200E2
:10C2B000D1180200D1180200D1180200D1180200D2
:10C2C000D1180200D1180200D1180200D1180200C2
:10C2D000D1180200D1180200D1180200D1180200B2
:10C2E000D1180200D1180200D1180200D1180200A2
:10C2F000D1180200D1180200D1180200D118020092
:10C3000053B94AB9002908BF00281CBF4FF0FF31BC
:10C310004FF0FF3000F00CB8ADF1080C6DE904CE21
:10C320000CF056F8DDF804E0DDE9022304B07047B4
:10C33000704700BF2DE9F00791E8F807B2E8021056
:10C340005B1854EB0C04B2E802104D4156EB0C069E
:10C35000B2E802104F4158EB0C08B2E8021059EB5A
:10C3600001095AEB0C0A80E8F80780410130BDE86A
:10C37000F00770472DE9F00791E8F807B2E80210DE
:10C380005B1A74EB0C04B2E802108D4176EB0C06DC
:10C39000B2E802108F4178EB0C08B2E8021079EB9A
:10C3A00001097AEB0C0A80E8F80780414042BDE8B9
:10C3B000F00770472DE9F007524290E87800B1E8A5
:10C3C00080071740DB1918EA020854EB080419EA41
:10C3D000020955EB09051AEA020A56EB0A0678C06B
:10C3E00090E87800B1E8800717407B4118EA02081E
:10C3F00054EB080419EA020955EB09051AEA020A86
:10C4000056EB0A0678C080410130BDE8F00770475E
:10C410002DE9F007524290E87800B1E88007174014
:10C42000DB1B18EA020874EB080419EA020975EB31
:10C4300009051AEA020A76EB0A0678C090E8780045
:10C44000B1E880071740BB4118EA020874EB080402
:10C4500019EA020975EB09051AEA020A76EB0A06DF
:10C4600078C080414042BDE8F00770472DE9F001F7
:10C4700052424FF0040890E8300091E8C000A31B3E
:10C480001340E41AF618EB1B1340ED1AFF1830C0E6
:10C49000C0C1B8F10108EED1BDE8F001704700BF9E
:10C4A00000B592E8DC072DE9DC07B1E8805702B45B
:10C4B000A7FB02510A95A8FB020BE7FB6310E9FBFF
:10C4C00062B00B91A8FB0351EAFB6201E7FB64B584
:10C4D000E7FB6605E8FB6615CDF830B0A9FB03B6AF
:10C4E000EAFB6316ECFB6356E8FB640BE9FB641B99
:10C4F000EAFB645BECFB646B0D90ACFB0230059CCB
:10C50000EEFB6250E9FB6460EAFB64B0E7FB643178
:10C51000E8FB6451069CE8FB6461E9FB64B1EAFB5B
:10C5200064010E93A7FB0432079CE7FB6462E8FBFF
:10C5300064B2E9FB6402EAFB6412049CE9FB645305
:10C54000EAFB6463089CE7FB64B3E8FB6403E9FB74
:10C550006413EAFB64230F955DF8049B99E80006D9
:10C56000DDF80080A9FB0854EAFB68B4DDF8108010
:10C57000ECFB6804EEFB6814E9FB6824EAFB683412
:10C58000DDF80480EEFB6865E9FB68B5EAFB680549
:10C59000DDF81480ECFB6815EEFB6825E9FB6835D7
:10C5A000EAFB68450F96DDF80880AEFB0876E9FBEC
:10C5B0006806EAFB6816DDF81880ECFB6826EEFBDF
:10C5C0006836E9FB6846EAFB6856DDF80C80ECFB50
:10C5D00068B7EEFB6807E9FB6817EAFB6827DDF838
:10C5E0001C80ECFB6837EEFB6847E9FB6857EAFB09
:10C5F000686708B000BD00BF2DE9F14F87B0FFF7B5
:10C600004FFFDDF81C8008F1200888E8FF00FFBC20
:10C6100087E87F08BDE8F08F00B591E89857A3FB45
:10C6200003520195A3FB0401E3FB6420E3FB6710C5
:10C630000292A3FB0752E3FB6802E4FB6415E3FBF1
:10C640006805E3FB69250391A4FB07B6E3FB6926B4
:10C65000E3FB6A56E4FB670BE4FB682BE3FB6A5BD6
:10C66000E3FB6C6B0490A4FB0810E4FB6950E3FB54
:10C670006C60E3FB6EB0E7FB6721E4FB6951E4FB10
:10C680006A61E3FB6EB1E4FB6E010592A7FB083221
:10C69000E4FB6A62E4FB6CB2E4FB6E02E7FB6E1241
:10C6A000E7FB6853E7FB6963E4FB6CB3E7FB6C03F0
:10C6B000E7FB6E13E8FB6E230695A7FB0954E7FB27
:10C6C0006AB4E7FB6C04E8FB6C14E8FB6E24E9FB3E
:10C6D0006E34E8FB6865E7FB6AB5E8FB6A05E8FBD2
:10C6E0006C15E9FB6C25E9FB6E35EAFB6E45079698
:10C6F000A8FB0976E8FB6A06E9FB6A16E9FB6C26EB
:10C70000EAFB6C36EAFB6E46ECFB6E56E8FB69B75B
:10C71000E9FB6907E9FB6A17EAFB6A27EAFB6C3762
:10C72000ECFB6C47ECFB6E57EEFB6E6700BD00BF89
:10C730002DE9F14F87B0FFF76FFFDDF81C8008F19E
:10C74000200888E8FF00FFBC87E87F08BDE8F08F7D
:10C7500030B44FF0000310F8014B11F8015B013ABF
:10C7600084EA050443EA0403F5D1A3F101034FEA87
:10C77000D37030BC704700BF4FF0000310F8012B9E
:10C78000013943EA0203F9D1A3F101034FEAD3705F
:10C79000704700BF30B411F8014B12F8015B6C40D8
:10C7A00000F8014B013BF6D130BC70472DE9F00792
:10C7B00091E8F807B2E802105B1854EB0C04B2E8F9
:10C7C00002104D4156EB0C06B2E802104F4158EBF7
:10C7D0000C08B2E8021059EB01095AEB0C0A894126
:10C7E000B3F1FF3374F1FF3475F1FF3576F10006D4
:10C7F00077F1000778F1000879F101097AF1FF3A41
:10C8000051F100015B184C414D4156F1000657F1C2
:10C81000000758F1000859EBD1795AEB010A80E87A
:10C82000F807BDE8F00770472DE9F00791E8F80731
:10C83000B2E802105B1A74EB0C04B2E802108D41EE
:10C8400076EB0C06B2E802108F4178EB0C08B2E8E8
:10C85000021079EB01097AEB0C0A89415B184C4113
:10C860004D4156F1000657F1000758F1000859EB09
:10C87000D1795AEB010A80E8F807BDE8F007704764
:10C8800018EB040859EB05095AEB060A5BEB070B9A
:10C890005FF0000C4CF1000C18EB050859EB060991
:10C8A0005AEB070A5BEB070B50EB0C005FF0000C38
:10C8B00051EB0C0152EB0C0263414CF1000CB8EB54
:10C8C000070879F100097AF1000A7BEB040BA84113
:10C8D000B141A241B3416CF1000CBBEB050BB0417F
:10C8E000B941AA41BB416CF1000C6FEAEC74B8EBA2
:10C8F000040879EB04097AEB040A7BF1000B70F170
:10C90000000071F1000172EBD472A3416CF1000CD4
:10C9100018EBEC7859EBEC795AEBEC7A5BF1000B05
:10C9200050F1000451F1000552EBDC7653EBEC774B
:10C930004CF1000C18EBEC7059EBEC715AEBEC720B
:10C940005BF1000354F1000455F1000556EBDC7671
:10C9500057EBEC77704700BF2DE9F14F87B0FFF739
:10C960009FFDDDF81080DDF81490DDF818A0FFF7CA
:10C9700087FFBDE8000FFFF783FF03B05DF8048B6E
:10C9800088E8FF00BDE8F08F2DE9F14F87B0FFF791
:10C9900043FEDDF81080DDF81490DDF818A0FFF7F5
:10C9A0006FFFBDE8000FFFF76BFF03B05DF8048B6E
:10C9B00088E8FF00BDE8F08F1FB5144C207A8DF891
:10C9C0000100E0798DF80000A079ADF804006079ED
:10C9D000ADF80200684606F04DF808B1A72110E056
:10C9E000E068029002A806F05BF808B1AB2108E00D
:10C9F00007480068039003A80FF078F9002803D0D7
:10CA0000AF21032000F0DCF81FBD0000980D0020CE
:10CA1000C8CC000010B528B11422044910F0D9F890
:10CA2000002010BD6FF0150010BD0000ECCC000020
:10CA300070B56FF02C03B8BB1E4C607808B198112C
:10CA400070BD01B36FF01505AAB11B48891E0629F8
:10CA50002BD2DFE801F0030616192A1C1178417069
:10CA600017E0917839B1D17829B111781B2902D317
:10CA700051781B2901D2284670BD1168C0F80510F5
:10CA800007E01168C16004E01178817001E011884D
:10CA900041820122084900200BF0EAFDB0F5803FF9
:10CAA00005DB6FF00B0070BDFFE71846FBE70121C7
:10CAB000A170F8E728000020980D002010B5074C61
:10CAC000607820B106F0CAFA20780BF0A1FB00F0E4
:10CAD00087FD00F05FFE0020607010BD2800002080
:10CAE00070B50C46050002D00CB1600702D06FF0A3
:10CAF000150070BD00F020F9A8B128460BF04EFBE0
:10CB00000A4D00220A49287020460BF0B1FD0FF0B3
:10CB100007FD0021287806F08BFAFFF74DFF012072
:10CB20006870002070BD4FF0FF3070BD28000020FD
:10CB3000980D002030B589B004000CD00BF0D4FA69
:10CB40004FF0FF3520B10BF067F9B0F5FA7F05D94A
:10CB5000284609B030BD6FF01500FAE7134D1448B0
:10CB60006C6000F00BFA00206870A870014620226B
:10CB7000684610F0A8F820220E49684610F029F8FF
:10CB8000202269460C4810F024F8EFF3108472B6A6
:10CB900000F034FD094800F009FE18B1C52103205A
:10CBA00000F00EF804B962B60020D2E72800002099
:10CBB000B9C90000CCCC0000980D002065CD000064
:10CBC0000EB572B6154A5568DDB1002203466E46B1
:10CBD0000A2403E0B0FBF4F0521CD2B20028F9D1D1
:10CBE000B0540AE0D8B2B0FBF4F7B3FBF4F304FBA3
:10CBF0001700521ED2B23030B054002AF2D1304663
:10CC0000A847BFF34F8F06480168064A01F4E06168
:10CC100011430160BFF34F8F00BFFDE728000020E4
:10CC20000CED00E00400FA05064810B58178407864
:10CC3000014302D04FF0FF3010BD06F01FFA002074
:10CC400010BD000028000020064810B5817840780B
:10CC5000014302D04FF0FF3010BD05F06DFF002002
:10CC600010BD000028000020064810B581784078EB
:10CC7000014302D04FF0FF3010BD0FF0D6F9002075
:10CC800010BD000028000020064810B581784078CB
:10CC9000014302D04FF0FF3010BD06F001FA002032
:10CCA00010BD000028000020064810B581784078AB
:10CCB000014302D04FF0FF3010BD0FF0C6F9002045
:10CCC00010BD00002800002001000000000101004C
:10CCD000001B1B03020000004C1D000000001F0091
:10CCE000000000000000000000000000D80C2D2F04
:10CCF00036AEE25C8026804C3F4D16535096C7738B
:10CD0000054A10B5526812B1BDE810401047922193
:10CD10000420FFF755FF0000B80D0020054A10B5AC
:10CD2000926812B1BDE81040104798210420FFF727
:10CD300047FF0000B80D00200548016829B141688F
:10CD400019B1806808B101207047002070470000C9
:10CD5000B80D002002490DC881E80D000020704781
:10CD6000B80D0020F8B5124C0026256811E0009897
:10CD7000022802D003280CD106E0206810B1002060
:10CD8000266005E028210CE0206868B101202660BB
:10CD9000A847684600F0D0FC0028E8D0052805D058
:10CDA00035210420FFF70CFF2D21FAE7F8BD000024
:10CDB000300000202DE9FC41254E0546001D06F1FE
:10CDC00044073060387858B1BA783C46791C284618
:10CDD000921C0FF0FEFE002020700420BDE8FC81B4
:10CDE0001B4801F07FFE0446022804D0042C07D023
:10CDF000082C27D02AE0164928460BF0D9FC25E05C
:10CE00003078082804D105213E200BF0A3FC60B146
:10CE10000F4928460BF031FD0028D3D0A978287897
:10CE20000BF098FC0028CDD010E0B088ADF80000E1
:10CE300001A968460CF00CF80028C3D0A7210820EF
:10CE4000FFF7BEFE024928460BF0E0FC2046C5E78E
:10CE5000C40D002070B50A7882703AB3012A25D833
:10CE60001323037000230AE001EB430400EB4305A6
:10CE7000A678EE706488240A5B1C2C71DBB29342A6
:10CE8000F2D300230BE000BF01EB430500EB4304AA
:10CE90002E796671AD882D0A5B1CA571DBB29342B9
:10CEA000F2D3012101EB8200C0B270BD002070BD41
:10CEB000402803D2401EC1B2054805E0FF2805D036
:10CEC0004038C1B2024808300BF0B9BE01207047AB
:10CED0003C000020401EC1B201480BF0B0BE000073
:10CEE0004C00002010B5074A0168064B916140686C
:10CEF000D0611C681832A1431160596888435060A2
:10CF000010BD000034000020064A016891604068AE
:10CF1000D060083241F48C2111600349084350600D
:10CF20007047000034000020F80740020249026800
:10CF30000A614068486170473400002007484FF09C
:10CF4000FF3100220160C90C416000F108011F207F
:10CF50000A604A600831C1E9000270473C000020C5
:10CF600010B5FFF7EBFF0EF0D9FF0446024800684A
:10CF700000B18047204610BD5400002001490860E0
:10CF800070470000540000200221018041800021F0
:10CF90000171D821417142F60C51C1800149816073
:10CFA000002070472F36AEE210B5022804D340F2BD
:10CFB00003211720FFF704FE0149085C10BD0000A3
:10CFC0000C0F0020F8B5050000950DD0002608785C
:10CFD00049780446A14200D90C46AA0706D04FF46E
:10CFE000E5711720FFF7ECFD0126F0E7124F3870CE
:10CFF00079703146684600F0D3F800210B4600985E
:10D00000C01C20F00300009066B907EB8102D060DD
:10D01000002005E0D2F80CC04CF82030401CC0B213
:10D02000A042F7D30098491C00EB8400C9B20090DD
:10D030000229E4D3401BF8BD0C0F002070B5044654
:10D04000857900F0E9F80C4AE17902EB85020EE0FF
:10D05000D36853F8213043B1481CE071A180D068F7
:10D0600050F821002060002070BD491CC9B28142E7
:10D07000EED3E171052070BD0C0F0020F0B421B19A
:10D08000012902D0F0BC002070470F4A00252B4632
:10D090004FF6FF7402EB8106575C0AE05A19D6F886
:10D0A0000CC092B25CF822C0BCF1000F04D05B1C33
:10D0B0009BB29F42F2D8224602801046A242E1D0A3
:10D0C000F0BC00F035B800000C0F00202DE9F04155
:10D0D0000646A0F57F400C4643F20207FF3820D0F9
:10D0E000022C02D30720BDE8F081304600F048F85A
:10D0F000050016D00C48294650F8242030469047A9
:10D100000A48002100EB8407F86840F82610204602
:10D1100000F078F80246294678680CF027F90020DC
:10D12000E1E73846DFE7000030D200000C0F0020B6
:10D1300070B50E4605460CF053F958B10F4800EB98
:10D140008604E06850F8250038B14FF4C571172007
:10D15000FFF736FD40F28911F9E7606800280BD02F
:10D16000304600F04FF8014660680CF0A7F8002840
:10D1700002D0E16841F8250070BD00000C0F0020CE
:10D1800070B50C4605460CF02BF9002805D0034875
:10D1900000EB8400C06850F8250070BD0C0F002023
:10D1A0002DE9F843164E8846054600242868C01C21
:10D1B00020F003002860204600F024F8315D484349
:10D1C000B8F1000F01D0002200E02A680146009269
:10D1D00032B100274FEA0D000CF0A1F81FB106E0B4
:10D1E00001270020F8E706EB8401009A4A602968CD
:10D1F000641C0844E4B22860022CD7D3BDE8F8834D
:10D200000C0F0020034931F810004FF6FC71C01CD0
:10D21000084070472CD200000349087849788842BA
:10D2200000D20846704700000C0F0020F8021801D9
:10D23000BFB0010069A601002DE9FF4F244C06464E
:10D2400081B020689A46934658B1017AB14203D919
:10D25000406850F8260040B143F2020005B0BDE836
:10D26000F08FA5211820FFF7ABFC194602980CF0AF
:10D27000DAF8804658460E990CF0CBF8054608EBD4
:10D280000500001D87B22068A146394600680CF0F1
:10D2900015F804001AD0678025802946201D0E9DB0
:10D2A00007465A46092300950BF082FF2088414625
:10D2B00038440A23029ACDF800A00BF079FFD9F880
:10D2C0000000406840F826400020C7E70420C5E77A
:10D2D0005800002070B5144C23688BB1197A814234
:10D2E00012D95A6852F8201071B1002542F8205026
:10D2F0004A8818680CF03AF8216800200A7A0CE095
:10D30000C6211820FFF75CFC43F2020070BD4B6899
:10D3100053F8203033B9401CC0B28242F7D80868B5
:10D320000CF019F8002070BD580000202DE9F041E4
:10D330000D46040090464FF0000606D00027A007D7
:10D3400005D086211820FFF73BFC0127F7E7CDB178
:10D35000114600200BF0E3FF0C3000EB85068FB97F
:10D360000A4F04F10C00AA003C602572606000EBDB
:10D3700085002060002160680FF0A5FC41463868F8
:10D380000BF0CDFF3046BDE8F081000058000020D2
:10D3900070B5084D286800280AD0002404E0204613
:10D3A000FFF798FF641CE4B22868007AA042F6D820
:10D3B00070BD000058000020094910B502460968F8
:10D3C000002049B10B7A934205D9496851F82210DF
:10D3D000002900D0081D10BDEC211820FFF7F0FB3C
:10D3E000580000200A4910B502460968002059B1CA
:10D3F0000B7A934207D9496851F82210002902D0CC
:10D4000031F8040B084410BDFA211820FFF7D8FBAF
:10D410005800002070B51E4B456804460022A1B19B
:10D4200001206070588881085FF0000004EB400321
:10D4300004EB80061A83198400FB015373602318E0
:10D44000401C1A750428F1D370BD62705FF00000B3
:10D4500004EB40010A830A8404EB80014A6021182E
:10D46000401C0A750428F3D35888B0F5FF7F01D219
:10D47000460800E0FF260CF04AF865602084291871
:10D48000A1606684E560A0842161E68470BD00002F
:10D490005C0000202DE9F04158B100251144244ED4
:10D4A000CCB200273470810705D04E210920FFF748
:10D4B00087FB0125F2E71F2B04D84FF6FF7101EA25
:10D4C000830109E05900FF2B0CD903F1FF02B2EBF5
:10D4D000430F00D2114689B24FF6FC72C91C1140AD
:10D4E00035B107E07C22B2EB430FF4D37C21F2E7A5
:10D4F0007060718004EB840207EBC203002276683F
:10D500004FF0010C0DE04DB902EB820700EB030E6A
:10D5100006F837C006EBC707C7F804E0521C0B44F7
:10D52000D2B2A242EFD3DB1D23F00700BDE8F081A9
:10D530005C00002070B5104A00205168127814E099
:10D5400000EB800311F833306BB100EB800011EB7E
:10D55000C0040CD00025A57001212046FFF75AFF1A
:10D560002570204670BD401CC0B29042E8D3A9216E
:10D570000920FFF725FB00005C000020044810B5DF
:10D58000408884080BF0C3FF844200D3204610BDBE
:10D590005C00002030B50D4901204860821EC1F8B2
:10D5A00008230B4988600023C1F80032C1F8082322
:10D5B000084C2360251D28608860C1F8082323607B
:10D5C000286006490448086030BD000000E00040C3
:10D5D00000F0004000F500400000F63F08F5014073
:10D5E00010B5FFF7D7FF0CF069F803490148086050
:10D5F00010BD00000000F63F08F5014010B5FFF730
:10D60000C9FF0CF05BF800F087F805490348086093
:10D6100000F0B8F8BDE8104000F0DCB80000F63FBC
:10D6200008F501402DE9F84F824638480FF0EFF930
:10D63000DFF8D8B028B101260BF10100FF210170FD
:10D6400000E000264FF48075314C4FF000082F1D8C
:10D6500001216160C4F80081C4F80481C4F804A504
:10D660002160DFF8B0901CE0D9F80000C00618D5A2
:10D670000E200CF032F8EFF31080009072B6032108
:10D680002046C4F8041329460CF034F830B9394662
:10D6900020460CF02FF808B90FF050FA009800B9A6
:10D6A00062B6294620460CF025F828B939462046AE
:10D6B0000CF020F80028D7D0394620460CF01AF894
:10D6C0000028C5D106BB9BF801108DF80010009909
:10D6D00000919DF8001009B1012500E000250BF133
:10D6E000010080F800800320C4F80803C4F8048116
:10D6F000C4F800810E200BF0F0FF04480FF09EF9F3
:10D7000015B11120BDE8F88F0020FBE76003002071
:10D7100000E0004010ED00E010B506480FF08AF977
:10D7200018B127211D20FFF74BFA02480021417054
:10D7300010BD00006003002070B511490A68EAB10D
:10D7400000231D4601244A68521C4A60092A00D35E
:10D750004D600E7904FA06F20E6816420BD0EFF314
:10D76000108372B60C6894430C6003B962B64968C2
:10D770000160002070BD5B1C092BE4D3052070BD47
:10D7800064000020024800210160416070470000F1
:10D790006400002010B5044C2078FF2803D00AF064
:10D7A00037FDFF20207010BD0000002010B5084C90
:10D7B000617809B10F2010BD0AF0F0FC2070FF283D
:10D7C00001D0002010BD73211F20FFF7F9F90000E0
:10D7D0000000002001490020487070470000002030
:10D7E0000648074A818C5288914204D190F8220061
:10D7F00008B100207047012070470000301400205D
:10D800004C03002001494880704700004C03002071
:10D810000848094A818C5288914209D14FF6FF711C
:10D82000818410F8221F19B1002101700120704776
:10D8300000207047301400204C030020074810F8E7
:10D84000221F012907D001210170054803490088E2
:10D8500088840120704700207047000030140020A9
:10D860004C0300200649074B8A8C5B889A4205D1FD
:10D8700091F8222012B1016001207047002070470A
:10D88000301400204C03002009498A8CA2F57F4304
:10D89000FF3B02D00021016007E091F822200449FB
:10D8A000012A02D00160012070470020704700006B
:10D8B0003014002001490880704700004C0300200C
:10D8C0000549002081F822004FF6FF708884034943
:10D8D0000880488070470000301400204C0300206E
:10D8E00005498A8C824205D1002081F822004FF63A
:10D8F000FF70888470470000301400200A4A10B17D
:10D90000012807D00EE0507860B1D2F8020008601C
:10D91000D08804E0107828B19068086090898880E9
:10D92000012070470020704762030020084A01234D
:10D9300038B1012804D113700868906088889081FC
:10D94000704753700868C2F802008888D08070471A
:10D9500062030020064910B1012802D005E0487892
:10D9600000E0087808B101207047002070470000EF
:10D97000620300200149087770470000720D002003
:10D9800001488078704700006C0000200148C07892
:10D99000704700006C00002070B50C46054600F092
:10D9A0001FF918B1D0212720FFF70AF903480121F8
:10D9B0000CF0CAFA0248C0E90B5470BD500D0020AB
:10D9C0006C00002001490120487170476C00002064
:10D9D0002DE9F84F5B4D0A9C2E78002E6BD1002A62
:10D9E00069D0002B67D0002C65D005F11406C5E97D
:10D9F0000F0186E81C0000276F712F71AF706F70E8
:10DA0000EF70AF81EF8100F03DF9064600F034F988
:10DA1000044605F0A7FF05F0FFFC94F96E0006F040
:10DA200025F8E06906F008F9606906F0FBF896F859
:10DA3000330006F031F905F13C00406890F81A0215
:10DA400008B105F00FFF94F86B10012005F04EFEB1
:10DA5000002870D03C4805F0B5FE2088FFF7C2FCD6
:10DA600068632088FFF7A8FC06F18802A86392E8A3
:10DA70000C11DFF8D89089E80C11D6F89820C9F875
:10DA80001920D6F89C10C9F81D1000F033F9014692
:10DA9000208FBA460BF0B5FFA18E814200D2084616
:10DAA000A871A84694F86B10E08F96F82370A58FA4
:10DAB000082904D102E040F2451140E004210BF0B6
:10DAC000A0FF0FB9001D80B2854200D22846C5B222
:10DAD00088F8075088F8085096F82300D04690B18F
:10DAE000012789F81870D6E92012C9E9041294F8C0
:10DAF0006B000BF08BFE03462A4614493846CDF8DE
:10DB0000008005F0F5FB012000F054FB1048006890
:10DB1000032812D00B2810D00C480E2200214A30C6
:10DB20000FF0D1F80948B18A4A304180218801803C
:10DB300096F833100171BDE8F88F40F202212720DA
:10DB4000FFF73EF86C000020B8E30000280D00202D
:10DB5000501500402DE9FC418846074600F092F838
:10DB60001A4C0546B807616A4E7816D5A06A30B3DC
:10DB70006289D21C0FF02DF8A06A6062694601AA82
:10DB8000A06B0BF092FA00980BF045FAC8F8000071
:10DB900031460122A06B0BF0F5F9F8070DD0D5E95D
:10DBA00020011835401C41F10001C5E91A0115F8A2
:10DBB0001809012808D001202876BDE8FC8140F230
:10DBC00066412720FEF7FCFF0020F5E76C000020EF
:10DBD0000248C089C0F38020704700006C0000201C
:10DBE0000448007808B10C207047034900200877EA
:10DBF000704700006C000020720D00200C4810B52A
:10DC0000017849B100F13C010078022808D040F2C7
:10DC10001E212720FEF7D4FFBDE8104000F0D8B940
:10DC20004868D0F83002BDE8104005F0D3BD0000D0
:10DC30006C000020F8B5002605464E701D20094FE7
:10DC40000C4608702E720E223946201D0EF0C1FFC0
:10DC5000287A8DF80000009800909DF800000028B8
:10DC6000F0D1F8BD800D0020024A938903439381CF
:10DC7000526910476C00002001484068704700005E
:10DC8000A80000200148406880307047A8000020AC
:10DC9000014A0021526910476C00002070B505460A
:10DCA000012918D8124CA1698847A0B1207990B9F0
:10DCB000E5B904F110000178C80605D4E06A0078DF
:10DCC000C00601D4012000E00020A26A2AB96289BE
:10DCD0001AB1C90601D4012070BDA1898A0703D5F4
:10DCE000226AD278022A01D00843F4D1002070BD04
:10DCF0006C00002010B5FFF7BFFF0446FFF7C2FF1E
:10DD00000246417F1648252910D026290ED0927F41
:10DD1000252A0BD020290DD021290BD0232A0FD062
:10DD200094F86A00042800D1082010BD406890F8DB
:10DD3000CE120EE0232A03D0406890F83E0105E0A1
:10DD4000416891F83E0191F8631008400BF054FDD2
:10DD5000014694F86A00BDE810400BF065BD000074
:10DD6000A80000202DE9FF5F8B468146FFF78AFF60
:10DD70000026664C07468DF80860039601962078C9
:10DD80003546022804D040F2EA412720FEF718FF6A
:10DD9000A07B400606D44020FFF77AFFE08940F0E0
:10DDA0004000E08197F82300B9F1000F3AD080B12C
:10DDB00005F06CFB05F046FB58B9606A417841B14B
:10DDC0000078397EC0F3C000884202D10120607023
:10DDD00097E0606A4178618121B1A06B0BF03BFA5A
:10DDE000A06200E0A562E08940F48070E081606A92
:10DDF000F97D0078C0F38000884207D003A800F0C6
:10DE00008BF9E08940F48060E08100E00126606ADF
:10DE1000397E0078C0F3C00088420DD102A800F01E
:10DE200031F909E008B105F02BFBA078401CA07087
:10DE3000E08940F40070E081DFF8D0A097F822007C
:10DE40000AF13C0A90B1FFF717FF31490D76D7E987
:10DE50001E23C1E9042390F86A000BF0D7FC0346A7
:10DE6000FB222B492846009505F042FA4FF00008A6
:10DE7000BBF1000F04D1A1780120FFF70FFF20B103
:10DE800005F0BCFE4FF0010802E0002000F0D0F9E0
:10DE90009DF8080018B101A90220FFF75BFE1C489D
:10DEA000BA8A4A303EB11AB9C2880AB9028912B197
:10DEB0004289521C4281B9F1000F08D0C188491C27
:10DEC000C1801248A5703C3001F060F902E0018980
:10DED000491C0181039840B10BF09DF8DAF8041059
:10DEE000401C05720E220CF0ADF8019830B1DAF842
:10DEF000041005722A2201980CF0A4F8B8F1000F62
:10DF000001D000F065F8BDE8FF9F00006C00002024
:10DF1000280D00202DE9F84388468146FFF7B2FE20
:10DF2000294D04462878012804D040F27541272065
:10DF3000FEF746FE207C0027012628B12774002129
:10DF40000420FFF791FEA674296A0878C043800771
:10DF500009D1A07D88BB0220FFF786FE286A0078E1
:10DF6000C043800729D0286A407810B10220A075EC
:10DF700000E0A67594F8230098B1FFF77DFE1349E1
:10DF80002D7A0E76D4E92023C1E9042390F86B00A2
:10DF90000BF03CFC03462A460C493046009705F03E
:10DFA000A7F938EA090004D000210846FFF776FEF9
:10DFB00028B1BDE8F84300F00BB80320D7E7BDE86F
:10DFC000F843002000F0F6B86C000020280D002077
:10DFD00010B505F001FB05F01FFA0D4CE089FFF7C5
:10DFE00057FE0C48007F58B10A490E2201F10E007D
:10DFF0000EF0EFFD0748242207491D300CF036F8DB
:10E00000E2692179607890470020207010BD0000FF
:10E010006C000020720D002035DC0000084810B5AF
:10E020000078022804D040F24D212720FEF7C8FDD9
:10E03000044901200873BDE81040FFF7C9BF000084
:10E040006C000020720D002030B404460C48007AA9
:10E050000BB1001DC0B23AB9FF2805D194F86B206E
:10E0600094F86A309A4209D021B194F86B1030BC10
:10E0700005F0E8BDFF2094F86A10F8E730BC70475F
:10E080006C0000202DE9F0410746FFF7FBFD214C15
:10E0900005460126616A087800F0030001280CD0CB
:10E0A00002280AD003281BD12E74E08940F40060B6
:10E0B000E0810120FFF7D8FD12E0487880B1E189C6
:10E0C00041F40061E181A16A002918D0FB2818D829
:10E0D000607920B1BDE8F0412020FFF7D9BD3E7046
:10E0E000287E012812D02E76606A4078002806D05B
:10E0F000F5E92001401C41F10001C5E90001BDE83E
:10E10000F081207940F010002071F8E70020287697
:10E11000EAE700006C00002070B50546FFF7B2FD8D
:10E120000446807D00282DD002280CD11B482946AA
:10E13000406B0AF0FFFE30B3D4E91E01401C41F1F0
:10E140000001C4E91E010025A575A07C20B1A574BD
:10E1500000211020FFF788FD607C70B16574FFF727
:10E1600057FB98B100210820FFF77EFDD4E91E017E
:10E17000401C41F10001C4E91E01E07D01280AD0E4
:10E180000120E07570BD40F2E33101E040F2FA3168
:10E190002720FEF715FDE57570BD00006C0000201E
:10E1A00003480078002801D0FFF712BF7047000035
:10E1B0006C0000202DE9F0410646FFF75DFD80462A
:10E1C000FFF760FD184C05463246E06A606295F83C
:10E1D000233001214046FFF737FF95F82300002741
:10E1E00070B1206B05F064FC104801210176D5E97F
:10E1F0002012C0E90412216B606A05F0CBF804E03C
:10E20000606A05F055FC05F007F916B9384605F0C7
:10E2100005FB002198F86A20084605F0D1FC022091
:10E220002070BDE8F08100006C000020280D002067
:10E230002DE9FC470446FFF725FD0546FFF71CFDC9
:10E2400000278DF800700646DFF8649195F82330BA
:10E2500022463946FFF7F8FEA87D4FF00108A9F1E4
:10E26000200440B1012820D002282FD003283BD021
:10E2700040F2FF2157E0A0795021ADF80400885307
:10E280004846FFF7EFFA30B18020216AFFF7ECFC37
:10E2900085F811802CE06A4601A9606B0BF0CEFA7C
:10E2A000206210B195F85B1011B1424820621FE066
:10E2B0009DF8001021B90780877001210BF044FE02
:10E2C000BDF80410206A0BF0C7FD11E0B6F850004D
:10E2D000ADF804006A4601A9606B0BF0AFFA20624A
:10E2E00030B940F2E9211EE04846FFF7BBFAC0B161
:10E2F000206A0823017801F0F7010170EA7D03EA42
:10E30000C202114301F0FB0101702A7E042303EADB
:10E310008202114301F0EF010170C943890705D062
:10E3200007E040F2F2212720FEF74AFCC0780228DD
:10E330000FD0606B0AF0FCFE08B101210AE0206AF0
:10E340000078C043800704D0FFF74AFA80F001014B
:10E3500000E00021206A027842EA0111017095F87C
:10E36000221081B1417871B1206B05F0A1FB1148F9
:10E3700028380776D5E91E12C0E90412216A206BFD
:10E3800005F008F803E005F093FB05F045F896F872
:10E390006B200121002005F013FC84F80380216A22
:10E3A0000A8822828978A17484F80080BDE8FC87FD
:10E3B0008C000020500D00201DE0000065DD0000F5
:10E3C00015DF0000A1E10000004870472916002079
:10E3D00004498A78824203D9084490F8430170477F
:10E3E000002070475614002004498A78824203D9DD
:10E3F00001EB001083307047002070475614002056
:10E40000054A01EB410102EB41010268C1F80B2111
:10E410008088A1F80F0170475614002004498A78BB
:10E42000824203D901EB0010C01C704700207047E6
:10E430005614002010B540F2D312002108480EF007
:10E4400042FC0822FF2107480EF03DFC0548002150
:10E45000001F017041704FF46171418010BD0000D8
:10E4600056140020540300200B4B10B59C788442B6
:10E470000FD9184490F8030103EBC00090F8533112
:10E480000B70D0F854111160B0F858019080012041
:10E4900010BD002010BD00005614002007498A78E6
:10E4A000824209D9084490F8030101EBC00090F8BA
:10E4B0005A0100F0010070470020704756140020F8
:10E4C00001484088704700005003002005498A78C1
:10E4D000824203D9084490F83B0108B100207047FC
:10E4E000012070475614002070B50D46064600F016
:10E4F000C1F8104C102807D004EBC00191F85A1154
:10E50000C90701D0012070BD6178082910D21028F8
:10E5100008D004EBC000012180F85A116078401C3B
:10E520006070EFE701222946304600F087F8F5E7F2
:10E53000002070BD5614002070B50B4D2878401E89
:10E5400044B20AE005EBC40090F85A01C00702D0BB
:10E55000E0B200F0EDF8641E64B2002CF2DA034978
:10E560000020487070BD00005614002050030020A9
:10E570002DE9F04100242546184E29E006EBC50799
:10E5800097F85A01C00721D0284600F043F8034607
:10E59000FFF744FF01460020102B09D0F21892F833
:10E5A0003BC1BCF1010F02D092F84B2102B1012016
:10E5B000401E01420AD10A4807F5AA7103552046B8
:10E5C000641C97F85321E4B205F020FC6D1CEDB2F9
:10E5D0003078A842D2D8BDE8F0810000561400205F
:10E5E000540300200246094810B500780B4658B184
:10E5F0000748817841B10BB1C01C01E00448833069
:10E6000004F0D0FD012010BD002010BD50030020FB
:10E6100056140020084910B5034600208A7806E009
:10E620000C1894F803419C4204D0401CC0B28242B2
:10E63000F6D8102010BD00005614002070B50C4B09
:10E6400004461878451C1D70102803D34621282045
:10E65000FEF7B6FA03EBC0030D68C3F8545189887E
:10E66000A3F8581183F8534183F85A2170BD000074
:10E6700056140020F0B51A4C0346002025782AE0F5
:10E6800004EBC0020F7892F854C192F8536187EA04
:10E690000C075E403E444F7892F855C187EA0C075C
:10E6A0003E448F7892F856C187EA0C073E44CF78F3
:10E6B00092F857C187EA0C073E440F7992F858C187
:10E6C00092F8592187EA0C073E444F795740F742A8
:10E6D00004D0401CC0B28542D2D81020F0BD00004A
:10E6E0005614002070B50546FFF794FF10281CD182
:10E6F0000E4C2078401EC0B22070A84215D004EB0A
:10E70000C00204EBC50102F58070D2F85321C1F8B4
:10E710005321D0F85700C1F857012078FFF77AFF4E
:10E72000102802D0204480F8035170BD56140020F8
:10E7300005494A78521E4A7001EBC001002281F857
:10E740005A21FFF7CFBF0000561400202DE9F047F3
:10E75000044600F180054FF0010971B104F1A607EC
:10E760007E1E012925D002294AD003291FD139460E
:10E770003046BDE8F0470BF094BA4FF43E720021EA
:10E780000EF0A1FA85F825902248E8660720286750
:10E7900014F8EC0F20F004002070FE2085F8A6008D
:10E7A0007F2068761C48A8600020C5E90000BDE80D
:10E7B000F0874FF00008A4F8368284F82B82216994
:10E7C00016480A460844B0FBF1F0C4F8C40040F60D
:10E7D000B830A4F8C800638B284600F021F8394609
:10E7E00030460BF05EFA0EF085F918B1606900F062
:10E7F00053FB10B184F81A82D9E784F81A92D6E74D
:10E800000169B4F8DA32D4F8D4222846BDE8F047DA
:10E8100000F006B82F49043400E0FCFF7FC3C901B3
:10E8200010B50024A0F84C4030F8504F4C43B4FBD6
:10E83000F2F420F8104940F27124634302EB031311
:10E840005B1EB3FBF2F3C381094BB3FBF2F35B1C1A
:10E8500083820389634302EB03135B1EB3FBF2F372
:10E86000436003684B43B3FBF2F1016010BD00004D
:10E87000005A6202024991F900100BF0C3B900007E
:10E880007003002008B57F208DF80000684605F071
:10E89000BDF940B105484078404241B29DF90000C1
:10E8A0000BF0B0F908BD9DF9000008BD7003002011
:10E8B00070B590F8322090F83130012403FB01212B
:10E8C0002522B1FBF2F302FB131100EBD10280F819
:10E8D000321001F0070392F8262004FA03F31A42DB
:10E8E00004D000BF80F83310002070BD90F83020B5
:10E8F000B1FBF2F302FB1311491CC9B20023C51886
:10E9000095F82B208A4212D395F82650002200BF9A
:10E9100004FA02F6354201D0491EC9B221B1521C97
:10E92000D2B2082AF4D304E002EBC301DAE7891A71
:10E93000C9B25B1CDBB2052BE1D31F2070BD000008
:10E9400070B5491C0023C9B20124C518AA798A42AE
:10E9500012D395F80150002204FA02F6354201D094
:10E96000491EC9B221B1521CD2B2082AF4D305E023
:10E9700002EBC300C0B270BD891AC9B25B1CDBB226
:10E98000052BE2D39D214620FEF71AF9417841B1CB
:10E99000C0782B2803D2044A105C884201D10120A0
:10E9A000704700207047000010CE010010B5012212
:10E9B000C1702B2902D2064A525C06E0FF2904D01E
:10E9C00040F275412A20FEF7FBF8427010BD0000AE
:10E9D00010CE01000449897C490700D408B1002009
:10E9E0007047012070470000200F00200348807C02
:10E9F000800701D40120704700207047200F0020BD
:10EA00000348807CC00701D0002070470120704778
:10EA1000200F00202DE9FE438846994615460446FE
:10EA200069460AF04EFFE0BB019E002780367DB1AB
:10EA30002046FEF7D7FC04000ED029460AF04AFB18
:10EA400018B11B494988A94208D20020BDE8FE83BD
:10EA5000012086F8240024E0672125E0014602AA6F
:10EA600020460AF030FB02980780877096F8241041
:10EA700009B14FF0020841460BF066FA02982A46A7
:10EA80004946C01C0EF0A5F8204629460AF0D9FADE
:10EA900048B168460BF0B3FA0198A0F8227286F8E4
:10EAA00024700120D2E77C212B20FEF789F800009A
:10EAB000200F0020094882B0007A8DF800000098ED
:10EAC00000909DF80000002805D102220449034867
:10EAD00002B00BF0B7BA02B070470000380F002048
:10EAE0008BA001002DE9F84FDFF89881DFF898A19D
:10EAF00083464FF001090026D8F80400007A8DF80B
:10EB00000000009800909DF800102A2906D19AF87C
:10EB1000131019B1BAF8140000287DD000278DF821
:10EB20000060684600F012F99DF800100029F8D145
:10EB3000002871D00446007A8DF8000000980090FB
:10EB40009DF80050A81E302867D2DFE800F0182793
:10EB500085218585276F696F6F6F2D6F852185856D
:10EB60006F6F21858585856F4585856F216F6F85E1
:10EB70006F2185854F55758585858585854F6268AB
:10EB800012B94FF4D27164E05946204690473CE0F8
:10EB90006268002AF8D140F2BB115AE06268002A8C
:10EBA000F2D140F24B2154E060685D4680B10488A8
:10EBB0002046FEF717FC68B16E700D222A70EC80BB
:10EBC000A5F80890314685F804900AF01AFB57E042
:10EBD000CE213EE0AE213CE0626822B1594620469B
:10EBE0009047012711E040F2632132E06268002A79
:10EBF000CAD140F26F212CE08BF8016016218BF80E
:10EC00000010D4F80910CBF804102672212D26D05C
:10EC1000142D27D0222D01E017E01DE029D02DE092
:10EC20006268002AB0D140F2812112E06268002AB5
:10EC3000AAD140F296210CE01448026822B1606823
:10EC400028B10088594690470220BDE8F88F40F26D
:10EC50009F211020FDF7B4FF40F2BD21F9E7FFF737
:10EC6000C5FE08E09BF80E0000F00100FFF7B2FEC1
:10EC700001E0FFF7C5FE00287FF43EAF002FFBD177
:10EC80000420E2E74C0F0020200F0020B0000020FD
:10EC90000149087000F0B0B8720300200249014831
:10ECA00008607047ADEC0000B000002038B50D00E2
:10ECB00014D0A88000216972FEF77EFB04460AF09A
:10ECC000E4F968B101466A4620460AF0FCF9E8809A
:10ECD00048B1FB280AD94FF4867132E0FC2130E0BC
:10ECE00040F205112DE04FF485712AE000980BF0F9
:10ECF000D7F8012804D0022802D04FF48E7120E00A
:10ED000028722868A8B10099EA88C91C0DF061FF33
:10ED100020460AF082F978B1204600210AF071FA03
:10ED200068B10948C17C002902D0818A491E8182CC
:10ED300038BD40F2231104E04FF4947101E040F239
:10ED40002D111020FDF73CFF200F002038B50246A2
:10ED5000114B002010705868017A8DF8001000994E
:10ED600000919DF800500124012D06D0EFF3108191
:10ED700072B605685D6011B102E0002038BD62B670
:10ED8000017A8DF80010009900919DF80030002B59
:10ED9000F4D1147038BD00004C0F002038B5D0B14C
:10EDA000416000F108010A70EFF3108372B6104C55
:10EDB0000460211F4A684AB1127A8DF80020009A37
:10EDC00000929DF80050012D00D10C600A6810607F
:10EDD00008602BB105E040F2E2211020FDF7F0FEC3
:10EDE00062B604480078BDE8384009F0F5B9000083
:10EDF000500F002072030020084810B50021416127
:10EE00008161C161016212220DF05DFF034814307F
:10EE100001210173011D4160016010BD380F002008
:10EE2000F0B450810C89134694818A89DA8148892B
:10EE30001882CD895D82CE8DAE4208D14D8D85423E
:10EE400005D10D8E954202D18A8DA24201D00122B8
:10EE500000E000221A754885588AC88598898885F7
:10EE6000D8890886F0BC1422014918460BF0FEB878
:10EE700049A201005081888A9081C88AD081088B7C
:10EE80001082488B134650822122024918460BF00B
:10EE9000D9B800007FA20100F0B56FF01F02010C8D
:10EEA00002EA90261F25A1F5AA4054380DD0A1F5FD
:10EEB000AA40553809D0A1F52850AA3805D0A1F5A7
:10EEC0002A40AA3801D0012000E000200022134689
:10EED0004FEA020482EA0107FF431F437F1C0FD061
:10EEE00006F00107520842EAC73205F001075B0845
:10EEF00076086D08641C43EAC733162CEAD3F0BDCC
:10EF00000020F0BD10B504480BF01DFA0248BDE822
:10EF1000104008300BF017BAB4000020014800F090
:10EF200009B80000B4000020014800F003B8000058
:10EF3000BC00002010B5D0E90021094B094C534317
:10EF40005443514081EAB21282EA41224FEAF14130
:10EF5000C0E9002143EAD46303EB8303184610BDE4
:10EF60006037EFC6BB79379E10B54068002290F835
:10EF70008C308030091DDB0701D0012010BD0C79D9
:10EF80000B6809490B4004F00701C3660167A0F84C
:10EF9000582090F85A10491C80F85A10C16841F066
:10EFA0000101C160002010BD2F49043710B5041DB8
:10EFB00004F0C8F8034A01F00701104020606160C6
:10EFC00010BD00002F4904372DE9F843037840684D
:10EFD0000F1D00F1800500F5A57406464FF00008EE
:10EFE0006A7F072128460AF096FCB0B13868154AB6
:10EFF0003979104001F00701E866296785F85680E5
:10F0000085F81D8094F8681040468DF8001000992E
:10F0100000919DF8001091B902E00120BDE8F8834D
:10F020003188A4F86A1084F869003968E166796863
:10F0300021670822044904F160000BF003F8002066
:10F04000ECE700002F490437B3A4010070B50D1D93
:10F05000446804F077F8064A104001F0070294F87B
:10F06000EC10014061F3070028606A6070BD000089
:10F070002F490437416882B001F5A57091F8B2219B
:10F080008DF80020009A00929DF80020002A0BD1F4
:10F090000988A0F86A101A2180F86910082203492B
:10F0A000603002B00AF0CEBF02B07047B3A40100D6
:10F0B00070B544680D46037894F89D20803400268E
:10F0C000082120460AF027FC20B9207B800701D5C3
:10F0D000012070BD94F85D00800719D428460AF01D
:10F0E0004DFF84F8670035F8050FA4F868006888BC
:10F0F000A4F86A0094F85D0040F0020084F85D0016
:10F10000C00709D00322114904F15E000AF0AEFFE6
:10F1100094F85D00C00710D1E068810703D54F2146
:10F120004020FDF74DFD40F00200E06094F85A00E9
:10F13000401C84F85A00A4F85860607F012802D16E
:10F14000667784F85660002070BD0000E1A40100DD
:10F15000074900F500600013097840B2494249B2FE
:10F16000084400F30700002800DC0020C0B270470C
:10F17000C4000020044A9268C2F580534B434243C6
:10F1800003EB223070470000C4000020F8B544684B
:10F19000064604F1800500F07FF894F82810012954
:10F1A0001AD1002818D0706890F852118DF800100C
:10F1B000009900919DF8001000F5A57000290BD171
:10F1C00021884181697E0173A97E4173BDE8F840C1
:10F1D0001F2202490AF036BFF8BD000083A50100D6
:10F1E00000F500610D4A10B500F500600913001329
:10F1F0004BB292F900404042002140B2A34202DAF1
:10F2000092F9021005E092F90140A34204DD92F95F
:10F210000310084400F30701084610BDC400002095
:10F220002DE9FC4100224A70A0F5FA750A70A0F59C
:10F23000BA7495F86B000CF0BFF90646A068FFF7AA
:10F24000CFFF070021D020460BF0A3F900281CD0E7
:10F25000288869460AF035FB18B189217A20FDF724
:10F26000AFFC761CF1B202233A4668460CF0C3F9B3
:10F2700000280AD1064807490079A0FB016507F07C
:10F280009DFD80196941C4E90001BDE8FC810000D1
:10F29000C400002040420F002DE9F0410746FFF76F
:10F2A000F1FA7C68054684F8990080347F283CD0C8
:10F2B00094F833007E68A0762946A068FFF75AFFCD
:10F2C000A0601B48407990B1786800F18008D0F8C0
:10F2D0008800FFF785FF50B140460BF05AF930B176
:10F2E00078683122134900F5FA700AF0BFFE94F9EC
:10F2F0001B000021281A00D5404296F8292082429E
:10F3000010DCFF2A0ED0207F401CC0B2207796F878
:10F310002A20904202D8E07E7F2803D10020E576A3
:10F32000207701210846BDE8F0810020FBE70000BE
:10F33000C400002021F2000070B50446007C00B338
:10F3400002281ED05FF0010004F1510184F8500042
:10F350000D46C0B1E07DF0B1D4F81100C4F8510001
:10F36000B4F81500A4F85500207C0BF03BF920768A
:10F370000820607694F8500029460BF01FF9A8B9D0
:10F380000EE00020E0E70020FEF7B8FA0028EBD1FD
:10F3900040F2B94101E040F2BD412D20FDF710FCE3
:10F3A00094F8500029460BF012F900B10120A07624
:10F3B000207E30B194F8570004F158010AF04DFA5C
:10F3C0006076FFF77DF80C49A0FB012304F14800AB
:10F3D0000BF08DFA002120460BF042FA002084F851
:10F3E0005E00A078400705D52046BDE870400021AA
:10F3F00000F0D0BD70BD000040420F0030B50C469B
:10F400008DB005460146242202A80DF0E2FB0BA8B0
:10F410000BF0CAFAA07A8DF8180020788DF8080051
:10F42000B4F80100ADF800009DF8000000F0010103
:10F43000C0F3400241EA4201C0F3800241EA820186
:10F44000C0F3C00241EAC201C0F3001241EA021156
:10F45000C0F3401241EA4211C0F3801041EA80102B
:10F46000ADF80A00207D012806D0022804D040F221
:10F47000EA210620FDF7A4FB8DF80C00617A0BA8A9
:10F480000BF079FA207D0121022802D1607D401C19
:10F49000C1B2A07E401CC2B20BA80BF033FABDF87B
:10F4A0000A00000701D5002020E00BA80BF03CFA71
:10F4B000BDF80A10282200F011FE40F2712100F27E
:10F4C000D920B0FBF1F04843D4F8021040F2712388
:10F4D0000A0A40F271214A43D4F80510090A594337
:10F4E000904201D8049204E0884201D8049000E0E0
:10F4F0000491A07C8DF81700207E012800D0002008
:10F500008DF81400686B0AF010F8686B0AF0B5F813
:10F51000242202A928460DF05CFB0B98A862BDF8D6
:10F520003000A885E07A68B102280BD05FF00100B6
:10F5300085F85700E068A865208AA5F85C000DB042
:10F54000002030BD0020F3E70A4A10B500211170F9
:10F55000094C606000F022F810B140F22D3104E057
:10F56000A068002804D14FF44C712D20FDF728FB32
:10F5700010BD00005C0F0020D000002002490148AF
:10F5800088607047C4000100D00000200249086074
:10F590008968096808470000D0000020084810B5B5
:10F5A000007810B10C24204610BD002418222146FA
:10F5B00003480DF088FB03F0E7FF03F00BFEF2E7D2
:10F5C0005C0F0020044910B50978012901D100F031
:10F5D000B5FB002010BD00005C0F0020024901486F
:10F5E0000860704769FE0000DC00002010B504468A
:10F5F0008078C0F3C00058B13C23FF222046E16967
:10F6000000F0C2FB1122044904F16C000AF01AFD5B
:10F61000012084F8690010BDF9A701002DE9F0412F
:10F620000F00044623D004F1280005460BF0A5F98D
:10F63000B0B9A078C0F3C00050B328460BF074F9FD
:10F64000064628460BF099F9301AC0B20BF0EAF9D9
:10F650000146354842681144416028460BF0ABF939
:10F6600028460BF06DF9014620460BF035F92F4D79
:10F6700094F85E600021686801800BF093F8608860
:10F68000132813D009DC102836D0122809D131E014
:10F690002046BDE8F04100F051BB15280FD01D28D1
:10F6A0000DD040F272612D20FDF78AFA00216868C2
:10F6B0000AF04FFB012168680BF074F820E001218B
:10F6C00068680AF046FB012168680BF06BF836B1F8
:10F6D00004F15F0168680AF057FB012106E004F1BC
:10F6E000580168680AF050FB94F8571068680AF0EF
:10F6F00051FB05E0062100E0022168680AF029FBC1
:10F70000204600F0BDFC60881D2807D0152805D0D4
:10F7100094F83C20A16B68680AF00BFB3946204640
:10F72000BDE8F04100F0F6B95C0F0020D0000020E9
:10F730002DE9F0412F4D80462878022805D0287801
:10F74000032802D040F62D512BE02B4C2668307B4D
:10F7500018B1FFF797F886F82E00D4F804C00027F8
:10F76000B8F1000F9CF8000000F00F0627D02168C8
:10F77000C00901F1510391F850200CF1090109F081
:10F78000D4FFE0B1394660680AF0C3FAB8B12A780C
:10F7900020683146022A07D02A78032A04D040F68E
:10F7A00006512D20FDF70CFAA2682B7852696FF0F4
:10F7B000070606EB8303D2589047064600E0012671
:10F7C000A87B18B103F0E0FE03F004FD002E0FD07B
:10F7D00020680BF03DF930B103F0FEFEA0688068B0
:10F7E000BDE8F04100472068BDE8F04100F0A6BA4E
:10F7F000BDE8F0815C0F0020D000002010B5032987
:10F8000002D005290AD102E000F092FB03E004498E
:10F81000096809B1884708B1002010BD012010BD5A
:10F82000DC000020094A0300106801D000F086BA0D
:10F83000002909D09168064A096912786FF00F0310
:10F8400003EB82028958084770470000D00000206F
:10F850005C0F002070B504464088102819D0104D68
:10F86000A87B20B103F0D6FC402003F09BFE0D489E
:10F87000406804F01DF9A078400704D400212279E3
:10F88000084604F09DF9002003F0C8FF022028700C
:10F8900070BD2046BDE870400121FFF7BFBE0000EB
:10F8A0005C0F0020D000002010B5124C206800F042
:10F8B00025F820680BF0CCF8002820680BD00E4902
:10F8C0000A78022A0BD00A78032A08D040F637417A
:10F8D0002D20FDF775F9BDE8104000F02FBAA268A1
:10F8E0000978D2686FF0070303EB81015158BDE836
:10F8F00010400847D00000205C0F002010B5017BAD
:10F9000021B10446FEF7BEFF84F82E000548807B37
:10F91000002805D003F038FEBDE8104003F05ABCC3
:10F9200010BD00005C0F00202DE9F0415D4D044644
:10F9300086B0287800284ED12078FF284BD04FF091
:10F940000008A5F80C80C5F8048085F8018085F8CA
:10F95000028084F86980544B544E0FCB8DE80F0021
:10F96000B06840680390684603F02CFF03F0FAFF8C
:10F9700004F07CFA03F008FE03F02CFC4C4804F081
:10F9800051F94C4804F058F904F1280007460BF0EF
:10F9900012F838460AF0D4FF014620460AF09CFFD0
:10F9A00094F90E0004F062F82179002003F09EFE25
:10F9B0000121A86098B104F13801606B09F024FEC0
:10F9C000074604F14001606B09F021FE4FB194F845
:10F9D000201051B905E00C2006B0BDE8F081297077
:10F9E0005EE020B194F8210008B1012700E0002773
:10F9F000A07E20B9207E10B9A078400723D5D4E995
:10FA000012106FF00042504070EA010106D007F07A
:10FA1000D5F9D4E91223801A994100D29FB1FEF79B
:10FA20004FFD2549A0FB012304F148000AF05FFFC8
:10FA3000012120460AF014FFA078400703D50121D8
:10FA4000204600F0A7FAFEF793FD7068C01C09F08D
:10FA5000F7FEA873A078C00722D0CDF81080FF2051
:10FA6000CDF81480E873E66906F10A0713E0049CF8
:10FA7000B44210D0727A607A3B4604F10A0109F070
:10FA800054FE40B1A078E873D4F803002861B4F8BC
:10FA90000700A88204E004A8FDF7D0FA0028E6D009
:10FAA000002099E75C0F0020A4000100D000002096
:10FAB000D6BE898E5555550040420F0010B50446FC
:10FAC000FFF732FF002808D104480078012803D04E
:10FAD00000212046FFF7A2FD002010BD5C0F002092
:10FAE0000A4810B50A490468087800280DD008783B
:10FAF000022802D00878032802D12046FFF7FEFE34
:10FB00002046BDE8104000F019B910BDD00000201B
:10FB10005C0F00202DE9F041044629480D4640685D
:10FB200003F0C6FF274E0420307055B360881028BC
:10FB300023D004F128008046B5680AF0F5FE074698
:10FB400040460AF01AFF381A401EC0B261882822C7
:10FB500000F0E4FA0544A078C0F3C00030B170684A
:10FB600005440AF063FF2844C4F8D80022792946E6
:10FB7000002003F0B3FF20B90CE02179002003F04E
:10FB80007BFD6088132811D007DC102815D01228BF
:10FB900007D10BE040F6A85105E0152806D01D2836
:10FBA00004D040F6BC512D20FDF70AF82279BDE8BB
:10FBB000F0410121002004F003B8BDE8F08100000D
:10FBC000D00000205C0F002038B5044690F8BC003F
:10FBD0000B468DF80000009800909DF8000000286A
:10FBE0003AD1207884F8BD00FF2B10D004F1BF0279
:10FBF000511E1846FEF738FC30B194F8BE0040F0B4
:10FC0000020084F8BE0011E041F2080121E013482F
:10FC100040680178C1F3801184F8BE10D0F8031059
:10FC2000C4F8BF10B0F80700A4F8C30094F92E0080
:10FC30007F280CD084F8C5007F2084F82E0004F1C2
:10FC4000B400BDE83840202205490AF0FBB940F66F
:10FC50006C612D20FCF7B4FF38BD0000D0000020FF
:10FC600049A801002DE9F04790460E4604460329B5
:10FC700004D094F8680008B1012000E0002081461B
:10FC800003F09CFC0546032E03D00127052E05D06A
:10FC900008E0A0780227C0F3400001E0A078C00788
:10FCA000002842D0B9F1000F3ED12248807B40B1FC
:10FCB00009F0C9FD88F80000FF2802D0FEF7EEFB2E
:10FCC00005431D4E94F8572004F15803716811F84C
:10FCD000030BC0F3801009F028FD98F80010FF29ED
:10FCE00004D090B9607E88420FD008E038B17168C6
:10FCF00011F8030BC0F380100AF05DFD28B100205D
:10FD0000A178490703D590B90EE00120F8E775B94D
:10FD1000E07B08B1B84207D1716811F8030BC0F35A
:10FD200080100AF048FD10B10020BDE8F0870120E6
:10FD3000FBE700005C0F0020D000002070B50446F7
:10FD4000008E104D401C2086A87B002620B103F0B9
:10FD50001BFC03F03FFAAE732E7094F8690008B1F3
:10FD600001210AE0607B38B1218E884204D801214C
:10FD700020460AF07FFE70BD00212046BDE870409D
:10FD80000AF078BE5C0F00202DE9F041044680F8AF
:10FD900075300888A4F87600FF2084F893004FF6A9
:10FDA000FF7016460D46A4F89400002B4BD128692D
:10FDB00009F098FDA4F88C00288BA4F88E00688BBD
:10FDC000A4F8900095F81B0284F89200207E04F1BC
:10FDD00051010F46002520B194F850000AF0F7FBBE
:10FDE00040B994F86A0070B194F8500039460AF0AE
:10FDF000E5FB40B1D4F85100C4F88000B4F85500D8
:10FE0000A4F8840003E0C4F88050A4F88450154896
:10FE1000FF2E40680178C1F3801184F8791050F802
:10FE2000031F17D0C4F886108088A4F88A0004F154
:10FE30007A02511E3046FEF717FB30B114F8790FE5
:10FE400040F002002070BDE8F08140F68B412D208B
:10FE5000FCF7B6FE44F87A1F8088A080E560258212
:10FE6000F1E70000D0000020F8B50446FF208DF82F
:10FE7000000001266A4605212046FFF7F3FE60B127
:10FE8000284D274F6968FA7B07F1100311F8030B1F
:10FE9000C0F3801009F049FC10B100263046F8BDCF
:10FEA0006A68E069127810F8A51FC2F34012114089
:10FEB000017001222046E16900F09AF800239DF8C4
:10FEC00000202046E169FFF75FFF1122164904F187
:10FED0006C000AF0B7F8E06905220188A4F8B010B8
:10FEE00090F8A50084F8B200104904F1A6000AF0C9
:10FEF000A9F80021E06939700A46214600F086FA27
:10FF00006868E169D0F8032041F8032FB0F80720B2
:10FF10008A800078E169C0F380108870BEE7000035
:10FF20005C0F0020D0000020F9A70100E9A7010024
:10FF3000F8B50446FF208DF8000001256A4603212C
:10FF40002046FFF78FFEE8B1207B20B19DF800101E
:10FF50002046FFF739FE0D4E002170680180042114
:10FF600009F0F7FE204600F08BF894F84420216C4D
:10FF7000706809F025FF064905200870706803F0D5
:10FF800097FD00E000252846F8BD0000D0000020C5
:10FF90005C0F002070B504460E46407EFEF73EFA28
:10FFA000050019D0102109F01EFE002814D10120EF
:10FFB00084F85E0004F15F0132460C46284609F0E1
:10FFC000E4FB2146054C606809F0DEFE6068BDE890
:10FFD0007040012109F0DEBE70BD0000D00000209D
:10FFE000024801210068FFF719BB0000D000002083
:10FFF0002DE9F041214E80460C467068154650F8B8
:020000040001F9
:100000000F1F6161416821F07F41E161408909F082
:1000100065FC0746206170683946807D09F0DAFD8D
:10002000A08470683946B0F8170009F0CFFD20624F
:10003000706830F81B1F2183418861834168C4F8D0
:10004000A610017A84F8AA10417A01F01F0184F801
:10005000B110407A400984F81B0204F16200057275
:100060004572FF218172002136380AF09AF898F81B
:100070000E0084F86E00BDE8F0810000D000002082
:1000800070B5074D044600F15101686809F089FE1A
:1000900094F850106868BDE8704009F088BE000010
:1000A000D0000020A9F8000031F7000025F800007A
:1000B00000000000FDF7000055F80000DDA701007A
:1000C000E3A70100BDFA0000E1FA0000E1FF000033
:1000D000C0000100B8000100B400010010B5421ECC
:1000E000022A01D9CA2109E0401E102909D012298B
:1000F0000CD013290AD0152905D0D8212F20FCF7C0
:100100005FFD054904E00449891D01E00249891F9A
:1001100031F8100010BD000044AA0100421E10B5C5
:10012000D2B2012A03D91D2901D0EE210DE01329F5
:1001300013D004DC10290BD0122904D10DE01529AD
:1001400008D01D290ED04FF481712F20FCF738FD07
:10015000074804E00648083001E00548001D30F873
:10016000120010BD40F25A3110FB01F010BD00002A
:1001700032AA01002DE9F041044690F8E00016464D
:100180000F4600285ED121464D4806F007FC054683
:10019000202857D05022002104F1C8000CF093FD14
:1001A00084F8C8500125C4F8CC7084F8E05037B109
:1001B000FEF7BAFE00F00700401C87F84C0220460C
:1001C0000AF0F5FDA4F8F000022084F8F200A84639
:1001D00084F8F350002504F8E85F07F06BFD07464C
:1001E0000CF06DFB2189E83C884200D80846384471
:1001F000CC3087B220460AF09DFA30B30CF033F9C8
:1002000000F5CD6081B2304607F074FE3044C4F88A
:10021000EC00903406F0D2FDC0196941C4E91A011E
:1002200084F8408024F86E5C01200AF0FBFB00F5A6
:100230008870301A60644FF0FF304108C4E91E0135
:10024000903C25E00C20BDE8F081002120460AF01A
:1002500000FDDFF87080C4F8EC000020B8F804104E
:1002600049B1618C39B1FEF75FFEB8F80410B0FBFC
:10027000F1F201FB1200074406F0A0FDC01969412C
:10028000C4E93E019EB1801951EB0501C4E9420168
:1002900094F8C80004F1E8010AF087FD58B1A4F809
:1002A0000051002120460AF075FA0020CBE74FF0FC
:1002B000FF304108EAE74FF4F4713020FCF780FC8E
:1002C00027AF0100E000002001498880704700004E
:1002D000E000002005480021017001228270417079
:1002E00042F21071818000F003B80000E0000020AD
:1002F0001CB50949D1E90001CDE9000102E00098EF
:100300000AF0CCFB6846FCF799FE0028F7D000F015
:10031000A9F800201CBD0000C40B010001490870B1
:1003200070470000E000002008494FF47A72B1FBEA
:10033000F2F110B501F5257109F04CFF40F64801C6
:10034000884200D3084680B210BD00007D520100F3
:100350002DE9F0410F4CD4E9026703F0C3FA0546DA
:1003600002463946304609F0C3FA0646A06886427E
:1003700005D02169301A0844206106F051FCA660BE
:10038000B54201D8607810B10020BDE8F0810120AD
:10039000FBE70000E000002010B5044606292ED23D
:1003A000DFE801F0051103141528002106E0D4F858
:1003B000AC0210B120460AF08BFC01212046BDE8BA
:1003C000104000F0F7B8032084F85C0210BD03F081
:1003D0008FFAC4F8AC0294F86B0003F04DFBD4F82C
:1003E000AC12091A084882680A448260C268114443
:1003F000C16010BD2046BDE810400AF054BC4FF467
:10040000E8613020FCF7DCFBE000002070B50C4612
:10041000054612B140F26A7110E003F063FA01463A
:10042000002220460AF033FD94F8C8002A46054908
:1004300006F06AF9002804D140F253713020FCF72D
:10044000BFFB70BDC9AF010010B50C2804D340F24A
:100450008B310620FCF7B4FB014931F8100010BDC8
:10046000E00B01002DE9FC41154D012068700024CE
:100470004FF6FF760BE0002108F0A8FF070009D037
:1004800097F8A40206F072F938460AF0F3FC0094DB
:1004900001940DE04FF490713020FCF791FB00982F
:1004A00030B190F85C1219B10088B042E3D104E099
:1004B0006846FCF7C3FD0028F1D06C70BDE8FC81F4
:1004C000E00000202DE9F047044639481E469046DA
:1004D000807889460025002863D007F0C1FCE0B38E
:1004E000B4F8480202285CD394F85C02022858D081
:1004F00094F8720288BB94F81B02FFF7A5FF00F581
:10050000C86081B2318094F85C02002701280DD0C8
:10051000206907F0EFFCB4F836224244A2EB09014F
:10052000D4F86422821A01FB027535E094F8A10028
:10053000032839D00121002009F0A5FA216A4718C3
:100540003188D4F8540207F0D5FCD4F85022D4F8FE
:100550005812821A01FB025500E022E0C4F8500252
:100560003188384607F0C6FCD4F86012C4F860023F
:10057000411A0D443188206907F0BCFCB4F83622DA
:100580004244A2EB0901D4F85822891AD4F8642213
:10059000821A491E01FB0255C4F86402012084F846
:1005A00072022846BDE8F087D4F85402C6E700007E
:1005B000E000002038B500250446012902D110488A
:1005C000407870B1042084F85C0200BF0AF079FB27
:1005D000A4F8A252B4F89400A4F86E0284F8715200
:1005E00038BD0095B4F8241201230022204600F003
:1005F00009F80028EAD040F2B5613020FCF7E0FAB3
:10060000E00000202DE9FF4F8BB0044690F86B000E
:1006100099460F46079305900BF025FF054694F881
:100620001B02FFF711FF2844ADF8040094F89E0068
:100630000D2804D0002008900D9810B12EE0012064
:10064000F9E794F85C02032828D1089830B3B4F88D
:10065000CC02B84222D1D4F86402C4F85002206916
:10066000C4F85402B4F8A202B4F836120844C4F82C
:100670005802204600F0C0FAD4F8D0022062B4F844
:10068000CE02A084D4F8D4022061B4F8D80220832A
:10069000B4F8DA026083022084F85C02B4F89400B3
:1006A00004F51E75381A0FFA80FAB4F8A002381A49
:1006B0000FFA80F8B8F1000F08DAD4F89002D4F8F5
:1006C0009412D046C4E9A6010120079001AB52461E
:1006D00041462046FFF7F6FE049094F85C02DFF8EE
:1006E00034B340B101287DD0022851D003287AD0FC
:1006F00040F243518AE10121002009F0C4F9064685
:10070000206ABDF80410304407F0F4FBC4F860021E
:10071000BDF80410206907F0EDFBC4F8640207A9D6
:1007200006A803F047F8D4E9A601DDE9062306F0A0
:1007300057FB824620460AF0B6FA94F86B00D4F8CC
:10074000A88203F0C5F94AF2A13101444FF47A704E
:10075000B1FBF0F0216AD4F860223144081A811A02
:1007600041442039A1EB0A065000A18C60300144BD
:1007700094F86B000AF007FB2230CBF81400D4F891
:10078000A802301AB0F5DE7F58D240F2DC413DE1DC
:10079000216AD4F854020844BDF8041007F0AAFBFB
:1007A000C4F86002BDF80410206907F0A3FBC4F888
:1007B000640220460AF077FAB4F8360210BBB9F1A9
:1007C000000F1FD094F86B80404603F081F94AF285
:1007D000A13101444FF47A70B1FBF0F0D4F860120B
:1007E000084401E02BE047E0226AD4F85412114497
:1007F0000E1A404603F040F9D4F8AC12081A064429
:10080000203E06E0216AD4F854020844D4F860126D
:10081000461AD4F85822D4F85012D4F8600201FBDA
:1008200002004000A18C6030014494F86B000AF093
:10083000AAFACBF81400012084F85C0261E0D4F835
:1008400064222069B4F83612861A01EB0A00D4F843
:100850005812D4F850C2401AD4F86032401E0CFB33
:10086000013100FB02104000A18C6030014406FB06
:1008700008F694F86B0040E02069D4F8641200FB9D
:1008800008F008FB110694F89D00252803D094F881
:100890009E00252809D1B4F8CC02381A00B20028ED
:1008A00003DB94F8CF0200B105900798D8B1B4F8F3
:1008B0003602C0B9D4F8AC0200287DD094F86B00A1
:1008C00003F006F94AF2A13101444FF47A70B1FB0A
:1008D000F0F0361A94F86B0003F0CEF8D4F8AC12AE
:1008E000081A0644203EB4F8361201EB0A00D4F888
:1008F000641248434100603105980AF044FACBF88D
:1009000014000498DBF81420311AD4F864622069CA
:10091000801BA0F24620CBF81800824200D8104677
:10092000C4F8300200262E7064202881D4E9A62065
:1009300051187041C5E9041004F12C0009F01BFCAA
:10094000D4F8301208446860D5E90401C4E9A6016E
:10095000A4F8A072AE72B4F82002C01B00B2002846
:1009600001DD0220A872089838B3B9F1000F1CD03D
:10097000B4F84812F1B3B4F84A0200BFA4F84A022E
:1009800094F84C22401C42438A420ED2A87A60B1AD
:10099000AE72B4F84A02401CA4F84A02FEF7BEFA4E
:1009A00000F00700401C84F84C0294F8A402294689
:1009B0000AF0FBF940B301E009E00BE00D9880F08C
:1009C000010084F8700200200FB0BDE8F08F40F203
:1009D0002E511BE0B9F1000FCAD194F85C02002837
:1009E000E3D0D4F864122069411A284609F05DF872
:1009F000000400E006E0000CD7D0189901B108808F
:100A00000120E1E70020B9E740F28C513020FCF7EB
:100A1000D7F80000E000002070B504460BF04FFF4F
:100A2000642801D9054600E0642594F86B0028216C
:100A30000AF0C7F82844D4F8641200F510700E18B4
:100A400094F86B0028210AF0BCF800F529722046C2
:100A5000E16A09F02FFB054632462046216909F07C
:100A600029FB09498542C86000D2284688600A7877
:100A700002B9C860D4F87C02A0F269100861BDE830
:100A8000704006F0CDB80000E00000207CB50446C0
:100A900006F094F9D4F89032D4F89422C01A61EB9D
:100AA000020100221346121A8B4102DB40F2096157
:100AB0004DE0421C71F1000102DB40F20A6146E0A8
:100AC000226900210AB1B0FBF2F194F89E000D28D2
:100AD000B4F86E021BD0B4F894205318C31A1BB29A
:100AE000002B01DB401C01E0491C5018A4F86E02E9
:100AF00094F871028DF80000009800909DF80000B5
:100B000040B9B4F86E02B4F82412884202D1401CF5
:100B1000A4F86E02B4F8A202401CA4F8A202B4F831
:100B2000CE00B4F8CC10401AB4F89410401E08441B
:100B300085B226E001A8002300901A462046FFF760
:100B400061FD00283AD0012804D040F249613020EC
:100B5000FCF736F8B4F86E02B4F82012421A12B25A
:100B6000002A09DABDF804200244AA1A12B2002AA7
:100B700002DAA4F86E1204E0BDF804100844A4F8E8
:100B80006E02B4F86E12681A00B20028D2DA94F835
:100B9000A10088B15FF0080084F8BD000B2208496D
:100BA00004F1B40009F04EFA20460AF08EFA20460D
:100BB000BDE87C400AF05EB93E20EDE77CBD000058
:100BC00083A30100000000000000010000000000FD
:100BD0000000010000000000141E000030110000A1
:100BE000F401FA00960064004B0032001E0014006D
:100BF0000A0005000200010010B50446D0F8D40236
:100C00002169884209D1B4F8D812228B914204D1CB
:100C1000B4F8DA12628B914214D02188A4F8CA1178
:100C200008F060FEA4F8CC01B4F8D802A4F8CE0114
:100C3000B4F8DA02A4F8D0010922074904F5DF70FC
:100C400009F014FA02212046FDF780FD002004F887
:100C50009E0F0320E07010BDC7A3010006480549A0
:100C60000165064941650748054901650649416531
:100C700070470000DD1F010014010020C1200100A9
:100C8000EBB20100C001002015B301001E481D4950
:100C900081601E4941601E4901601E4981621E49F2
:100CA000C1621E49C1601E4981611E4901631E491E
:100CB00001621E49C1641E4981641E4941641E4986
:100CC00041631E49C1611E4941621F481D4981603F
:100CD0001E49C1611E4941621E49C1621E4901612E
:100CE0001E4941611E4941641E4941631E4981619B
:100CF0001E4901631E4981641E49C1641E49816306
:100D0000704700000124010014010020CD1D0100E6
:100D1000391E0100ADB10100F7B10100F91E01005B
:100D20000FB20100C5240100951F01007FB1010031
:100D300059B1010079230100AD23010039240100DC
:100D4000A11F01005FB40100C0010020A125010026
:100D5000E7B201007FB30100C1B2010041B401005C
:100D6000EFB301001FB401002D25010081B4010083
:100D700045B301006FB301003DB4010006480549C9
:100D80008165064901660748054981650649C165CF
:100D900070470000412101001401002025220100BC
:100DA000A5B30100C0010020CFB30100F8B57C4C11
:100DB0000121A4F110062170002560607580757016
:100DC000357080F82B120088FCF70CFB80B160684E
:100DD0000088FCF76FFD60680088FCF713FD606811
:100DE000B0F82212C9B180300AF07EF918B114E0CF
:100DF00040F659516CE0606890F830118DF80010A1
:100E0000009900919DF8001039B190F89F200123BE
:100E10001946803008F07FFD80B1606880300AF0AC
:100E200063F928B1606890F8260100BF00F0B4FBB8
:100E3000606890F82D1289B1B5801EE06068A0F856
:100E4000D05090F8311180F828110021022000F0D4
:100E500063FE606880F82A520220E7E790F8C61126
:100E60008DF80010009900919DF8001019B9C18CFF
:100E7000028B914200D8018BB180B0F82612491E36
:100E80008FB2B0F828123944A0F8281230F8CC1FDD
:100E90003944018001F0B2FB20B1606850F8C01FF6
:100EA000394401606168B1F82202012802D8401C6F
:100EB000A1F822020FB181F8345281F82A52B1F818
:100EC000262201F1800008F0CAFE20B14FF45A61D9
:100ED0003120FBF775FE606890F89E100A2901D05A
:100EE0000B2919D1B0F89420B0F8CC32D21A12B232
:100EF000002A11DBD0F8CE12C0F8A61090F8D2125A
:100F000080F8AA100321FDF721FC606880F89E504C
:100F1000FF2180F8F41026E0252911D1B0F89410B3
:100F2000B0F8CC22891A09B2002909DB80F89E505A
:100F300000F0ACFE0028606880F83C5129D012E037
:100F400090F89D10252901D027290CD1B0F89410D4
:100F5000B0F8CC22891A09B2002904DB80F89D5030
:100F600000F094FEA8B10F480090D6E904010E4BA2
:100F70000E4AFCF72DFD60680123052190F89E20A4
:100F8000803008F0C8FC002809D0BDE8F840FCF724
:100F900019BDBDE8F8400021084600F0C9BBF8BD06
:100FA0000C010020311701006D120100D91B010056
:100FB00004480021406820F8D81F8178491C8170BE
:100FC000704700000C010020074810B5416811F877
:100FD000DA0F401E40B20870002804DA40F2012106
:100FE0003120FBF7EDFD10BD0C0100201D4908B5B7
:100FF000496891F89E20C0B1112A06D0152A07D061
:10100000162A09D01C2A28D109E001210B2008E06A
:1010100014480AF00DF906E000F09CFD03E0012100
:10102000062000F079FD012008BD222A04D02F2AD5
:1010300013D101211120F4E791F83C0102280ED0D0
:1010400091F83C01012808D191F83D018DF800008C
:10105000009800909DF8000008B1002008BD012113
:101060001720DEE70C01002038B5002876D13C4C73
:101070006068D0F88C10CA0702D00121092069E00D
:101080008A070AD501210C2000F046FD606810F89F
:10109000DD1F41F0010101705EE04A0702D5012128
:1010A000132057E00A0706D590F8201180F8281180
:1010B000012107204EE011F0300F47D090F8331196
:1010C0008DF80010009900919DF80010D9BB90F8A0
:1010D000321100258DF80010009900919DF8001044
:1010E000C1B190F89E1025292ED090F89D10252989
:1010F0002AD0002300F2CE2200F5997108F0CCFF2F
:10110000606850F88C1F21F0200141F0100101604F
:1011100080F8A650606890F88C10C9061ED508F0BB
:10112000D6FF05216068FFF737F900F025F96168FF
:1011300001F12C00C28BA1F82821408CA1F82A01D2
:101140000121152006E009E00123D3E7480605D573
:101150000121242000F0E0FC012038BD002038BD32
:101160000C01002070B50D46064608F0D3FE04467B
:10117000304608F0D1FE294600F01EF8B8B12046EE
:1011800008F073FC01000DD00A48406890F86B200D
:101190008A4207D090F83C11012905D090F86700E9
:1011A000204204D0012070BD90F83F01F8E70020F4
:1011B00070BD00000C01002070B50D46044608F01B
:1011C00054FC50B31649496891F86A20824224D0F1
:1011D00091F83C31012B05D091F86630234213D0B1
:1011E0001DB11AE091F83E31F8E791F86310214201
:1011F00013D15AB1042A0ED004280CD0082A0AD0E0
:10120000082808D0824208D9002070BD40F2A311FE
:101210000620FBF7D5FC8242F6D3012070BD00000A
:101220000C01002010B5104C01230021606890F8DB
:101230009D20803008F06FFB40B1606801230421DD
:1012400090F89E20803008F066FB08B1002010BDA9
:10125000606890F8CA000028F9D00021122000F040
:101260005BFC012010BD00000C0100200D4902466E
:101270004878A0B901F11000406842B189780907A7
:1012800003D590F89F00072809D00120704700F18E
:101290002C018A8C818E8A4201D8FFF759B8002030
:1012A00070470000FC00002038B5324C05466068ED
:1012B000803009F019FF00285BD1002D59D16068FA
:1012C0000123194690F89F20803008F024FB002865
:1012D0004FD1606890F830118DF80010009900919E
:1012E0009DF80020002142B1A0F8D01090F83111F3
:1012F00080F828110021022030E090F89E20012380
:101300000421803008F007FB0546FFF7ADFE0028FA
:101310002FD12846FFF76AFE00282AD1FFF782FF67
:10132000002826D1606890F89D1009291AD0002D58
:101330001FD100F01DFB00281BD160680123002194
:1013400090F89D20803008F0E6FA002811D06068FF
:1013500090F8C40200280CD00021FF20BDE83840DE
:1013600000F0DABB90F8211180F828110021072045
:10137000F4E738BD0C0100200848436893F860008A
:10138000012806D003F5B17203F12C011888FDF78E
:1013900047BD022083F86000704700000C01002068
:1013A000F8B52B4D060005F1100433D100F0AAF872
:1013B00000F052F806002DD16988480706D560680C
:1013C00090F89F00062801D101202870880716D5C3
:1013D000A868C0782B2807D21E4951F8201019B1EF
:1013E0001B48103088470AE0FF2804D040F602115D
:1013F0003120FBF7E5FB1648103009F058FFA878BC
:10140000C00607D5606890F89E100A2902D10B210A
:1014100080F89E106878000718D5606801230521C0
:1014200090F89E20803008F076FA08B108260DE08A
:101430000025694603200095FCF78CFB009828B135
:1014400005722A226168009808F0FCFD3046F8BD5C
:10145000FC000020C001002070B5284D0020A978B4
:10146000C90717D0E86805F110040123C678606841
:10147000052190F89E20803008F04DFA58B1B61E34
:101480000A2E06D2DFE806F007070505070705055F
:101490000707082070BDE868FDF778FA38B3E868F8
:1014A000C5781DB1012D01D0162D13D1606890F8BB
:1014B0009D0008F088FA68B1616891F89D002028C5
:1014C00008D0212803D0162D0FD0022070BD2E2069
:1014D00081F89D002B2D0AD2094850F8251031B112
:1014E000BDE87040054810300847202070BDBDE8B9
:1014F00070400248103000F059BD0000FC00002090
:101500001401002070B5234EB078000740D506F1D5
:1015100010046068803009F0E7FD48B16068FE2182
:10152000002580F8261190F89E101A290CD104E0AD
:1015300040F60E113120FBF743FB80F8DB50FFF73C
:1015400043FD606880F89E50606890F89D102029E7
:1015500002D0312913D10BE090F89E0008F033FA45
:1015600008B12E2000E02120616881F89D0006E08E
:10157000012180F8C51280F89D5080F8D65060682F
:1015800090F89F10072903D10221317080F82611AD
:1015900070BD0000FC00002038B505466846FCF729
:1015A00073F908B32222002100980BF08CFB032171
:1015B000009808F0C9FC0098017801F0EF01017073
:1015C0002946FDF7F3F9594C112D2DD00FDCA5F16B
:1015D00002050D2D1FD2DFE805F0211E519E9E2130
:1015E0001E5E1E9E3A348C0040F6B53199E0172DF0
:1015F00070D008DCA5F11205052D0CD2DFE805F04E
:101600008B8B50503300232D77D0242D75D0252D72
:1016100073D0FF2D77D040F6614182E06068009979
:1016200090F82801087176E0606890F8231100981E
:1016300008F076FC606890F82211009808F074FCBD
:1016400069E06168009891F82211017163E00098E7
:101650000C21017159214171002181714B21C1710E
:101660001221017257E00098D4F8041091F83E114D
:101670000171616891F83F1141714CE06168009817
:1016800001F5107108F007FC6168009801F58E7192
:1016900008F0FEFB3FE025480099FDF7D7FC3AE053
:1016A0006068B0F84C10009808F056FC6068B0F81C
:1016B0002A11009808F054FC6068B0F848100098AF
:1016C00008F052FC6068B0F82811009808F050FC4F
:1016D00021E0FFE7616891F83C0101280098C5D03E
:1016E00091F866100171616891F86710C4E704E031
:1016F00009E00098FDF75AFC0DE00C4A28460099D5
:1017000009F012FF07E0606890F8C722D0F8C8120D
:10171000009808F00BFCFCF791F8002804D140F683
:1017200065413120FBF74CFA38BD00000C01002068
:101730002DE9F35F8C4E8A4670680088FBF752FEF5
:1017400007000CD0A6F110054FF000046888C00512
:101750000AD57068A0F8CC4080F8344209E040F621
:1017600045713120FBF72CFA716831F8CC0F401C21
:10177000088000F043FF4FF0010940B3688800057E
:1017800006D5706890F8A31011B1C0F8C0401EE0F3
:101790007068D0F8C010491CC0F8C010D0F8C42040
:1017A0008A4201D3531A00E00023B5F804C00CF1BB
:1017B000050C634501D880F8CA90914207D3C0F860
:1017C000C0400F22694900F5AC7008F04FFC6888F2
:1017D0004FF0020B10F4407F0ED0706890F8A1100B
:1017E00011B1032908D102E080F8A19001E080F84E
:1017F000A1B00121FEF7D0FD7068B04690F8A110AD
:10180000012904D16988490501D580F8A1B0009962
:10181000002979D1A978490602D5A0F8484204E008
:10182000B0F84812491CA0F848125046FFF7B8FD1E
:1018300040EA0A008246FFF737FDD8F80460B6F8A0
:101840002802401CA6F8280296F82C0228B1FCF7C2
:10185000BFF9B0B1A6F8284213E0FCF797F808B139
:10186000A6F82842FCF78CF858B196F83402401CD0
:10187000C0B286F83402022803D9A6F8284286F8B6
:101880003442D8F804004646012390F89E200021F7
:10189000803008F040F820B9706890F89E000B285E
:1018A0005FD170680123002190F89D20803008F0FE
:1018B00032F850B370680123002190F89F208030E7
:1018C00008F029F808B3706890F8A110022948D1EF
:1018D00090F83402C8B9384607F024FBA8B1706804
:1018E000803009F001FC80B97168B1F8220201284A
:1018F00037D981F82A92B1F8CE20B1F8CC00931EE6
:10190000984203DB012004E01CE02AE0101A401E8C
:1019100080B2B1F82832AA88934201D3012202E0B2
:10192000D21A521C92B2904200D91046012801D11D
:1019300081F82A427168B1F894201044A1F8240279
:1019400000F028FFA8785246C0F38011009800F0FC
:1019500069FED8F8040080F82B42BDE8FC5FFBF775
:1019600057BF01207168E3E70C010020CFA40100FC
:101970007CB5684C01230021606890F89D20803080
:1019800007F0C9FF00287AD0606890F8431100255D
:1019900039B100210E2000F0BFF8606880F8435193
:1019A000B5E090F8421119B190F8DD10890716D012
:1019B00090F832118DF80410019901919DF80410EE
:1019C00041B190F833118DF80010009900919DF805
:1019D000001089B190F83C11012930D040E000217D
:1019E0000C2000F099F8606810F8DD1F41F001014B
:1019F000017080F865508AE090F89E1025291CD06F
:101A000090F89D10252918D05FF0000300F2CE2237
:101A100000F5997108F040FB606880F832510021B0
:101A2000142000F079F8616801F12C00C28BA1F854
:101A30002821408CA1F82A0169E00123E6E790F80B
:101A40003D118DF80010009900919DF8001039B9F2
:101A500090F89E2001230B21803007F05CFF78B1C5
:101A6000606890F849118DF80010009900919DF878
:101A70000010B9B30021232000F04EF847E030E019
:101A8000606890F86A0009F037FB0546606890F8D6
:101A90006B0009F031FB0646606890F83E1128465D
:101AA00009F035FB50B1606890F83F11304609F0FD
:101AB0002EFB18B1002000F041F911E0606801230D
:101AC000032190F89E20803007F025FF40B9606820
:101AD0000123022190F89E20803007F01CFF10B1F6
:101AE00000207CBD02E000211620C5E790F84601E9
:101AF0008DF80000009800909DF800000028F0D0BC
:101B00000021252000F008F8606880F84651012087
:101B1000E7E700000C01002070B50D4C06460D46AD
:101B20006068803009F0E0FA20B140F66A41312067
:101B3000FBF746F862680020012D82F8266104D088
:101B400022F8D20F0120107170BDA2F8D80070BD2C
:101B50000C01002038B51F4C0025606890F8B012C9
:101B600001290CD0022933D190F8DC1000294FF064
:101B700006011AD080F828110121022023E090F8F4
:101B800012128DF80010009900919DF800100029A4
:101B90001ED100F5847300F50E71002200F2B12011
:101BA00007F071FE012105200DE0032000F0B4FCD8
:101BB000606890F8EC00800810F0010F01D011204F
:101BC00000E00D200121FFF7A7FF606880F8B05208
:101BD00038BD00000C01002070B52B4B0246588820
:101BE0001043588003F11000402A40680DD096073A
:101BF0004FF000054FF001044FEAC2760CD54EB10C
:101C000040F6B2613120FAF7DBFFBDE870400421F5
:101C1000FEF7C2BB99601CE0C6B1D960C97806293D
:101C200002D00B2912D109E090F89E1018290DD18D
:101C30000021C0E93E1180F8A24007E090F89E1014
:101C4000122903D180F8A25080F8DC40910716D504
:101C50009968C978052902D00B2910D109E090F8BC
:101C60009E1016290BD10021C0E9401180F8A34035
:101C700005E090F89E10112901D180F8A35090063C
:101C800001D50820587070BDFC0000202DE9F041FE
:101C9000294C0125636893F8CE1209B1012700E0B1
:101CA000002793F8CF0208B1012600E000260FB903
:101CB00093F86A100EB993F86B0083F86A1083F8F2
:101CC0006B0003F16202FF209072184609F0EEFCEF
:101CD000606890F83C01012801D007B916B10020D6
:101CE00000F02CF860682C3008F045FA0646606871
:101CF00008F0EDF930B1616801F5B17231F82C0BE3
:101D0000FDF78EF805216068FEF746FB60682C3011
:101D100008F031FA0446A6420AD203F091FF0146C8
:101D2000A01B652800D2652003F0ACFE00B10025A1
:101D30002846BDE8F08100000C01002010B5104CD1
:101D400061680A88A1F8A62181F8A40191F86A00C7
:101D500009F0D2F9616881F8A80191F86B0009F0E7
:101D6000CBF963681522074983F8A90103F5CD7003
:101D700008F07CF96168002081F83C0110BD00008A
:101D80000C0100209BC4010070B50F4D6C6894F8E5
:101D90009D10212902D02E2903D011E0FFF7CEFF9C
:101DA00008E094F89E2004F1800001230B2107F045
:101DB000B2FD38B16968002081F89D0081F8D60035
:101DC000002070BD2A20E9E70C01002070B5044610
:101DD00040680123002190F89E20803007F09BFD91
:101DE000B8B1134DE86808F001F86168A1F8CC02B9
:101DF0006168B1F8941009F098F960B16168282021
:101E00000B2281F8BD0060680A49B43008F01AF965
:101E10000BE0012070BD6168E86801F2CE2107F097
:101E2000E0FF61680A2081F89E00002070BD00007C
:101E3000FC00002083A3010070B504464068012324
:101E4000002190F89E20803007F065FDE0B1284D1C
:101E50000021E86807F0CDFFC0B1E8686168B0F81C
:101E60000D00A1F8CC026168B1F8941009F05DF999
:101E700088B1616828200B2281F8BD0060681D4987
:101E8000B43008F0DFF830E0012070BD2046BDE836
:101E9000704000F08BB8E86807F0D5FF07F01EFD32
:101EA000064660683146C0F8D462E868007907F0F9
:101EB00091FE6168A1F8CE02E8683146B0F80500ED
:101EC00007F084FE6168C1F8D002E86807F0BEFF41
:101ED0006168A1F8D802E86807F0BBFF6168A1F863
:101EE000DA0261680D2081F89E00002070BD0000BC
:101EF000FC00002083A3010070B504464068012364
:101F0000002190F89E20803007F005FD70B96068D0
:101F100090F89E20132A09D001230521803007F074
:101F2000FAFC08B1082070BD012070BD606890F80F
:101F3000DC0008B9FFF73CF8144D616801F50E713B
:101F4000E86807F09FFF6168E86801F58C7107F0A9
:101F500090FF60680188A0F8E6126168E86801F502
:101F60003A7107F08AFF6168E86801F53C7107F093
:101F70007DFF60680A22064900F5377008F062F8B4
:101F80006168152081F89E00002070BDFC000020D3
:101F900039A401000149C968FCF7E6BFFC00002034
:101FA0000149C968FDF710B8FC00002010B542686F
:101FB000D2F88C100B0701D5012010BD41F00801AB
:101FC000C2F88C1004494068C968C97880F82011AB
:101FD000FEF7EEFF002010BDFC0000202DE9FC41C3
:101FE0000546406890F88C0010F0300F02D00120B8
:101FF000BDE8FC81314CE06807F05EFF30B3E0687B
:1020000007F054FF8046E06807F054FF0746E06899
:1020100007F04AFF0646E06807F04AFF0146CDF8A0
:10202000008068683B4632462C3008F0DEF8A07825
:1020300081074FF0010003D5A168C97814290AD09F
:10204000696891F89D101D2905D007E02846BDE874
:10205000FC41FFF7ABBF696881F86000686890F8E1
:102060006010012911D090F833118DF804100199F6
:1020700001919DF8041041B990F832118DF80010CB
:10208000009900919DF8001041B150F88C1F41F06B
:1020900010010160FEF78CFF0020A9E750F88C1FAB
:1020A00041F02001016005481030436803F12C0124
:1020B000188803F5BC72FCF7DDFEEBE7FC0000209E
:1020C0002DE9F8430446406801230A2190F89D2039
:1020D000803007F020FC70B3184DE86807F0ECFE84
:1020E000E8B1E86807F0E2FE0746E86807F0E2FEBC
:1020F0008046E86807F0D8FE0646E86807F0D8FE94
:10210000014600976068434632462C3008F06DF86F
:10211000606807F0DCFF05216068FEF73DF9616843
:10212000002081F8D600616881F89D00FFF724F94E
:102130000020BDE8F883FFE70120FAE7FC0000205B
:1021400038B50446406801230B2190F89E2080306A
:1021500007F0E1FB60BB60680123002190F89E203E
:10216000803007F0D8FB08B3606890F89D00252800
:102170001ED02A4DE86807F0B1FED8B1E868626861
:10218000417901F0070182F86310007900F007013E
:10219000606880F86210606890F83D218DF800203A
:1021A000009A00929DF800207ABB08E0012038BD1B
:1021B000202038BD2046BDE83840FFF7F7BE90F834
:1021C0003C21012A21D000F16A0290F86330557851
:1021D0008D4206D11178994203D1022180F83C1139
:1021E00013E00E481030416801F5CB700A8820F8E2
:1021F000022B91F8622000F8012B91F8631000F88F
:102200000D192222064907F01DFF6168222081F87E
:102210009E00FEF7CDFE002038BD0000FC0000202F
:10222000C5C401002DE9F8434568044695F89D00B2
:10223000212808D05FF0000695F89E00232804D0DE
:102240008EB39D3502E00126F6E79E35DFF820814A
:10225000D8F80C0007F04EFE002740B33146D8F8FE
:102260000C00FEF77FFF10B36A4646466068D8F858
:102270000C1007F065FCC0B3F06807F039FE616828
:10228000A1F8CC026168B1F8941008F04EFF68B371
:10229000616828200B2281F8BD0060683549B430A0
:1022A00007F0D0FE58E0FFE70220BDE8F883606841
:1022B0004FF0000990F83C11012918D080F83C71CA
:1022C0000EB3D8F80C0061680122C07881F82101B2
:1022D00082406168C2F3006068B1092081F89D0006
:1022E000606890F8D600A8B908E015E028E01E2044
:1022F000FFF724FDE4E740F2834101E040F28B4127
:102300003120FAF75DFC2F70FEF75EFE2046FFF7E6
:102310004DFE81464846C8E7606890F83C110129A7
:1023200009D080F83C71606800F19E01A94213D188
:1023300080F89E7010E00020FFF700FD2F70F2E79C
:1023400061689DF8000081F8CE0261689DF8010087
:1023500081F8CF0225202870606800F19E01A94213
:1023600002D1FEF731FE01E080F8D67000209CE734
:10237000FC00002083A3010070B5044640680A4DAC
:1023800010F8EC1F41F004010170E86807F0C6FD89
:102390000646E86807F0C6FD014622463046BDE81D
:1023A000704000F095B80000FC0000200246134881
:1023B000C068017911481030436893F89D002128C6
:1023C00010D02E280ED028280ED004280ED00F288A
:1023D0000ED01D280ED093F89E0023280CD0FE208E
:1023E00000F076B81620FBE72320F9E70E20F7E788
:1023F0001220F5E71420F3E71720F1E7FC00002096
:1024000010B5044640680123194690F89F2080309B
:1024100007F081FA08B1002010BD0648C06807F037
:10242000ABFD616881F8A0006168062081F89F001B
:10243000F1E70000FC00002070B504461F480025AD
:10244000C06803796068162B90F89D0013D006DCF5
:102450000E2B09D0122B07D0142B2CD104E0172BF4
:1024600002D0232B27D11FE022460121184609F074
:1024700009F805461FE0212801D02E281BD120464F
:1024800008F05FFE606890F89E10222913D00821A2
:10249000EC3008F00AFE60680B21EC3008F005FE15
:1024A0001A20FFF74BFC06E0282804D104480168F5
:1024B00009B120468847284670BD0000FC00002076
:1024C000700200200149C968FCF7F2BDFC00002041
:1024D00003460020172B17D00ADC0E2B14D0122B2A
:1024E00012D0142B10D0162B12D10846FFF74CBC7B
:1024F000232B03D0242B01D0252B09D1054A1268A8
:10250000002A05D0184610470021184608F0BABF27
:10251000704700006C020020034A526882F82301D1
:1025200082F82211704700000C01002070B50446AB
:10253000406890F89E101C2904D040F64E013120CE
:10254000FAF73EFB002580F8DB50606890F8DC105D
:1025500061B180F8DC5060680D220188A0F8161285
:1025600060680D4980F8145260680CE00188A0F89A
:102570001612606880F81452616801200C2281F8FC
:1025800018020649606800F20A2007F05BFD6068E7
:1025900080F89E5070BD000023A4010005A4010036
:1025A000154910B589680A79416891F89D30092B61
:1025B0000AD191F82131934206D1002281F89D2061
:1025C000406880F8D62010BDD1F88C301C0707D5A4
:1025D00023F00800C1F88C00BDE81040FEF7F4BC01
:1025E000FF2A04D040F2EA713120FAF7E9FABDE897
:1025F000104008F05CBE0000FC000020084810B548
:10260000406890F8A31041B990F89E20012306215C
:10261000803007F080F9002800D0012010BD0000B4
:102620000C010020F8B5594C06461546606800229A
:1026300011B1A0F8362206E0B0F83612B0F8262222
:102640001144A0F8361290F830118DF8001000995E
:1026500000919DF8001039B990F89F200123194688
:10266000803007F058F930B1606830F8D01FB0F80A
:10267000562111440180606890F8D62032B1B0F83C
:10268000D210B0F826321944A0F8D21090F9DA30FE
:10269000002B06DDB0F8D810B0F826723944A0F847
:1026A000D81090F8BD1009BBBEB938491039097867
:1026B000022906D001290AD0F5B1E9060BD51E2161
:1026C00042E090F8281106293ED016213CE090F80F
:1026D000A01059B954E0290701D53D2134E0A906DD
:1026E00001D5232130E0A90701D02A212CE040F6B2
:1026F0005E613120FAF764FA2AB1B0F8D210B0F86E
:10270000D420914216D2002B05DDB0F8D810B0F8D5
:10271000D42091420ED2B0F8D020B0F8CE108A4228
:102720000AD390F830218DF80020009A00929DF88D
:1027300000200AB1222107E090F8A12072B1B0F880
:10274000CC208A421CD3082190F8BC208DF80020B0
:10275000009A00929DF800206AB905E0B0F8CC100C
:1027600006290DD33E21EFE780F8BD100B22084962
:10277000B43007F067FC6068BDE8F84008F0A5BC1D
:10278000BDE8F8400021FDF707BE00000C01002065
:1027900083A3010070B52E4D686890F8A11051B167
:1027A000012908D0022909D0032907D040F6D741D2
:1027B0003120FAF705FAB0F8241237E090F89F10AC
:1027C000072936D0B0F8CC20B0F8CE100024931CE6
:1027D000994206D3891A891E0C04240C01D0641E68
:1027E000A4B290F8CA1039B190F89D2001230921B4
:1027F000803007F090F840B3FFF700FF78B16A68C7
:102800000020D2F8C410D2F8C020931C994203D300
:10281000881A801E00D0401EA04200D284B20CB1A3
:10282000641EA4B26868B0F824122144A0F82012F3
:1028300070BDB0F8CC100329BDD330F8941F428F7F
:102840001144491CA0F88C1170BD0024EAE7000077
:102850000C01002070B544680D2204F59875002124
:1028600004F16F000AF02FFA4FF4A3700021A4F8CE
:1028700044110155A5F81710697608465FF07F01ED
:1028800004EB4002401CC0B282F874100228F7D357
:1028900094F96E10204608F0E3FE0020FF21221874
:1028A000401CC0B282F877100228F8D370BD000037
:1028B00003494A880280097881700020704700002F
:1028C000200F00203EB50C4605460088694606F0FC
:1028D000F8FF002228B1C4F80220A2712280022051
:1028E0003EBD019911F1800181F87420D1F82600D4
:1028F000C4F8020091F82A00A0712888208091F87D
:1029000074008DF80800029802909DF808000028D5
:10291000EAD13EBDFEB50D4606460088694606F082
:10292000D0FF00281AD1DDF80440002784F86C702D
:1029300014F86A0F09F0A0FBA870607809F09CFBFE
:10294000E870A0788DF80800029802909DF80800C1
:102950006A3C0028EAD1308828800020FEBD0000B3
:1029600003498A880280C98841800020704700009E
:102970007C0200203EB5002402A98DF804408DF8A9
:102980000840009182784178007801AB09F0E8FCBA
:10299000002812D19DF8040009F022FC70B19DF8C6
:1029A000080009F01DFC48B105489DF8041081732A
:1029B0009DF80810C173048200203EBD11203EBD69
:1029C000200F00202DE9FC410F460546067809F04E
:1029D000BAFB00280AD1284609F08FFB002805D150
:1029E0000120FAF7E1FA864202D30720BDE8FC8114
:1029F0000121304606F0EAFC040004D008F077F824
:102A000068B10C20F2E70121304606F0D5FC040045
:102A100013D0174890F90010204607F02AFE2046F0
:102A200007F092FE3870E87429462046FCF7E6FC71
:102A30000646687ED0B12EB118E041F2E831392067
:102A4000FAF7BEF800226846616B06F071FD0022BD
:102A50000121606B06F0E6FD04226846616B06F01A
:102A600067FD00221146606B06F0DCFD3046BDE7D5
:102A700074020020017871B1417861B141881B294D
:102A800009D381881B2906D3044902680A6080881B
:102A9000888000207047122070470000200F00201F
:102AA000006840F2E241884203D303498860002075
:102AB0007047122070470000200F0020034AD2E91F
:102AC00004120160426000207047000008300100DD
:102AD0000EB50088694606F0F4FE60B9019809F069
:102AE000FBFB40B10198014690F84221803001F58E
:102AF000A17162B901E002200EBD90F866208DF848
:102B00000820029A02929DF8083001220BB13A2067
:102B10000EBD90F85D309B0706D0032205495E305C
:102B200007F0A4FA00200EBD0A70684607F067FAA5
:102B3000F8E70000E1A4010010B5052000F0F6FA66
:102B4000FEF78CF802490148486010BD812B010056
:102B5000740200201CB50949D1E90001CDE900014A
:102B600005E0009807F0C3FF08B101201CBD6846CE
:102B7000FAF764FA0028F4D000201CBD08300100E8
:102B80002DE9FE431346334A0F46B0F8541014881B
:102B9000B0F852608C4200D2214688469188B142FA
:102BA00000D20E46518840F64804A14200D3214687
:102BB000D588A54200D32546A14200D20C464FF449
:102BC000A4721B2E01D0954204D1B8F11B0F3ED048
:102BD00094423CD06A46194609F025FBBDF8060030
:102BE0004146404500D90846F880BDF80810A1428A
:102BF00000D80C463C81BDF80210B14200D80E4608
:102C00007E80BDF80410A94200D80D46BD80FF218A
:102C100039701B38E02802D940F66E5114E01B3E93
:102C2000E02E02D94FF457610EE04FF4E060A4F5B6
:102C3000A474844202D940F6725105E0A5F5A4754A
:102C4000854204D940F674513920F9F7B9FFBDE83F
:102C5000FE8300007C02002010B50D4800210D4BC2
:102C6000C17481821B221A804FF4A4745C809A8004
:102C7000DC808173C173032303700223437042809D
:102C8000828040F6A66282608174017310BD0000EC
:102C9000200F00207C02002010B50121002006F04A
:102CA00095FB04000AD1012106F086FB040007D041
:102CB000064890F90010204607F0DBFC204610BDC6
:102CC0004FF42C713920F9F77BFF000074020020CB
:102CD0002DE9F04387B00C468046054607F037FDE6
:102CE00098B1284607F026FD30B1B4F80110122043
:102CF00000290BD0802909D8284607F00CFD40B1E7
:102D0000404607F077FC30B109E0422007B0BDE84B
:102D1000F0830C20FAE7404607F006FDC8B34046B2
:102D200007F0E5FE0028F4D1404607F07EFC0028BD
:102D3000EFD14046FCF700FBB4F8010042F21071FD
:102D400000FB01F9E178404607F0DCFC404607F063
:102D5000EDFC08B3002101A8FAF790F904007BD03C
:102D60000021FBF7F3FCBDF804002080214640461B
:102D700007F004FD00F0E6F9400940EAC160C00731
:102D8000414D04F12C0011D06988AA88C1840285C4
:102D90000FE0FFE71220B9E74A4600214046FDF761
:102DA000E9F90028B2D041F222615FE01B22C2841F
:102DB000028500F0C7F988074FF0010605D58DF8A8
:102DC000086002A80394FFF745FDA868E06241F699
:102DD0004C57404607F0B2FC10B9404607F0CCFC17
:102DE00027612188ADF80810A97B8DF80A10E97BCE
:102DF0008DF80B10298AADF80C1005A9009130460A
:102E000004AB02AA214609F044FA40B10021BDF802
:102E10000400FAF75BF9F0B141F27C6126E09DF81D
:102E200010008DF818009DF814008DF81900BDF8F9
:102E30000C00ADF81A0006A9204606F012FE6878CC
:102E400000902B78AA8869882088FAF7F5F928B1CC
:102E500041F287610AE0FFE7092057E74A46214629
:102E60004046FDF787F920B141F289613920F9F731
:102E7000A7FE0648436823B1002204F59971204655
:102E80009847002042E70000200F00207402002035
:102E90002DE9F04188B00446008806A906F011FD2E
:102EA000002847D1079890F880118DF808100299F2
:102EB00002919DF80810803001B101218DF80C10AD
:102EC000017B4FF00008890602D59DF80C1049B12E
:102ED0005FF000018DF8041005216C3008F030FC23
:102EE00010B104E00121F5E79DF8040008B3218941
:102EF000E08809F08AF900281CD1A188608809F0CF
:102F000084F9002816D12189E08809F074F9002895
:102F100010D1A188608809F06EF906000AD10798DF
:102F200000F59975FF276F709DF80C1029B13A26AE
:102F30002EE01A2008B0BDE8F081414603AA09F04E
:102F400072F96188BDF81200814200D20846E8801B
:102F5000A188BDF81400814200D208462881E28889
:102F6000BDF80E108A4200D2114669802289BDF850
:102F700010108A4200D2114640F64802A9809142C0
:102F800000D31146A980904200D202462A812F70B8
:102F900085F801803046CDE71CB50C49D1E9020126
:102FA000CDE900010AE0009C204607F0A0FD28B111
:102FB000204607F0F2FB08B101201CBD6846FAF775
:102FC0003DF80028EFD000201CBD000008300100B3
:102FD00010B50446C188808809F017F900280FD180
:102FE0006188208809F011F9002809D10548A188D5
:102FF000818021880180E188C18061884180002032
:1030000010BD00007C020020000000000000010054
:1030100000000000000001000C4B120C59004B1284
:10302000000000000000010000000000000001009E
:1030300010B5FBF72DFE054C606809F0EDF908F0BE
:1030400092FFFBF75FFF0120207010BD840200207B
:1030500001480078704700008402002010B5064C3B
:10306000A06809F0D9F9E06809F0D6F908F0E0FFA6
:103070000020207010BD00008402002010B505491A
:10308000054809F0BCF90448BDE810400349001D9B
:1030900009F0B5B994020020880200209C020020AB
:1030A00010B50849084809F0AAF907480749001D62
:1030B00009F0A5F90448BDE810400549083009F0B9
:1030C0009EB90000AC02002088020020B40200205B
:1030D000A4020020014840787047000084020020CC
:1030E00010B5FCF74BFAFDF7F5F8BDE810400148C4
:1030F000FCF72ABA391600200A4910B50120487099
:10310000FCF76CFAFDF7C2FD06F00DFB0649A1F5D0
:103110008170FAF741FC002006F035F9BDE8104057
:10312000FBF7BCBD840200203B170020044AC10805
:1031300000F0070301209840535C03435354704749
:10314000200000200149D1E9000170472000002043
:10315000064801880079020642EA112000F00100C9
:103160000018C0B240F001007047000020000020AD
:1031700010B504F051FE0022084B114633F82140EF
:10318000844203D303EB8100827803E0491CC9B277
:103190000C29F3D30248027010BD00006AC401007C
:1031A0007303002070B5054616460C46022000F059
:1031B000B7F906490120F61E087005480660044864
:1031C00008380560001F046070BD00007403002013
:1031D00010F5004010B50C4C207880B10B494FF42D
:1031E0000000086000F06AF8002120B10120607042
:1031F0000748006801E061701020A0702170BDE8F0
:103200001040002000F08CB97403002008F5014044
:1032100000F4004010B5022000F082F904490120BA
:10322000087000F059F803494FF40000086010BD21
:103230007403002004F5014003480021017041702F
:10324000102181707047000074030020074810B5FA
:10325000017841B100F032F818B105480068C0B2F9
:1032600010BD102010BD807810BD00007403002038
:1032700000F40040084810B5017859B10748D0F86B
:10328000000128B100F00CF8002800D0012010BD8A
:10329000022010BD407810BD7403002000F00040F3
:1032A0000548D0F8041111B1D0F8080108B1002088
:1032B000704701207047000000F00040054810B53D
:1032C000D0F8000120B1FFF7EBFF08B1012010BDDD
:1032D000002010BD00F0004004480021C0F800119B
:1032E000C0F80411C0F808117047000000F0004059
:1032F0002DE9F04104461E4690460F46012000F09D
:103300000FF91E4D1E4804F003012E7100683204AF
:1033100061F3070066F30F20000C1A4E42EA0060CA
:103320000843C6F804051848076009F0C7FB38B918
:1033300015481030016821F0FF0141EA08010160E1
:1033400000F0E4F80CB1042C07D111480D490F4AE4
:10335000091DC0F81025C0F8141501206870EC7024
:103360001CB1012C01D0022C06D128700021C6F816
:103370000011C6F800123060BDE8F081770300202C
:103380001C35010000F0004008F5004000F100404D
:1033900088F0014070B51C4A5378A3B11B4B1960EB
:1033A000191D0860012595701046D678184B0078D5
:1033B000184C002156B1042E1BD008B3C4F80411D8
:1033C0006806186070BD40F2BD111AE078B1204661
:1033D000C4F804114FF400361E60711209F0BDF8F4
:1033E0000028EFD065600A48001D066070BDB3215B
:1033F00007E01570C4F80411C4F80052256070BDD0
:10340000C6213C20F9F7DCFB770300200CF50040D7
:1034100004F5014000F0004070B5054D0024287807
:1034200010B100F073F82C706C70AC7070BD0000BF
:1034300077030020024800210170417081707047BD
:10344000770300200B4810B5007858B14FF4827113
:10345000094809F082F840B108480068002800D007
:10346000012010BD40F2232101E04FF409713C20FE
:10347000F9F7A6FB7703002000F0004000F40040BD
:10348000014801218160704700F000402DE9F047BC
:103490001B480078D8B1DFF86C804FF48276314653
:1034A000404609F05AF8002828D10220C8F8040341
:1034B000154C2068C04340F30015206840F0100010
:1034C00020604FF400474FF0E0296D1C08E040F207
:1034D0002F213C20F9F774FBC9F8807209F02EFB0C
:1034E0003146404609F039F80028F5D01DB920686A
:1034F00020F0100020600220C8F80803BDE8F08723
:103500007703002000F0004010ED00E00249014880
:10351000086070470000020208F501400000010049
:1035200010B5044600F020F8002C0ED00B4A0B48D2
:103530000B491432012C05D0022C07D082213D20EA
:10354000F9F73EFB02230360116010BD0323036003
:10355000116004494FF40000086010BD00F5004000
:103560003D18002004F50140054810B50021016018
:103570000160FFF751FF03494FF40000086010BDE0
:1035800000F5004008F501400548D0F8001221F090
:103590004001C0F800120021C0F86015704700001B
:1035A000001000400449C1F86005D1F8000240F065
:1035B0004000C1F80002704700100040014890F838
:1035C00022007047840F00200249085C00F5166055
:1035D000704700001E430100F8B5244CD4F80403E2
:1035E00010F0100F01D0012700E000271020C4F8D0
:1035F00008030220C4F800021D4800251D4980F878
:103600002C504FF460200860D4F850054FF48876B1
:1036100010F0FF0F19D0FF208DF80000C4F81051F2
:103620000120206105E000BF9DF80000401E8DF8DC
:1036300000009DF8000028B13146204608F0BCFF8C
:103640000028F1D09DF8000058B100F057FCC4F8F4
:10365000105100F0E5FD002F02D01020C4F8040343
:10366000F8BD40F6AA013E20F9F7AAFA0010004082
:10367000840F002008F501402DE9F041184D074660
:1036800095F82C00C2070FD0164CD4F8002242F057
:103690000102C4F8002240F0020085F82C00012647
:1036A0003FB1012F0BD010E040F285713E20F9F7B9
:1036B00087FA084600F00EFE6E72266005E00846A6
:1036C00000F0EEFD0220687266600748C664064896
:1036D0000C30D0F840153846BDE8F04100F072BD1E
:1036E000840F002000100040008000402DE9F047CA
:1036F0002C4C06002C4D94F82C00DFF8B08040F0E4
:103700000200894684F82C004FF0000702D0012EF9
:1037100020D036E0084600F0DDFD01206072E0793F
:10372000012805D1D5F8000240F00800C5F80002D4
:10373000A06A40F48010A0624FF48010C8F8000026
:103740001B4931F819004FF47A7100F5FA70B0FB9B
:10375000F1F716E0084600F0A3FD02206072E07960
:10376000012805D1D5F8000240F00400C5F8000298
:10377000A06A40F40010A0624FF40010C8F80000E6
:10378000292700F027FC09F091F820B1FFF724FF6A
:103790000020BDE8F0870021304600F013FD3846D8
:1037A000F7E70000840F00200010004004F50140FE
:1037B00018430100024A136B0360506B08607047A6
:1037C000840F002010B51DC8014981E81D0010BDFF
:1037D000740F00200F4910B5CA69824202D340F627
:1037E0003A110BE001220A7308610B494A640A1D71
:1037F000D2F84035834204D340F643113E20F9F716
:10380000DFF90023C1F84431C2F84005BDE810409B
:1038100000F0ACBC840F00200080004070B50F4C5D
:1038200003460220207394F82150962094F820102B
:10383000227D012D0ED000F0ABFD20610848002153
:10384000C0F844112169E06908440549091DC1F81F
:10385000400570BD00F0BAFDEFE70000840F0020C6
:103860000080004010B509F045F9002806D0044852
:10387000016821F0010141F08071016010BD00007C
:10388000741700402DE9F04138220021134809F057
:103890001AFA00F0C5FC09F0E6F8114D104E0024AC
:1038A0000F4F0835103628B909F0F4F810B909F0AF
:1038B000FBF808B1242206E009F036F910B909F046
:1038C00029F940B14022FF21384609F0FCF92C606B
:1038D0003460BDE8F0813822F5E70000840F002055
:1038E000000E00400148C06970470000840F0020AE
:1038F0000148806970470000840F002010B500F077
:1039000043FCFFF769FE04F023FD30B1401C04D0F6
:1039100040F26D513E20F9F753F90F480F4A816A82
:1039200041F044611160002484620473C4618461C5
:1039300000F02AFC0A48C0F84841C0F84441C0F8E9
:103940004041C0F84C41012008F025FEBDE8104080
:10395000012008F013BE0000840F002008F501408C
:103960000080004070B5012008F015FE374C0020A3
:10397000C4F8FC0F0120C4F8FC0F09F0ABF8344D7B
:1039800018B1286840F48060286009F097F828B1E1
:103990002868304920F069000843286009F0AAF837
:1039A00038B12B48001D016821F47F4141F4B0512A
:1039B0000160274928483C31086004F003FD40B10C
:1039C0004FF08050D0F83003411C02D02049103114
:1039D00008604FF01020006E411C04D01F490A6897
:1039E00060F317420A6040F2031140F25B60C4F8D2
:1039F0003415C4F838050120C4F8300500F042F849
:103A000040F20120C4F850060220C4F80002144914
:103A10004FF04060086013490020134D08861031B4
:103A2000C86181F82C002870012008F0A7FD102043
:103A3000C4F804034FF0E0210220C1F800016868D7
:103A4000002802D0BDE87040004770BD0010004063
:103A50003C170040960000802C0000898C15004027
:103A600004F50140740F0020BC0200200149487594
:103A700070470000840F0020014951F82000704772
:103A80006C430100084910B508750849012806D0A3
:103A9000022806D040F686513E20F9F791F803201F
:103AA00000E00420086010BD840F002010150040C5
:103AB0000549C1F80405054810F82C1F41F0010123
:103AC000017000F04DBA000000100040840F00208B
:103AD000014951F820007047784301002DE9F04773
:103AE000304E314C8846070015464FF0010906D08C
:103AF000012F12D040F62D013E20F9F761F8104653
:103B000000F0E8FB294884F8099030F81510404689
:103B100000F08EFB054630460CE0104600F0C0FB7E
:103B20000220607249F6BA71404600F081FB0546FA
:103B30001C48001D00F03AFBDFF87480C8F84055BF
:103B4000DFF874A01B48CAF810051020C6F804035B
:103B5000A06A4FF4002640F40020A06217480660D7
:103B600000F038FA4146C8F84C9011480C30D0F8B3
:103B70004005A84210D30020C1F84005CAF814053A
:103B8000A06A20F40020A0620C48001D0660FFF728
:103B900023FD0020BDE8F0872946384600F012FBDF
:103BA0000120F7E700100040840F002018430100B7
:103BB000008000404081004098F0014004F5014041
:103BC0000D4B10B5D8719A7251B1022018720128AC
:103BD00008D002280FD040F663213E20F8F7F0FF0E
:103BE0000120F3E7587A022805D100F07DF9BDE8FD
:103BF000104000F0B1BA10BD840F0020024900202F
:103C0000C1F8400570470000008000400449D1F829
:103C1000481501F07F014942017001207047000002
:103C2000001000400349020EC1F824250002C1F82B
:103C30001C057047001000400149C1F83C05704761
:103C40000010004010B50022012906D0022902D040
:103C500040F2D92114E04FF080720B490A430B491E
:103C60000A600B4908430949091D08600948D0F852
:103C70005005C0B2032801D00B2804D140F2F12135
:103C80003E20F8F79DFF10BD0801100014150040FC
:103C900000000302001000400149887570470000D1
:103CA000840F00202DE9F04753484FF0010AC0F877
:103CB0004CA051480C30D0F8407508F0F5FD4F4C41
:103CC000C4E90C0700F01AF94D49A06A0860DFF852
:103CD00034810020A062D8F8002240F21D139A43DC
:103CE000C8F8002284F82C0000F088F90546424804
:103CF0000830D0F84005404EE061361DD6F840054A
:103D0000A06194F82100217D84F82010617A84F864
:103D10002110A14600243946284600F0E3F910B9E5
:103D2000C8F810A00124354FE807A7F1100702D00A
:103D30003868804734E0A80729D5680721D408F0FF
:103D4000D9FEF0B908F0C6FED8B92F480068C0F314
:103D50004252C0F3006100F00F0CC0F30313C0F334
:103D6000032871B1BCF1000F03D013B1B8F1000FFB
:103D700007D1C0F30440012803D1032A01D245F042
:103D8000040545F380002146401C7A6807E015F0E1
:103D9000280F05D045F34011BA682046491C9047CA
:103DA000E80601D5F868804799F8091048460229C5
:103DB00020D1017B00291DD0022904D0012909D07E
:103DC00040F666410DE0C169D9F810000844C6F814
:103DD00040050BE00169D9F81C00814204D840F687
:103DE00067413E20F8F7ECFEC6F84015BDE8F04705
:103DF00000F0BCB9BDE8F08700800040840F0020CF
:103E000008F50140001000405014004070B5164BFA
:103E10008C8803EB8005C5F820460C78D1F801109A
:103E200044EA0121C5F80016D3F840160124844065
:103E3000C9B2E5B2294332B1012A0AD040F2D451C5
:103E40003E20F8F7BDFED3F84006C0F30720A0439C
:103E500004E0D3F84006C0F30720284341EA0020DD
:103E6000C3F8400670BD0000001000400149012069
:103E700008707047BC0200200B48817D0B48405CF5
:103E800000F51660B0F5166F04D2A0F6381040F4B5
:103E9000807001E0A0F51660054AC2F8080501F03F
:103EA0007F00C2F854057047840F00201E430100B4
:103EB0000010004008B50B496B4691F91520897D2B
:103EC00000F0D0FA9DF9000000F0A0FA0DF1010019
:103ED00004F062FA002804D040F215613E20F8F7A1
:103EE0006FFE08BD840F00200348017A012902D12A
:103EF000807AFFF7DFBF7047840F00200D4810B5B0
:103F0000407A01280CD0022813D104F027FA0028A7
:103F10000FD0401C0DD040F6C1013E20F8F750FEF6
:103F200004F02EFA002804D0401C02D040F6BB0159
:103F3000F3E710BD840F002008480021C0F80011ED
:103F4000C0F80C11C0F81011C0F80411C0F8141119
:103F5000C0F81811C0F808117047000000100040A8
:103F6000184810B590F82C00C10729D0810714D546
:103F70001548D0F8001241F00101C0F80012D0F845
:103F80005005C0B20B2805D00A2803D0032801D061
:103F9000022815D140F23E610FE0400710D50A48D3
:103FA0000A490830C1F814054FF4A071084808F018
:103FB00008FB002804D040F246613E20F8F700FEDE
:103FC00010BD0000840F00200010004098F0014058
:103FD0000080004008480146C27991F82C1012B1C7
:103FE000012A03D006E041F0020101E041F00401A2
:103FF00080F82C10FFF7B4BF840F00202DE9F041AA
:10400000344D0024287B38B14FF4A271324808F0B7
:10401000D8FA08B1012600E00026687A2F4F4FF445
:104020008671012802D0022806D016E0384608F032
:10403000C3FA90B1082410E0384608F0BDFA00B188
:104040000224D7F80004C04340F30000401C01D113
:1040500044F004040EB144F0010414F00B0F07D136
:104060004FF48871384608F0A7FA08B144F01004FC
:104070001B480078F8B1D7F8400610F0FF0607D0CB
:104080004FF48A71384608F097FA08B1012000E031
:10409000002085F822003EB14FF48C71384608F0BC
:1040A0008BFA08B1012000E0002085F82300D7F842
:1040B000100485F82400FFF73FFFE00606D520072F
:1040C00004D4687A012801D144F020042046BDE8D8
:1040D000F0810000840F00200080004000100040AC
:1040E000BC0200202DE9F0411A4C0D46217A29B17D
:1040F00010F0110F07D0FFF76FFA24E000F090F8EE
:10410000002020731FE0012901D0012600E00026D5
:10411000E07901280ED0002700F082F89621304681
:1041200000F094F801464FB13B358D4204D9002090
:10413000BDE8F0810127EFE70120E071A27A304667
:10414000FFF7CCFC08B10120F2E740F6C4213E2085
:10415000F8F736FD840F00200348D0F8001241F430
:104160008871C0F800127047001000400448816A4E
:1041700041F48001816203494FF480000860704778
:10418000840F002004F50140074A00200832064948
:10419000C2F840050A1DC2F84005C1F840050249B1
:1041A0000C31C1F840057047008000400349C979CF
:1041B000002902D10249C1F814057047840F00207C
:1041C00098F0014010B5144A20B1012811D040F2F6
:1041D00069711CE001F12800C2E902100F490E4884
:1041E00004F0D4F8002815D0401C13D04FF4EB6134
:1041F0000DE001F12900C2E902100849064804F067
:10420000B3F8002806D0401C04D040F265713E206F
:10421000F8F7D6FC10BD0000C4020020484301009E
:1042200002480021C171017241727047840F002061
:10423000054AD279012A06D04FF47A7201F5FA7153
:10424000B1FBF2F1401A7047840F002070B5134C97
:1042500003460D4694F8212000205AB1214691F8DA
:10426000201063B1012B11D1012A284612D008F089
:10427000ADF909E040F66E013E20F8F7A1FC012AF5
:10428000284604D008F0B0F9E169084470BD00F098
:10429000D1F8F9E700F0C0F8F6E70000840F00203D
:1042A00010B5FFF7EFFBFFF7E7FDFFF71DFEFFF788
:1042B00053FF08F01FFC002808D108F00BFC002871
:1042C00004D10348016841F4C021016010BD000021
:1042D0006815004010B50446FFF7D4FBFFF7CCFD8E
:1042E0002046FFF7E7FD08F005FC00280DD0094A3D
:1042F00011685006022CD0F8200307D0C0F3062026
:1043000021F4FE4141EA0020106010BDC0F30660B8
:10431000F6E700008815004000002CA6E0A1040686
:10432000080A0C0E10121416181C1E20222426280F
:104330002A2C2E30323436383A3C3E4042444648ED
:104340004A4C4E021A5000000100000010110040BB
:10435000000000000000000000000000000000005D
:1043600000000000141E00003011000000000000DA
:10437000280000001800000000000000141E0000CB
:10438000301100000000000070170000A00F0000B6
:1043900070B5054614460846FFF79AFB05EB450144
:1043A000C1EBC511C0EBC101074850F82400084417
:1043B0004FF47A7100F6B730B0FBF1F52046FFF705
:1043C0005BFB2844401D70BD5844010070B50E4D84
:1043D0001C46083D0C4B35F8111000EB400553F816
:1043E0002230C5EBC01001EBC00003F6B733184410
:1043F0004FF47A71B0FBF1F51046FFF73DFB28440E
:104400002044401D70BD0000584401000149C0B265
:10441000086070470C150040054A32F811104FF43F
:104420007A7201F2E731B1FBF2F10844801E704765
:1044300050440100054A32F811104FF47A7201F528
:104440007A71B1FBF2F1084470470000504401005A
:104450000000DC05E803000000000000141E00005E
:10446000301100002DE9F8431E4617460C4605465C
:1044700000F056F8DFF8A490804699F80000A842B2
:1044800010D199F801104846A1420BD190F90210C1
:10449000B94207D1C278424504D181883180807900
:1044A000B07037E03A462146012D09D0022D09D0DF
:1044B000042D09D0082D09D040F2624106200CE0FD
:1044C000002004E0012002E0032000E002206B460F
:1044D00000F09EF818B13D217520F8F771FB2046D9
:1044E000FFF772F80246002331469DF9000003F001
:1044F0005FFF014689F807103188A9F80410B178E8
:1045000089F8061089F8005089F8014089F802708E
:1045100089F8038099F90700BDE8F8837C0300203F
:104520000148007870470000DC02002070B5174C8D
:104530006078002823D10120607008F0B5FA6FF090
:10454000270528B908F0E6FA10B908F0EDFA20B10D
:104550000F486060A570082010E008F07AFA40B9B2
:1045600008F081FA28B908F095FA10B908F0A6FA0F
:1045700030B1074831306060A5700420E07070BD34
:1045800040F23F11742003F053FD0000DC020020D4
:1045900049CE0100064A00B592F90320904201DBA2
:1045A000104600BD00F008F80249085600BD0000A2
:1045B000DC0200203BCE01000246134810B590F902
:1045C00003309A4201DB0D2010BD90F902309A426F
:1045D00001DC002010BD01B10121D41A4368185D2F
:1045E0000A4C24569442F5D0084C08443F34C0B2DB
:1045F000D2B2A342EED10029ECD0012A01D0022A86
:10460000E8D1401CC0B210BDDC0200203BCE01004E
:104610002DE9F0411C4690460D4606466FF0150701
:10462000042804D81CB107F0EAFFA84202D8384693
:10463000BDE8F0810548424650F8260018B14057C1
:10464000824200DD024622700020F1E7BC0F00200C
:1046500070B50D4604000CD094F8286000210220AB
:10466000092D6ED2DFE805F008113636667189A68D
:1046700094004FF4CB71F7E094F8260004287BD027
:104680000328FCD040F2A111EEE094F826000428A3
:1046900004D0032802D040F2A511E5E0052084F8FB
:1046A000260084F8291094F82400B8BB0021204685
:1046B00008F006F82078012807D0D4E9040100BFEB
:1046C000C4E906010021226A48E094F8270001F0BD
:1046D000C7FAF5E794F82610042904D0032902D07C
:1046E00040F2C311C0E094F8242022B121463046A4
:1046F00008F026F8B0E0042900D0012084F8260054
:10470000226A022D0BD006213046904700286DD03A
:10471000007800286AD040F2DD11A5E034E00521E0
:1047200030469047002870D0007800286DD04FF4B4
:10473000EC7199E094F82600052803D04FF4F2714B
:1047400092E080E00221226A08E094F82600052821
:1047500002D04FF4F57187E0226A0121304690477C
:104760000146204607F057FF022875D0E8B301281C
:104770006CD040F22A2177E070E094F826000528FA
:1047800002D04FF4F8716FE0BDE8704000F09EB8C1
:1047900094F82600052802D040F2F51164E0226A60
:1047A0000A21304690470146204607F034FF4FF477
:1047B000FC7159E094F82620052A07D094F825309A
:1047C0000BB1032A02D04FF4FE714DE094F824207F
:1047D0002AB121463046BDE8704007F0B1BF94F8D9
:1047E00029209AB184F8291001E032E034E084F8FD
:1047F0002600226A082130469047002837D00078EA
:10480000002834D04FF402712EE030E094F82520D7
:104810005AB184F8251094F82700214607F04EFF7E
:10482000002824D140F20D211EE084F82600226ADF
:10483000072130469047002819D00078002816D06C
:104840004FF4057110E040F219210DE00421226AB5
:1048500084E70321226A81E7002D08D108F026F8B9
:10486000002804D040F233216A2003F0E1FB70BD40
:10487000002819D003781349134A13B1012B0ED025
:1048800011E00379012B00D06BB943790BB1012BF7
:1048900009D18368643B8B4205D2C0680EE003797E
:1048A000012B02D00BB10020704743790BB1012BD3
:1048B000F9D1C368643B8B42F5D280689042F2D84C
:1048C000012070473D860100FF3F420F10B5054CA7
:1048D000206810B1804700202060BDE8104002F041
:1048E00085B80000E40200202DE9F0410E460500E5
:1048F00004D000F047F8074600240BE06FF01500E5
:10490000BDE8F081204600F043F890F8260030B171
:10491000641CE4B2BC42F5D36FF00B00F0E727460D
:10492000FF2CF9D0204600F033F8044607F023FFAF
:1049300084F828702146084802F030F884F82700EF
:10494000202806D00120256284F826003770002038
:10495000D6E76FF02200D3E75146010010B5820779
:1049600002D06FF00D0010BD054A1170506028B1E3
:1049700001EB41010A01002108F0A5F9002010BD5A
:10498000E80200200148007870470000E80200209B
:1049900005490A78904201D300207047496800EB2E
:1049A000400001EB00107047E80200200E4910B5EE
:1049B00091F83200202812D091F83200A1F58062DF
:1049C000C0EBC00002EB800091F832104068C1EBF0
:1049D000C10152F82120BDE810400421104740F6E3
:1049E000BC01702003F024FBD013002070B50546F5
:1049F000202A28D019481A4C00EB831C03EB4303F0
:104A00000CEB42002344202922D00CEB41014078DA
:104A10004C784870204601460CEB410091420570ED
:104A20004078F8D193F82220202A1ABF0CEB4202DA
:104A3000547083F8214020220CEB410C8CF80120AB
:104A400083F8221070BD4FF42671702003F0F0FA45
:104A500093F82040407883F82000DBE750130020D3
:104A6000D01300202DE9FF4F8DB015460C4602F003
:104A700009FA284420F07F4008902168081A0002B3
:104A8000C11700EB11600012002800F3F080DDF880
:104A90004080CD4808EB48010844099090F8205028
:104AA0002020CA4E0DF1180A0DF11C098DF81800CE
:104AB000202D1CBFC64800EB881B38D0C5EBC500B5
:104AC00006EB800000F10801C0682768381A000270
:104AD000C21700EB1260001229D4E08900B3C88924
:104AE000F0B90868039003F0E5F8B0F5C67F08BF99
:104AF0000D200BD0A0F54070563808BF1C2005D003
:104B0000A0F500709F3814BF00203220411C03988C
:104B1000381A0002C21700EB12600012884206DB4E
:104B20000BEB45008AF800504578202DC6D19AF845
:104B3000000089F80000202D1CBFA54800EB881B51
:104B400000F03E81C5EBC50006EB80076168D7F831
:104B5000088007F10800A8EB01010902CA1701EB60
:104B60001261091227D4C089002800F02981E08948
:104B7000002840F02581D4F800A003F09BF8B0F5A0
:104B8000C67F08BF0D200BD0A0F54070563808BF77
:104B90001C2005D0A0F500709F3814BF00203220E3
:104BA000411CA8EB0A000002C21700EB12600012C1
:104BB000884280F2058189F80050387E217C884245
:104BC00006D90BEB45004578202DBBD100F0F8B895
:104BD0009DF81C00C0EBC00006EB8000C18AC568D0
:104BE000E1BBE189D1B3876803F064F8B0F5C67F13
:104BF00008BF0D200BD0A0F54070563808BF1C2010
:104C000005D0A0F500709F3814BF00203220411C51
:104C1000E81B0002C21700EB1260001288421DDA86
:104C200003F048F8B0F5C67F08BF0D200BD0A0F503
:104C30004070563808BF1C2005D0A0F500709F3882
:104C400014BF002032209DF81C10401CC1EBC10194
:104C500006EB81018968084420F07F450898281AEE
:104C60000002C11700EB11600012002803DD11B033
:104C70000020BDE8F08F2068A84202D9A168491C35
:104C8000A16061680DF1180A081A284425F07F41D7
:104C900020F07F40C4E9001010980B9009980DF1A6
:104CA0001C0890F8205020208DF81800202D3CD0B2
:104CB00047490B9801EB801BC5EBC50006EB800054
:104CC00000F10801C0682768381A0002C21700EB1B
:104CD0001260001229D4E08900B3C889F0B9D1F874
:104CE000009002F0E7FFB0F5C67F08BF0D200BD0A3
:104CF000A0F54070563808BF1C2005D0A0F5007004
:104D00009F3814BF00203220411CA7EB090000028D
:104D1000C21700EB12600012884206DB0BEB450065
:104D20008AF800504578202DC6D19AF8000088F8FE
:104D300000000B98202D1CBF254901EB801B3FD0A4
:104D4000C5EBC50006EB80076068D7F8089007F14F
:104D50000801A9EB00000002C21700EB126000126C
:104D600022D4C88960B3E08950BBD4F800A002F017
:104D7000A1FFB0F5C67F08BF0D200BD0A0F5407095
:104D8000563808BF1C2005D0A0F500709F3814BF0E
:104D900000203220411CA9EB0A000002C21700EBE0
:104DA0001260001288420BDA88F80050387E217CAD
:104DB00088427FF60DAF0BEB45004578202DBFD123
:104DC00011B00120BDE8F08FD0130020D00F0020DB
:104DD000501300202DE9F84F0F46064601EB47001F
:104DE0004B4999460844924690F820402020107084
:104DF000A1F58068202C1CBF464800EB871B38D0EB
:104E0000C4EBC40008EB800000F10801C0683568FD
:104E1000281A0002C21700EB1260001229D4F08990
:104E200000B3C889F0B90868009002F043FFB0F5FC
:104E3000C67F08BF0D200BD0A0F54070563808BFC4
:104E40001C2005D0A0F500709F3814BF0020322030
:104E5000411C0098281A0002C21700EB12600012D1
:104E6000884206DB0BEB44008AF800404478202C93
:104E7000C6D19AF8000089F80000202C1CBF2548F4
:104E800000EB871A40D000BFC4EBC40008EB8007DA
:104E90007068BD6807F10801281A0002C21700EB0C
:104EA0001260001222D4C88970B3F08960BBD6F8B2
:104EB00000B002F0FFFEB0F5C67F08BF0D200BD09A
:104EC000A0F54070563808BF1C2005D0A0F5007032
:104ED0009F3814BF00203220411CA5EB0B000002BC
:104EE000C21700EB1260001288420DDA89F8004008
:104EF000387E317C884202D80020BDE8F88F0AEB6A
:104F000044004478202CBFD10120BDE8F88F000078
:104F1000D0130020501300202DE9F74F98B015460C
:104F200002F072FA044602F0EDFC064619980128D8
:104F300018BF022805D040F692114FF0700003F020
:104F400077F8FA4901200860F9498968086000206B
:104F50008DF846000A90401E0B90F649C5EBC5003F
:104F600001EB8001D1E90203D1E904C2CDE90C03D0
:104F7000CDE90EC28969109107F0AAFC0246BDF87E
:104F80003E809DF83C00EC4B4044411C50189A4236
:104F900054D8EA4DA94258DC6A4291425DDB591C63
:104FA0008142DCBF00F5F700A0F1F85005DD0028D4
:104FB000BCBFA0F5F70000F1F8501490E048B8F13C
:104FC000000F808BADF8440014BF4FF0010A4FF082
:104FD000000A02F0B5FF1690BAF1000F08D0D848C9
:104FE000C06AB0F1FF3F02BF16980028012701D028
:104FF0004FF0000702F05EFEB0F5C67F08BF0D203F
:105000000BD0A0F54070563808BF1C2005D0A0F585
:1050100000709F3814BF002032204FF00009CB46AB
:105020001390464536D9149BDFF80C936FEA060CB3
:10503000694617AA03EB0C004B4504D940F29E5178
:10504000702002F0F5FFAC4504DD40F29F51702066
:1050500002F0EEFFBB4B9C4504DA4FF4B4617020C4
:1050600002F0E6FFB84B8342DCBF00F5F700A0F189
:10507000F85005DD0028BCBFA0F5F70000F1F8509E
:1050800001F01CFF00980C9920F07F400090081A56
:1050900020F07F49002F18BFDDF84CB005D19DF8F6
:1050A0004400002818BF4FF0020BB4F1807F08D0F5
:1050B0000C98001B0002C11700EB116000120128C0
:1050C00002DA0320189D0DE057B19D4890F830009A
:1050D00030B19DF8440010F1000B18BF4FF0020BE7
:1050E0002546002083440C98A0EB090020F07F4166
:1050F000481E20F07F40421B1202D31702EB1362BE
:1051000012125A4504DBB9F1000F18BF0C912DE0C3
:10511000B9F1000F05D09DF8450020B902F0E8FB79
:1051200008B1AFB90CE02FB99DF84400002818BFB2
:10513000ABF1020B4FF000098DF844904E4607E0AA
:105140009DF8440020B100208DF84400ABF1020B23
:105150000C98A0EB0901481E20F07F40421B120270
:10516000D31702EB136212125A457DDB744AD26ADE
:10517000891A0902CB1701EB1361169B09123BB97F
:10518000B2F1FF3F1CBF139A9142B8BF002100DB70
:1051900001213AEA010167D1199905464FF000094A
:1051A000059101F0F5FF281A0002C11700EB11600C
:1051B0004FEA202B02F07EFDB0F5C67F08BF0D2020
:1051C0000BD0A0F54070563808BF1C2005D0A0F5C4
:1051D00000709F3814BF002032200B3058451FDD6F
:1051E0000598012801D047B112E0B4F1807F1CD1AD
:1051F00040F61311702002F01BFFB4F1807F07D03E
:10520000601B0002C11700EB11600012042804DDCE
:105210002C46204601F0E2FF07E0002863DC04E0B2
:105220002C46204601F0DAFFD146B4F1807F55D0FC
:105230000C980D9A001B121B20F07F4022F07F4239
:10524000012850D3B0F5000F98BFB2F5000F4AD82F
:10525000204607F03DFB1499384A0D1A4FF0000B19
:10526000AA1A7BF1000200E03DE016D3334A431A4C
:105270009A1A7BF1000210D32F4AAA423EBFC0F512
:10528000902000F1F450451807D39A422FD2C1F56F
:10529000902101F1F45108444542294FB87F58B399
:1052A0001998012805D0022002F0E8F9012002F047
:1052B000E5F9B0452CD2A5EB06014FF0020002F053
:1052C00027F990B3B8F1000F1CBFA5EB080101202E
:1052D00044D000BF02F01CF938B33FE040F6312162
:1052E000702002F0A5FE1BB00020BDE8F08F40F654
:1052F0000531702002F09CFEB04534BF3046404678
:105300001E30A842CCDB40F64521702002F090FE12
:105310001CD9A5EB0801012002F0FAF828B1002EF3
:105320001CBFA91B022019D0D4E742E008050040A9
:10533000F0020020D00F0020FF7F841E0040420FAB
:10534000D013002000C0BDF00080841E56EA080083
:1053500004D040F67611702002F06AFE2946002043
:1053600002F0D6F828B30126BAF1000F04BF97F86F
:105370003000002802D0B9F1000F24D0F86AB0F153
:10538000FF3F04D002F09CFC4FF0FF30F862B9F10F
:10539000000F1CD01398201A20F07F41052002F046
:1053A000B7F860B397F83000002808BF87F830607E
:1053B00015E0022002F062F9012002F05FF91BB053
:1053C0000020BDE8F08FF86AB0F1FF3F12D097F8E7
:1053D000300020B1052002F051F987F830B0A5EB7C
:1053E0000800A0F1190100290EDC40F66E217020A2
:1053F00002F01EFE02F080FC01F0CAFEC6E74FF488
:105400003E71702002F014FE032002F081F8C0B15A
:105410000E488068C0F800B00D48C0F800B00AAC73
:1054200094E80F0038607960BA60FB600EAC94E8D5
:105430000F0038617961BA61FB611BB00120BDE8E2
:10544000F08F40F67621702002F0F2FDF00200208D
:10545000080500402DE9FF4F14460D464FF0000AA5
:105460000A89514662F31F41AA7AD14662F30709BD
:10547000EA7A064662F30F292A7883B04068C4F8B6
:1054800000A062F31749C4F804A0C4F81090C4E95E
:1054900002019D4F7068A0FB0789306807F018FA79
:1054A00010EB08014AEB090228784FEA6709C9F1B5
:1054B000000B70B1E08994F81180C043D5F804A0C6
:1054C00004F10C0248457CDD40F29F51702002F04F
:1054D000AFFDDFF838C2D5E9040311EB0C0A42F145
:1054E000000CB0EB0A0A73EB0C0C72D2411A73EB8E
:1054F00002016ED3B0EB0806B7422BD8E089A6F1C3
:10550000F458A8F59028C143814A08EB01004245B0
:105510002BD34945D8DC594566DB8742DCBF00F513
:10552000F700A0F1F85005DD0028BCBFA0F5F7009A
:1055300000F1F8506A4601A901F0C0FCE0899DF82D
:105540000010301A401A401EB84202D3A068401C16
:10555000A0604646E0896E4BC1436D6894F81180A7
:10556000701804F10C029E4204D940F29E51702042
:1055700002F05EFD4945A7DC594535DB8742DCBFBB
:1055800000F5F700A0F1F85005DD0028BCBFA0F53C
:10559000F70000F1F850214601F090FC206820F05F
:1055A0007F417019401C2160B8F1000F08BF7A30AC
:1055B00004D0B8F1010F08BF48303AD101F062FCC5
:1055C00001E00EE005E020F07F40606007B0BDE83C
:1055D000F08F3068401E20F07F40206000F57A7028
:1055E000F3E70146584504DA4FF4B461702002F045
:1055F0001FFD8742DCBFA1F1F450A0F5902005DD2E
:105600000028BCBF01F1F45000F59020214601F0C4
:1056100055FC2068B8F1000F20F07F410AF101002D
:10562000216008BF7A3009D0B8F1010F08BF4830B7
:1056300004D040F23961702002F0FAFC01F022FC43
